:100000000C948A280C94BB280C94BB280C94BB2815
:100010000C94BB280C94BB280C94BB280D94F311B2
:100020000C94BB280C94BB280C94BB280C94BB28C4
:100030000C94BB280C94BB280C94BB280D948D9475
:100040000C94BB280C94BB280C94BB280C94BB28A4
:100050000C94BB280C94BB280C94BB280C94BB2894
:100060000C94BB280D9493120D94C2120C94BB28CF
:100070000C94BB280C94BB280C94BB280C94BB2874
:100080000C94BB280C94BB280C94BB280C94BB2864
:100090000D94FD120D942C130C94BB280D94C816CE
:1000A0000C94BB280D94BA940C94BB280C94BB28D8
:1000B0000C94BB280C94BB280D94E7940C94BB289B
:1000C0000C94BB280C94BB280D94121D0D9467133F
:1000D0000D9496130C94BB280C94BB280C94BB284D
:1000E0000C94BB28632C682C6D2C722C772C7C2CE8
:1000F000812C862C8B2C902C952C9A2CA52C9F2C0B
:10010000216A246A276A2A6A2D6A306A336A366A43
:100110003A6A126EBF6DFA6DC86DDC6DFA6D126EC3
:10012000FA6D126EFF6DC26EDE6ED16F02704C7092
:100130009D70AA70E6706F71A0727E7396739E7345
:1001400086738E73A673EE73CE73C673BE73D67347
:10015000DE73E673AE73B67333740874F673197492
:100160002074277433742E74FF8CF78C078D0C8DDC
:100170003D8D278D4D8D1C8D328D488D548D5F8D1D
:10018000F08D6C8DDE9D98A0429EF79D109E539E33
:10019000869E98A0749F3F9F98A0DB9E98A0759E16
:1001A00098A098A08C9FA59FBE9F98A0299EF49E82
:1001B000269F98A0529F649E98A00D9F98A0D79FBD
:1001C000E89FF99F98A0A89EB99ECA9E979E12A0EC
:1001D00042A0639F5BA066A184A199A19CA3F8A102
:1001E00060A2CFA10DA29CA39CA39CA39CA39CA3B3
:1001F0009CA39CA39CA39CA39CA39CA39CA39CA307
:100200009CA39CA39CA38EA286A696A69FA6A9A605
:10021000D9A7EAA6D9A7D9A784A78DA798A79CA6EE
:10022000A0A7D9A7B2A7BBA7CAA702AF20AF25AF87
:100230002CAF31AFA1BB38AFA1BBA1BBA1BB3DAFC0
:1002400044AF49AF1E26DA2596276A265A2860252C
:1002500000268C26FE26802580258227822782275D
:10026000E624E624E624BC2590269026C827062707
:100270000827C0270427AE25A426B62782265228A1
:100280006E259A27EA27F225A2254A276626F62711
:10029000F4252226222512277A25942478250A2857
:1002A0007A270626D024D025A227D0263428A026B7
:1002B000DA246E27D6273827B226B2254C26AE265A
:1002C000D4273228A4246E2648258026AE24C625AD
:1002D0007C267E257E2830267E2628269426D0273A
:1002E0001425BA256227F02754258E24E226722889
:1002F000CE276A289C264227D4253E272025702514
:10030000C2270C286225A427802716276C251427CE
:10031000BC24B6241427BC24B6241427BC24B62439
:100320000A25642764270A250A25642764270A25E5
:100330000A250A250A25B22408264E26AA264E2674
:100340004E26CA2410254E264E2698260A26C22658
:100350004E264E264E264E264E264E264E264E26FD
:100360004E264E264E2676254E264E264E264E26C6
:100370004E264E264E263225C6244E264028E626F8
:100380004E2670284A284E264E264E264E268A2570
:100390006E286E28BC2796250C2788268225642582
:1003A000BA24BE27036EDB363D9A9999993DABAAD4
:1003B000AA2A3E000000803F084AD73B3BCE016E90
:1003C00084BCBFFDC12F3D6C74319ABD56833DDAAC
:1003D0003D00C77F11BED9E4BB4C3E916BAAAABEBB
:1003E000000000803F072C7AA5BA6CC590DA3B93D9
:1003F00065FC8BBC53F810FD3C5692834DBD879D28
:100400003AB63DCBC9BF5BBE73DA0FC93F05A84CF6
:10041000CDB2D44EB93836A9020C50B991868808AD
:100420003CA6AAAA2ABE000000803F08000000BE29
:10043000922449123EABAAAA2ABECDCCCC4C3E0097
:10044000000080BEABAAAAAA3E00000000BF0000C8
:1004500000803F0000000000084178D3BB4387D1F3
:10046000133D190E3CC3BD4282AD2B3E68EC827633
:10047000BED98FE1A93E4C80EFFFBE01C4FF7F3F94
:1004800000000000000664EC1B3C04BC163E3BE58B
:10049000B93CC93C37C29E5A3D660498083EEA6999
:1004A000AAAA3E000000803F0253595349445F53BB
:1004B000575F4D5245560000000000BF0600000087
:1004C000000153595349445F53575F5459504500F5
:1004D00000000001C1060000204102535953494465
:1004E0005F544849534D41560000000070C2060059
:1004F00000803F0253595349445F4D5947435300CD
:10050000000000000071C40600007F430153455203
:1005100049414C335F42415544000000000072C61F
:1005200006000064420154454C454D5F44454C4132
:100530005900000000000073C706000000000252CE
:10054000544C5F414C5400000000000000000000CB
:10055000A0C8060080BB4401534F4E41525F454E38
:1005600041424C45000000000094CA060000000013
:1005700001534F4E41525F54595045000000000056
:1005800000009ACB060000000004534F4E41525F1A
:100590004741494E000000000000001ECC06CDCCB3
:1005A0004C3F0146535F424154545F454E41424CDB
:1005B00045000000C1D006000000000446535F4221
:1005C0004154545F564F4C54414745000097D10663
:1005D000000028410446535F424154545F4D414856
:1005E00000000000000025D5060000000001465371
:1005F0005F4750535F454E41424C4500000000C3E9
:10060000D9060000803F0146535F4743535F454E84
:1006100041424C4500000000C6DA0600000000021E
:100620004750535F48444F505F474F4F44000000CE
:100630000023DB0600004843014D41475F454E4122
:10064000424C450000000000000092DD06000080E2
:100650003F01464C4F575F454E41424C450000001C
:1006600000000096DE060000000001535550455280
:100670005F53494D504C4500000000009BDF0600D1
:100680000000000252544C5F414C545F46494E41B9
:100690004C00000000A3E00600000000015253538C
:1006A000495F50494E00000000000000000018E3C0
:1006B00006000080BF0157505F5941575F424548CF
:1006C0004156494F5200001AE4060000004001570D
:1006D000505F544F54414C000000000000000000E7
:1006E000D3EB06000000000157505F494E444558C7
:1006F000000000000000000000D4EC060000000034
:1007000002434952434C455F52414449555300000E
:100710000000D7ED060000204104434952434C45F8
:100720005F524154450000000000001DEF0600002C
:10073000A0410352544C5F4C4F49545F54494D45BE
:1007400000000000A2F30600409C45024C414E44CC
:100750005F535045454400000000000000D9F706F3
:10076000000048420250494C4F545F56454C5A5F76
:100770004D41580000001CF90600007A430254481D
:10078000525F4D494E00000000000000000000B420
:10079000FB0600000243025448525F4D41580000DE
:1007A0000000000000000000B5FD0600007A4401D2
:1007B00046535F5448525F454E41424C450000004D
:1007C00000B6FF06000000000246535F5448525F27
:1007D00056414C55450000000000B8000700C073AA
:1007E00044025452494D5F5448524F54544C4500B2
:1007F000000000B902070000E143025448525F4D77
:10080000494400000000000000000000C20407008E
:1008100000FA4301464C544D4F444531000000005E
:100820000000000000C806070000000001464C540C
:100830004D4F444532000000000000000000C90791
:10084000070000000001464C544D4F444533000062
:1008500000000000000000CA080700000000014678
:100860004C544D4F4445340000000000000000008F
:10087000CB09070000000001464C544D4F4445355C
:10088000000000000000000000CC0A07000000008B
:1008900001464C544D4F4445360000000000000016
:1008A0000000CD0B07000000000153494D504C459E
:1008B0000000000000000000000000CE0C07000057
:1008C0000000024C4F475F4249544D41534B0000DA
:1008D00000000000140D0700804F44014553430001
:1008E00000000000000000000000000000BA0F0738
:1008F000000000000154554E4500000000000000BB
:10090000000000000000BB1007000000000254556A
:100910004E455F4C4F57000000000000000000BD36
:100920001307000000000254554E455F48494748F0
:100930000000000000000000BC110700007A440124
:100940004652414D4500000000000000000000003C
:10095000009515070000803F014348375F4F505412
:1009600000000000000000000000981607000000D2
:1009700000014348385F4F50540000000000000061
:100980000000001F1707000000000141524D494EB2
:10099000475F434845434B00000000002018070014
:1009A00000803F02414E474C455F4D4158000000DA
:1009B000000000000022E50600A08C4503414E47E0
:1009C0004C455F524154455F4D415800000026E7B9
:1009D0000600A08C46085243315F00000000000072
:1009E00000000000000000AA1907B64600000852E7
:1009F00043325F0000000000000000000000000023
:100A0000AB3607B6460000085243335F00000000D3
:100A1000000000000000000000AC5307B6460000D4
:100A2000085243345F000000000000000000000096
:100A30000000AD7007B6460000085243355F000065
:100A40000000000000000000000000AE8D076B46B3
:100A50000000085243365F00000000000000000064
:100A600000000000AFAB076B460000085243375F41
:100A700000000000000000000000000000B0C907F6
:100A80006B460000085243385F0000000000000081
:100A9000000000000000B1E7076B46000008524369
:100AA00031305F000000000000000000000000B2D4
:100AB00005086B46000008524331315F000000001A
:100AC0000000000000000000B323086B4600000295
:100AD00052435F53504545440000000000000000B1
:100AE00000C041080000F543044143524F5F52509B
:100AF0005F500000000000000000DD43080000908F
:100B000040044143524F5F5941575F50000000007D
:100B1000000000F4470800009040044143524F5F3A
:100B200042414C5F524F4C4C00000000F24B080019
:100B300000803F044143524F5F42414C5F50495453
:100B40004348000000F34F080000803F014143523A
:100B50004F5F545241494E455200000000001B5364
:100B60000800000040014C45445F4D4F44450000E3
:100B7000000000000000009EE20600001041085244
:100B80004154455F524C4C5F0000000000000000E3
:100B9000DF5408AB2C000008524154455F504954C3
:100BA0005F0000000000000000E06E08AB2C0000B9
:100BB00008524154455F5941575F00000000000052
:100BC0000000E18808AB2C0000084C4F4954455206
:100BD0005F4C41545F000000000000E7A208AB2C0E
:100BE0000000084C4F495445525F4C4F4E5F000087
:100BF00000000000E8BC08AB2C0000085448525F1D
:100C0000524154455F0000000000000000ECD6088F
:100C1000AB2C0000085448525F414343454C5F00F1
:100C2000000000000000F1F008AB2C0000084F4667
:100C30005F524C4C5F00000000000000000000ED1F
:100C40000A09AB2C0000084F465F5049545F000072
:100C50000000000000000000EE2409AB2C0000089A
:100C60005354425F524C4C5F0000000000000000F3
:100C700000E25A09D72D0000085354425F504954EE
:100C80005F000000000000000000E36809D72D00AD
:100C900000085354425F5941575F000000000000B4
:100CA000000000E47609D72D0000085448525F4147
:100CB0004C545F000000000000000000EB8409D7E6
:100CC0002D000008484C445F4C41545F0000000078
:100CD0000000000000E53E09D72D000008484C4404
:100CE0005F4C4F4E5F000000000000000000E64C2B
:100CF00009D72D00000852454C41595F0000000003
:100D0000000000000000000D54114843000008439B
:100D10004F4D504153535F000000000000000000A1
:100D2000938B0F7933000008494E535F0000000099
:100D3000000000000000000000031B0B9C3E0000B0
:100D400008494E41565F000000000000000000000E
:100D5000000064970B513E00000857504E41565F0B
:100D6000000000000000000000000065210E282D9A
:100D70000000085352305F00000000000000000037
:100D8000000000006E790D850E0000085352335F9D
:100D9000000000000000000000000000006FCB0D0C
:100DA000850E000008414852535F0000000000001B
:100DB0000000000000009FAD093B2E0000084241EA
:100DC00054545F00000000000000000000000024F8
:100DD00094069132000008474E445F000000000076
:100DE00000000000000000000B060F4E2F0000085E
:100DF00053434845445F000000000000000000002D
:100E0000000C96097A4300000846454E43455F00B2
:100E100000000000000000000000459D05FC2B00C4
:100E20000008475053474C495443485F00000000B6
:100E3000000000467010C73C0000084D4F545F0092
:100E40000000000000000000000000005AA90CC3D0
:100E50004100000852434D41505F00000000000077
:100E60000000000000C75911CB4200000000000044
:100E70000000000000000000000000000000000072
:100E8000000000000002005241575F53454E5300DE
:100E9000000000000000000032000000000002011D
:100EA0004558545F535441540000000000000000B6
:100EB00000340000000000020252435F4348414EEC
:100EC00000000000000000000000360000000000EC
:100ED00002035241575F4354524C0000000000008F
:100EE0000000003800000000000204504F53495435
:100EF000494F4E0000000000000000003A000000D2
:100F00000000020545585452413100000000000025
:100F100000000000003C000000000002064558549C
:100F200052413200000000000000000000003E00BE
:100F300000000000020745585452413300000000F1
:100F40000000000000000040000000000002085007
:100F50004152414D5300000000000000000000001D
:100F600042000000000000FF000000000000000040
:100F700000000000000000000000000000000088E9
:100F8000690200C20128A502008403B5480100904F
:100F9000019F990A00D002DDA70A003200FEAD0AC7
:100FA000000A0003400A008C00CD350A00E803ADBA
:100FB000A00A0020033E9D21005A00DF360200A453
:100FC00001BE280200FA00FF3F02006400ECAC649E
:100FD00000A40101770A0014001CBD02002602F6DD
:100FE0007464009600F3740200D002C6750200B665
:100FF00003BF280200C20164480A000401494802F4
:1010000000DC00256CE803C800B4360A003200504A
:101010004552463A2025752F257520256C750A0006
:1010200050726541726D3A205243206E6F74206396
:10103000616C696272617465640050726541726DC1
:101040003A204261726F206E6F74206865616C7423
:1010500068790050726541726D3A20436F6D70611E
:101060007373206E6F74206865616C7468790050CA
:10107000726541726D3A20436F6D70617373206EBB
:101080006F742063616C6962726174656400507290
:101090006541726D3A20436F6D70617373206F66A6
:1010A000667365747320746F6F2068696768005099
:1010B000726541726D3A20436865636B206D6167AC
:1010C000206669656C640050726541726D3A204912
:1010D0004E53206E6F742063616C69627261746537
:1010E000640050726541726D3A20494E53206E6F14
:1010F00074206865616C7468790050726541726D26
:101100003A20436865636B20426F61726420566FBA
:101110006C746167650050726541726D3A20436876
:101120003726436838204F70742063616E6E6F7489
:101130002062652073616D650050726541726D3A81
:1011400020436865636B2046535F5448525F5641A5
:101150004C55450050726541726D3A204368656395
:101160006B20414E474C455F4D41580050726541E0
:10117000726D3A204143524F5F42414C5F524F4C97
:101180004C2F50495443480050726541726D3A20CB
:101190004261642047505320506F73005265616371
:1011A00068656420436F6D6D616E6420232569005E
:1011B0008059464D54000042426E4E5A00000000D5
:1011C00000000000000000547970652C4C656E67CB
:1011D00074682C4E616D652C466F726D61740000F1
:1011E00000000000000000000000000000000000FF
:1011F00000000000000000000000000000000000EF
:101200000000000000000081175041524D004E6662
:1012100000000000000000000000000000004E611F
:101220006D652C56616C75650000000000000000C3
:1012300000000000000000000000000000000000AE
:10124000000000000000000000000000000000009E
:101250000000000000000000000000000000822DDF
:10126000475053000042494842634C4C6565456510
:1012700066490000005374617475732C54696D6580
:101280004D532C5765656B2C4E536174732C484439
:101290006F702C4C61742C4C6E672C52656C416CD9
:1012A000742C416C742C5370642C474372732C560D
:1012B0005A2C540000831F494D550000496666664C
:1012C00066666600000000000000000054696D655D
:1012D0004D532C477972582C477972592C477972A3
:1012E0005A2C416363582C416363592C4163635A00
:1012F00000000000000000000000000000000000EE
:1013000000000000000000000000000084434D5376
:101310004700005A0000000000000000000000002C
:101320000000004D657373616765000000000000F8
:1013300000000000000000000000000000000000AD
:10134000000000000000000000000000000000009D
:10135000000000000000000000000000000000008D
:1013600000000019194154554E00424266666666F7
:1013700066000000000000000000417869732C54F2
:10138000756E65537465702C526174654D696E2C71
:10139000526174654D61782C52504761696E2C52D0
:1013A000444761696E2C53504761696E000000002C
:1013B000000000000000000000001A0941544445EC
:1013C0000063660000000000000000000000000054
:1013D00000416E676C652C5261746500000000006E
:1013E00000000000000000000000000000000000FD
:1013F00000000000000000000000000000000000ED
:1014000000000000000000000000000000000000DC
:101410000009134355525200684968686866000025
:1014200000000000000000005468724F75742C54D6
:101430006872496E742C566F6C742C437572722CE2
:101440005663632C43757272546F74000000000081
:10145000000000000000000000000000000000008C
:1014600000000000000000000B0F4D4F540000680A
:101470006868686868000000000000000000004D17
:101480006F74312C4D6F74322C4D6F74332C4D6F43
:1014900074342C4D6F74352C4D6F74360000000081
:1014A000000000000000000000000000000000003C
:1014B0000000000000000000000000000000000C20
:1014C0001C4F4600000068684263636666656500FD
:1014D00000000000000044782C44792C53517561C1
:1014E0006C2C582C592C4C61742C4C6E672C526F00
:1014F0006C6C2C50697463680000000000000000F0
:1015000000000000000000000000000000000000DB
:1015100000000000000005314E54554E0045636642
:10152000666666666666666565000000005750443C
:1015300073742C57504272672C504572582C50458A
:1015400072592C4456656C582C4456656C592C566F
:10155000656C582C56656C592C444163582C444199
:1015600063592C44526F6C2C445069740004194325
:1015700054554E00686365666368686868000000DB
:1015800000000000546872496E2C536F6E416C74F9
:101590002C426172416C742C5750416C742C446520
:1015A00073536F6E416C742C416E674273742C439D
:1015B000526174652C5468724F75742C44435261A7
:1015C000746500000F154D41470000686868686841
:1015D00068686868000000000000004D6167582CD2
:1015E0004D6167592C4D61675A2C4F6673582C4FCB
:1015F0006673592C4F66735A2C4D4F6673582C4D99
:101600004F6673592C4D4F66735A0000000000005E
:1016100000000000000000000000000613504D0014
:101620000000424248484968424842000000000029
:10163000000052656E436E742C52656E426C772CBE
:101640004E4C6F6E2C4E4C6F6F702C4D6178542C3D
:10165000504D542C4932434572722C494E534572B9
:10166000722C494E41564572720000000000000085
:1016700000000814434D4400004242424242654C7F
:101680004C000000000000000043546F742C434ED7
:10169000756D2C4349642C434F70742C50726D311E
:1016A0002C416C742C4C61742C4C6E670000000053
:1016B000000000000000000000000000000000002A
:1016C000000000000000000000011141545400001F
:1016D0006363636363434300000000000000000095
:1016E000526F6C6C496E2C526F6C6C2C5069746329
:1016F00068496E2C50697463682C596177496E2C67
:101700005961772C4E617659617700000000000026
:1017100000000000000000000000000000000000C9
:101720001125494E415600636363666666696966C2
:101730006600000000000042416C742C49416C744A
:101740002C49436C622C41436F7272582C41436F99
:101750007272592C41436F72725A2C474C61742C2F
:10176000474C6E672C494C61742C494C6E670000E5
:101770000000000000000003064D4F4445004D6886
:1017800000000000000000000000000000004D6F9D
:1017900064652C54687243727300000000000000FE
:1017A0000000000000000000000000000000000039
:1017B0000000000000000000000000000000000029
:1017C00000000000000000000000000000000A030C
:1017D00053545254000000000000000000000000BC
:1017E00000000000000000000000000000000000F9
:1017F00000000000000000000000000000000000E9
:1018000000000000000000000000000000000000D8
:1018100000000000000000000000000000000000C8
:1018200000000000000D04455600000042000000CA
:1018300000000000000000000000000049640000FB
:101840000000000000000000000000000000000098
:101850000000000000000000000000000000000088
:101860000000000000000000000000000000000078
:1018700000000000000000000000000014064431D9
:101880003600004268000000000000000000000078
:1018900000000049642C56616C7565000000000072
:1018A0000000000000000000000000000000000038
:1018B0000000000000000000000000000000000028
:1018C0000000000000000000000000000000000018
:1018D0000000001506445531360042480000000063
:1018E0000000000000000000000049642C56616CFC
:1018F000756500000000000000000000000000000E
:1019000000000000000000000000000000000000D7
:1019100000000000000000000000000000000000C7
:1019200000000000000000000000160844333200F0
:1019300000426900000000000000000000000000FC
:101940000049642C56616C756500000000000000C1
:101950000000000000000000000000000000000087
:101960000000000000000000000000000000000077
:101970000000000000000000000000000000000067
:1019800000170844553332004249000000000000AF
:10199000000000000000000049642C56616C756571
:1019A0000000000000000000000000000000000037
:1019B0000000000000000000000000000000000027
:1019C0000000000000000000000000000000000017
:1019D0000000000000000000180844464C5400427B
:1019E0006600000000000000000000000000004948
:1019F000642C56616C75650000000000000000005A
:101A000000000000000000000000000000000000D6
:101A100000000000000000000000000000000000C6
:101A20000000000000000000000000000000000EA8
:101A30001C504944000042696969696966000000F8
:101A400000000000000049642C4572726F722C5037
:101A50002C492C442C4F75742C4761696E00000092
:101A60000000000000000000000000000000000076
:101A70000000000000000000000000000000000066
:101A8000000000000000121B43414D000049484C7B
:101A90004C656363430000000000000000475053A2
:101AA00054696D652C4750535765656B2C4C6174B8
:101AB0002C4C6E672C416C742C526F6C6C2C5069E2
:101AC0007463682C5961770000000000000000007A
:101AD00000000000000000000000000000130545A9
:101AE00052520000424200000000000000000000CE
:101AF000000000005375627379732C45436F646571
:101B000000000000000000000000000000000000D5
:101B100000000000000000000000000000000000C5
:101B200000000000000000000000000000000000B5
:101B30000000000041726475436F70746572205636
:101B4000332E312D7263382028290047524F554ECD
:101B50004420535441525400494E530A002D00472B
:101B60005F6F66663A2025342E32662C2025342E8F
:101B700032662C2025342E32660A00415F6F66667D
:101B80003A2025342E32662C2025342E32662C2025
:101B900025342E32660A415F7363616C653A2025F5
:101BA000342E32662C2025342E32662C2025342EFD
:101BB00032660A0043616C6962726174696E672003
:101BC0006261726F6D65746572006261726F6D65DE
:101BD0007465722063616C6962726174696F6E20F2
:101BE000636F6D706C6574650041726D3A20546866
:101BF000722062656C6F772046530041726D3A2007
:101C000053616665747920537769746368004C6F1B
:101C100077204261747465727921004C6F7374206F
:101C200047505321000A0A496E6974204172647555
:101C3000436F707465722056332E312D72633820D5
:101C400028290A0A467265652052414D3A202575B9
:101C50000A004E6F2064617461666C61736820696C
:101C60006E7365727465640045524153494E472056
:101C70004C4F4753000A507265737320454E5445CC
:101C80005220332074696D657320746F2073746102
:101C9000727420696E74657261637469766520730D
:101CA000657475700A000A526561647920746F204A
:101CB000464C592000496E697469616C6973696E9C
:101CC000672041504D2E2E2E004657205665723A01
:101CD0002025640A004669726D7761726520636829
:101CE000616E67653A2065726173696E672045456C
:101CF00050524F4D2E2E2E0A00646F6E652E008DB1
:101D0000000100424154545F4D4F4E49544F520020
:101D100000000000A8000100424154545F564F4C9F
:101D2000545F50494E00000000A900010042415498
:101D3000545F435552525F50494E000000008E00E0
:101D40000400424154545F564F4C545F4D554C541F
:101D50000000008F000400424154545F414D505F29
:101D6000504552564F4C5400910003004241545488
:101D70005F4341504143495459000000006C6F617A
:101D8000645F616C6C20746F6F6B20256C7575736C
:101D90000A0045726173696E67206C6F67730A0091
:101DA0004C6F6720657261736520636F6D706C6541
:101DB00074650A00456E746572696E672045534309
:101DC0002043616C6962726174696F6E3A20706C55
:101DD0006561736520726573746172742041504D42
:101DE0002E0A004553432043616C69627261746935
:101DF0006F6E206163746976653A207061737369F0
:101E00006E67207468726F74746C65207468726F8A
:101E100075676820746F20455343732E0A00434F43
:101E20004D5041535320494E4954204552524F5230
:101E3000004175746F54756E653A20537563636520
:101E40007373004175746F54756E653A204661690D
:101E50006C6564004175746F54756E653A205374F7
:101E6000617274656400636F6D6D616E642072658C
:101E70006365697665643A200041726475436F70EA
:101E80007465722056332E312D7263382028290054
:101E9000556E6B6E6F776E20706172616D657465E3
:101EA0007220696E64657820256400556E6B6E6FD4
:101EB000776E20706172616D6574657220252E31B8
:101EC000367300666C6967687420706C616E20758B
:101ED00070646174652072656A6563746564006628
:101EE0006C6967687420706C616E207265636569E7
:101EF0007665640043726173683A20446973617265
:101F00006D696E670046656E636520427265616348
:101F1000686564004C6F670064756D7000000000B8
:101F20000000000000003637657261736500000034
:101F3000000000000000F976656E61626C650000CB
:101F4000000000000000414D64697361626C65002F
:101F5000000000000000414D7365747570006163FE
:101F600063656C000000000000000000D158636F42
:101F70006D70617373000000000000001756636FFE
:101F80006D706173736D6F74000000002195657250
:101F9000617365000000000000000000A52B667260
:101FA000616D65000000000000000000494B6D6F8E
:101FB0006465730000000000000000008B936F70E8
:101FC00074666C6F77000000000000008D2B72615A
:101FD00064696F0000000000000000003C91726125
:101FE0006E6765000000000000000000AB4C7265E9
:101FF000736574000000000000000000FA40736583
:10200000740000000000000000000000104E736823
:102010006F7700000000000000000000DD42736FD9
:102020006E6172000000000000000000264C41724A
:102030006475436F707465722056332E312D726350
:1020400038006C6F677300000000000000000000A3
:1020500056367365747570000000000000000000C3
:102060005C3674657374000000000000000000001E
:1020700050367265626F6F7400000000000000004F
:10208000262C68656C700000000000000000000055
:102090000F2C74657374006261726F0000000000A1
:1020A00000000000006A76636F6D7061737300005A
:1020B0000000000000585767707300000000000027
:1020C00000000000008531696E7300000000000010
:1020D000000000000076566C6F6767696E6700004D
:1020E00000000000006E316D6F746F7273000000AD
:1020F0000000000000E7906F7074666C6F7700005E
:102100000000000000B92C70776D00000000000096
:102110000000000000CA8F726164696F0000000057
:102120000000000000618F72656C617900000000A2
:102130000000000000B22D736F6E6172000000009D
:102140000000000000BB2C52656C6179206F6E0AA4
:102150000052656C6179206F66660A0048697420D8
:10216000456E74657220746F20657869742E0A0A52
:1021700000494E2020313A20256409323A20256456
:1021800009333A20256409343A20256409353A2078
:10219000256409363A20256409373A2025640A0067
:1021A000494E3A20313A20256409323A2025640903
:1021B000333A20256409343A20256409353A20252C
:1021C0006409363A20256409373A20256409383AEB
:1021D0002025640A00436F6E6E656374206261742B
:1021E0007465727920666F722074686973207465F3
:1021F00073742E0A4D6F746F72732077696C6C2044
:102200007370696E206279206672616D6520706FEF
:10221000736974696F6E206F726465722E0A4672FC
:102220006F6E74202826207269676874206F66209C
:1022300063656E7465726C696E6529206D6F746F6D
:10224000722066697273742C207468656E20696EE2
:1022500020636C6F636B77697365206F726465725E
:102260002061726F756E64206672616D652E0A5210
:10227000656D656D62657220746F20646973636F4C
:102280006E6E656374206261747465727920616634
:10229000746572207468697320746573742E0A41C2
:1022A0006E79206B657920746F20657869742E0AC9
:1022B0000054657374696E672064617461666C6153
:1022C0007368206C6F6767696E6700436F6D6D613F
:1022D0006E64733A0A20206C6F67730A202073655E
:1022E0007475700A2020746573740A202072656208
:1022F0006F6F740A0A006F6E006F6666000A4F7097
:102300003A5B6F6E2C206F66662C20302D335D0A91
:1023100000536F6E61720A00547970653A2025642B
:102320002028303D584C2C20313D4C562C20323D3D
:10233000584C4C2C20333D48524C562900656E00B9
:102340006469730061626C65640A00506172616D5A
:1023500065746572206E6F7420666F756E643A20C6
:10236000272573270A00526164696F0A00434831C8
:102370003A202564207C2025640A004348323A2014
:102380002564207C2025640A004348333A202564D4
:10239000207C2025640A004348343A202564207CB0
:1023A0002025640A004348353A202564207C2025F6
:1023B000640A004348363A202564207C2025640ABC
:1023C000004348373A202564207C2025640A0043D6
:1023D00048383A202564207C2025640A0046726132
:1023E0006D650A0048657861206672616D650A0056
:1023F00058206D6F64650A002B206D6F64650A00BC
:1024000056206D6F64650A000A42617474204D6F36
:102410006E3A0A00766F6C747300766F6C7473207A
:10242000616E642063757200466C69676874206D24
:102430006F6465730A00506F732025643A09002C9D
:10244000090953696D706C653A20004F46460A00D1
:1024500053544142494C495A45004143524F00416F
:102460004C545F484F4C44004155544F0047554928
:10247000444544004C4F495445520052544C00438B
:102480004952434C4500504F534954494F4E004C1C
:10249000414E44004F465F4C4F4954455200445210
:1024A0004946540053504F5254004D6F64652825DF
:1024B0007529004F4E0A00436F6D706173730A00F7
:1024C0004D6167204465633A2025342E34660A0046
:1024D0004D6167206F66663A2025342E34662C20C5
:1024E00025342E34662C2025342E34660A004D6F98
:1024F000746F7220436F6D703A20004F66660A0059
:102500005468726F74746C650043757272656E7492
:10251000000A436F6D70205665633A2025342E32D1
:10252000662C2025342E32662C2025342E32660A65
:1025300000496E76616C696420636F6D6D616E64D5
:102540002E2055736167653A20736574203C6E6177
:102550006D653E203C76616C75653E0A0050617287
:10256000616D206E6F7420666F756E643A202573FE
:102570000A0056616C7565206F7574206F66207255
:10258000616E676520666F72207479706520494EB0
:1025900054380A0056616C7565206F7574206F663B
:1025A0002072616E676520666F7220747970652095
:1025B000494E5431360A0043616E6E6F7420736564
:1025C0007420706172616D65746572206F6620742D
:1025D0007970652025642E0A000A275927203D209E
:1025E000666163746F72792072657365742C206103
:1025F0006E79206F74686572206B657920746F2026
:1026000061626F72743A0A000A5265626F6F7420D9
:1026100041504D000A434820362052616E67657371
:10262000206172652064697669646564206279203E
:10263000313030303A205B6C6F772C2068696768E6
:102640005D0A000A54554E453A0A002025642C20A4
:102650004C6F773A25312E34662C20486967683AEA
:1026600025312E34660A000A0A526164696F2053CC
:10267000657475703A000A4D6F766520616C6C2048
:10268000636F6E74726F6C7320746F2065787472F0
:10269000656D65732E20456E74657220746F2073AE
:1026A0006176653A20000A53617665640A000A4D36
:1026B0006F64652073776974636820746F20656444
:1026C00069742C2061696C65726F6E3A2073656C59
:1026D000656374206D6F6465732C20727564646526
:1026E000723A2053696D706C65206F6E2F6F66664D
:1026F0000A00780070002B0076000A4F703A5B7871
:102700002C2B2C765D0A000A45726173696E672076
:10271000454550524F4D0A00646F6E650A00726164
:1027200064696F206E6F742063616C69627261749A
:1027300065640A00636F6D7061737320646973610F
:10274000626C65640A0054686973207265636F7215
:1027500064732074686520696D70616374206F6EA6
:102760002074686520636F6D70617373206F6620DD
:1027700072756E6E696E6720746865206D6F746F18
:1027800072732E20204D6F746F72732077696C6C9A
:10279000207370696E210A486F6C64207468726FD0
:1027A00074746C65206C6F772C207468656E207271
:1027B0006169736520746F206D696420666F722093
:1027C00035207365632C207468656E2071756963AC
:1027D0006B6C79206261636B20746F206C6F772E55
:1027E0000A507265737320616E79206B657920746D
:1027F0006F20657869742E0A0A6D65617375726958
:102800006E6720636F6D7061737320767320004371
:10281000555252454E540A005448524F54544C4558
:102820000A007468726F74746C65206E6F74207A1D
:1028300065726F0A00636865636B20636F6D70611A
:1028400073730A000A496E746572666572656E6319
:10285000652061742066756C6C207468726F747486
:102860006C652069732025642525206F66206D61C5
:1028700067206669656C640A0A004661696C656474
:102880002120436F6D70656E736174696F6E206493
:10289000697361626C65642E202044696420796FDD
:1028A0007520666F7267657420746F20726169733A
:1028B0006520746865207468726F74746C65206834
:1028C00069676820656E6F7567683F007468723A63
:1028D0002564206375723A25342E3266206D6F743C
:1028E00020783A25342E316620793A25342E316607
:1028F000207A3A25342E31662020636F6D7020785F
:102900003A25342E326620793A25342E3266207AE2
:102910003A25342E32660A006F6E006F6666000A32
:102920004F703A5B6F6E2C6F66665D0A00496E6988
:102930007469616C6973696E67206779726F73007F
:102940005365747570204D6F64650A0A0A000A2188
:102950005761726E696E672C20726164696F206EB8
:102960006F7420636F6E6669677572656421000A13
:1029700020547970652027726164696F27206E6F1B
:10298000772E0A0A00494E530A002E2E2E646F6ECF
:10299000650A00612025372E34662025372E3466DF
:1029A0002025372E346620672025372E34662025D3
:1029B000372E34662025372E346620742025372E96
:1029C0003466200A004C61743A20002C204C6F6E53
:1029D00020002C20416C743A20256C646D2C20233F
:1029E000736174733A2025640A002E00436F6D7082
:1029F0006173733A2000436F6D7061737320696E69
:102A0000697469616C69736174696F6E206661696C
:102A10006C6564210048656164696E673A20256CC5
:102A2000642C2058595A3A2025642C2025642C20E7
:102A300025642C0958595A6F66663A2025362E327D
:102A4000662C2025362E32662C2025362E32660A3C
:102A500000636F6D70617373206E6F7420686561C1
:102A60006C74687900736176696E67206F6666734F
:102A7000657473006E6F74206865616C74687900AA
:102A8000416C743A2025302E32666D2C20526177CD
:102A90003A2025662054656D7065726174757265A3
:102AA0003A20252E31660A006C6F677320656E61CF
:102AB000626C65643A20006E6F6E6500204154546C
:102AC00049545544455F46415354002041545449AC
:102AD000545544455F4D4544002047505300205015
:102AE0004D00204354554E00204E54554E00204971
:102AF0004D550020434D44002043555252454E54FD
:102B000000204D4F544F525300204F5054464C4FCD
:102B10005700205049440020434F4D50415353002B
:102B200020494E4156002043414D455241006D69B8
:102B30007373696E67206C6F6720747970650A0023
:102B4000616C6C0041545449545544455F464153AF
:102B5000540041545449545544455F4D4544004741
:102B6000505300504D004354554E004E54554E00A6
:102B70004D4F444500494D5500434D440043555287
:102B800052454E54004D4F544F5253004F505446EF
:102B90004C4F570050494400434F4D504153530050
:102BA000494E41560043414D45524100656E6162B8
:102BB0006C650064756D70696E6720616C6C0A00ED
:102BC000626164206C6F67206E756D6265720A00C9
:102BD0000A41726475436F707465722056332E31EA
:102BE0002D7263382028290A467265652052414DAE
:102BF0003A2025750A0041504D2032000100454E13
:102C000041424C45000000000000000000000002AE
:102C10000000000000010154595045000000000070
:102C2000000000000000000003000000404001021E
:102C3000414354494F4E00000000000000000000D6
:102C40000004000000803F0403414C545F4D415894
:102C50000000000000000000000005000000C84265
:102C60000404524144495553000000000000000094
:102C700000000009000000164304054D4152474979
:102C80004E00000000000000000000000D000000E9
:102C9000004000FF000000000000000000000000F5
:102CA00000000000000000000000000400500000D0
:102CB0000000000000000000000000000000000014
:102CC00000000000040149000000000000000000B6
:102CD00000000000000000040000000000040244A6
:102CE00000000000000000000000000000000000E4
:102CF0000800000000000203494D41580000000098
:102D00000000000000000000000C000000000000B7
:102D1000FF000000000000000000000000000000B4
:102D2000000000000000000004005350454544002E
:102D3000000000000000000000000011000000FA88
:102D40004304015241444955530000000000000073
:102D5000000000001D000000484304025350454598
:102D6000445F555000000000000000000015000006
:102D7000007A43040353504545445F444E0000002D
:102D800000000000000019000000164304044C4F2E
:102D900049545F5350454544000000000000000DB9
:102DA000000000FA430405414343454C0000000085
:102DB000000000000000000021000000C84200FFE9
:102DC0000000000000000000000000000000000003
:102DD000000000000000000400500000000000009F
:102DE00000000000000000000000000000000000E3
:102DF0000401490000000000000000000000000085
:102E00000000000400000000000202494D4158008B
:102E100000000000000000000000000008000000AA
:102E2000000000FF000000000000000000000000A3
:102E300000000000000000000000000402475053A2
:102E40005F4741494E0000000000000000002400E0
:102E50000000803F01034750535F55534500000079
:102E6000000000000000002C000000803F04045916
:102E700041575F500000000000000000000000000B
:102E80001C00CDCC4C3E040552505F5000000000A9
:102E90000000000000000000002000CDCC4C3E01EE
:102EA0000657494E445F4D415800000000000000A5
:102EB00000002D000000000005085452494D00009C
:102EC00000000000000000000000003E00000000C4
:102ED0000001094F5249454E544154494F4E00009C
:102EE000000000002E0000000000040A434F4D5077
:102EF0005F4245544100000000000000002800CD62
:102F0000CCCC3D010B4750535F4D494E5341545378
:102F10000000000000002F000000C040010C4750DE
:102F2000535F44454C415900000000000000003050
:102F3000000000004000FF00000000000000000052
:102F4000000000000000000000000000000004027B
:102F50004142535F505245535300000000000000AF
:102F6000000C0000000000040354454D5000000018
:102F70000000000000000000000008000000000049
:102F80000104414C545F4F46465345540000000035
:102F900000000010000000000000FF000000000022
:102FA0000000000000000000000000000000000021
:102FB000000050414E49433A2041505F4261726FD8
:102FC0003A3A7265616420756E73756363657373F5
:102FD00066756C20666F72206D6F72652074686113
:102FE0006E203530306D7320696E2041505F426134
:102FF000726F3A3A63616C696272617465205B3129
:103000005D0D0A0050414E49433A2041505F4261F4
:10301000726F3A3A7265616420756E7375636365A9
:10302000737366756C20666F72206D6F72652074A5
:1030300068616E203530306D7320696E2041505FBD
:103040004261726F3A3A63616C69627261746520C1
:103050005B325D0D0A0050414E49433A2041505FBA
:103060004261726F3A3A7265616420756E7375637E
:103070006365737366756C20666F72206D6F726521
:10308000207468616E203530306D7320696E204188
:10309000505F4261726F3A3A63616C696272617447
:1030A00065205B335D0D0A0050414E49433A204193
:1030B000505F4261726F5F4D533536313120646924
:1030C00064206E6F74206765742076616C6964207B
:1030D000535049206465766963652064726976653A
:1030E00072210050414E49433A2041505F42617283
:1030F0006F5F4D533536313120646964206E6F74D3
:10310000206765742076616C696420535049207390
:10311000656D617068726F65210050414E49433A98
:10312000206661696C656420746F2074616B652032
:103130005F7370695F73656D203130302074696D25
:10314000657320696E206120726F772C20696E2074
:1031500041505F4261726F5F4D53353631313A3ABB
:103160005F7570646174650050414E49433A204177
:10317000505F4261726F5F4D533536313120646963
:1031800064206E6F74206765742076616C696420BA
:103190004932432073656D617068726F652100501C
:1031A000414E49433A206661696C656420746F2022
:1031B00074616B65205F6932635F73656D203130C8
:1031C000302074696D657320696E206120726F779D
:1031D0002C20696E2041505F4261726F5F4D533504
:1031E0003631313A3A5F7570646174650050414E12
:1031F00049433A2041505F4261726F5F4D5335360B
:1032000031313A204E554C4C2073657269616C2007
:103210006472697665720050414E49433A204150CC
:103220005F4261726F5F4D53353631313A206661CE
:10323000696C656420746F2074616B6520736572BE
:1032400069616C2073656D6170686F726520666F6F
:103250007220696E69740050414E49433A204150D2
:103260005F4261726F5F4D533536313120746F6F3D
:103270006B206D6F7265207468616E203130303064
:103280006D7320746F20696E697469616C697A6509
:103290000001004D4F4E49544F5200000000000005
:1032A000000000000000000000000101564F4C54D7
:1032B0005F50494E000000000000000000010000C7
:1032C0000050410102435552525F50494E000000E8
:1032D0000000000000000200000040410403564FBF
:1032E0004C545F4D554C540000000000000000039A
:1032F000009A9921410404414D505F504552564F68
:103300004C54000000000000070000008841040544
:10331000414D505F4F4646534554000000000000A9
:10332000000B000000000003064341504143495494
:10333000590000000000000000000F0000404E4552
:1033400000FF00000000000000000000000000007E
:103350000000000000000000004661696C65642008
:10336000746F2067657420484D43353834332073BB
:10337000656D6170686F72650005014F465300000E
:10338000000000000000000000000000110000002C
:10339000000004024445430000000000000000005B
:1033A00000000000001D000000000001034C45412A
:1033B000524E0000000000000000000000000F005E
:1033C0000000803F0104555345000000000000004C
:1033D0000000000000000021000000803F010541C6
:1033E00055544F4445430000000000000000000019
:1033F00022000000803F01064D4F5443540000005E
:103400000000000000000000009E00000000000519
:10341000074D4F54000000000000000000000000B5
:1034200000009F000000000001084F5249454E5423
:10343000000000000000000000000010000000007C
:1034400000010945585445524E414C00000000000F
:103450000000000023000000000000FF000000004A
:10346000000000000000000000000000000000005C
:1034700000000043757276653A00783A0009793A9F
:103480000009736C6F70653A0043757276653A0097
:10349000783A0009793A0009736C6F70653A004315
:1034A000757276653A00783A0009793A0009736CCA
:1034B0006F70653A0043757276653A00783A000994
:1034C000793A0009736C6F70653A004375727665DE
:1034D0003A00783A0009793A0009736C6F70653ADE
:1034E0000043757276653A00783A0009793A000926
:1034F000736C6F70653A0096918C87827D78736EDD
:1035000069645F5A55504B46413C37322D28231E83
:1035100019140F0A050004090E13181D22272C3157
:10352000363B40454A4F54595E63686D72777C81E3
:10353000868B90959A9FA4A9AEB3AFAAA5A09B969F
:103540008F89837E78736E69645F5A55504B47420A
:103550003E3935302C27231F1B16120E0905010397
:10356000070B1014191D22262B2F34393D42474CCE
:1035700051565B60656B70757B80868C92979DA3BE
:10358000A9AFB2ACA6A09A948F827C76706B65606E
:103590005C57524E4A46413D3936322E2A26221F6A
:1035A0001B1713100C08040102060A0E12161A1E2D
:1035B00022262B2F33383D41464B4F54595E6469C8
:1035C0006F747A80878D949BA2AAB1AEA69F9790C4
:1035D00089826F68635E5955514D4946423F3C3878
:1035E00035322E2B2824211E1A1714100D0A06031B
:1035F000000306090D1014181C2024282C3034391F
:103600003D41464A4F54585D62676D737980878F9C
:1036100098A2ACB0A59A90867D766F55514D4A47D9
:1036200044413F3C3A383533312E2B292623201D87
:103630001A1713100D0A070401010306090D1013D0
:10364000171A1E22262A2E32363A3E42464A4E5338
:10365000575B5F64696E757C85909FB2A08D7D70AD
:1036600067605A553E3C3A393736343332302F2E64
:103670002C2A292724221F1C191613100D0A0704AF
:1036800002000305080A0D1013161A1D2125292D05
:103690003135383C4043464A4D505356595B5E6184
:1036A00065696F826D544D4A474442403E2E2E2D2F
:1036B0002C2C2B2A2A2929282726252423211F1CA4
:1036C0001A1714100D0A07040101030507090C0E4F
:1036D0001013161A1D2124282C3033373A3D40424E
:1036E0004447484A4A4B4A48443D3019021621286B
:1036F0002B2D2E2F2E2E06090C0F121517191B1C01
:103700001B1811040E2231383C3C3C3A3835322F1C
:103710002B2824201C1915110D09050102060A0E7B
:103720001115181C1F222527292A2B2B2926211980
:1037300011080004080A0A0A080704020003061612
:10374000181A1C1E20211F1712516063625F5D59F9
:1037500056524E4A46423E3935312C2824201B17FA
:10376000130E0A060102060A0F13171B1F23262A2F
:103770002D313437393C3D3F3F3E3D39352F2821EF
:103780001C17151313131416A8ADB2B0ABA6A19C49
:1037900097928D88837E79746F6A65605B56514C11
:1037A00047423D38332E29241F1A15100B060103FA
:1037B000080D12171C21262B30353A3F44494E5331
:1037C000585D62676C71767B80858A8F94999EA321
:1037D000A800000001FFFFE000000000000001FF62
:1037E000FFF000000000000001FFFFF800000000F3
:1037F000000001FFFFFE00000000000003FFFFFFCC
:1038000000000000000003FFFFFFF00000000000C8
:103810000FFFFFFFFE00000003FFFFFC000007FC9E
:1038200000007FFFFFFC000000000000001FFFFE03
:103830000000000000241E191512100E0C0B0A09BE
:10384000090908080807060605040404030404041B
:10385000000000000000000000002726212325238F
:1038600025242722292A2A1C27282B3332272522E0
:103870002C333130370000000000000000000080D1
:10388000114011407132733433321312113211125C
:10389000933413145352310021030406080B2D0AEC
:1038A000090705040241C011C0511253547312118B
:1038B00012515273147332310021020405060708B5
:1038C0000908060706240302010200012001201155
:1038D000C00111003132137413143312F112D312D8
:1038E000510001022325060746442342210001E03E
:1038F000A0313213B43311121100112011005233D0
:1039000012133211200122248504230402034241B0
:103910000001E0A051121413151315341332514055
:103920000120115213323100012223040504050441
:1039300023010382612001E0118011321354151418
:1039400033323140210201003172314102234423DC
:1039500002012201220102614001A01180511214D2
:1039600013341514331231400102010302012052B5
:10397000111220212243042241022102A10001E070
:1039800020114051537413321140210203020302EB
:1039900001001112113200114122232221004102A3
:1039A000A1800160116011001132337413121140B3
:1039B00001620302032131121112114001020102BE
:1039C000030201000100E121E0A011201211733473
:1039D0003331200162036240121112110011010003
:1039E000010201220001200100E1C001001180114B
:1039F0000012111312141334522001E2022120315B
:103A000012110011000100210201000140210002F9
:103A1000410001E06011401112111312141314132C
:103A20003211002122034201022100010011001283
:103A300011001120010041600100C100014011206E
:103A4000016011405112131213143312310001425C
:103A50000322010221000140110031001100010088
:103A6000010001A0E10001A0018011203152931258
:103A7000110021C22100214031001120110001005C
:103A800001E0E16001E01100117273123100214286
:103A900003010201022021401100112011600140A8
:103AA0001160010001022102000120014001A0512A
:103AB0003213125332112001020182210021000130
:103AC00000110031E000110011602100010201022B
:103AD0000101002120010001601100115213121494
:103AE0001352110041820102000100214011001116
:103AF0000011A011003100112081220101000201FA
:103B0000002100016011005213121314133231010D
:103B100000020122014201002100010001112011D7
:103B20000011201140710011400102210201020127
:103B300000210221000100010011001211123312B4
:103B4000341332112001020142012201004100011F
:103B50006011201100110011005112312061020189
:103B6000220200020102812011001211733413326B
:103B70001100410201820100610001801100110069
:103B8000913231402142010202006261401152141F
:103B9000135433310041820122000102004100012F
:103BA0006091121152512001220103010202008290
:103BB00061005133541514333100210201220342B4
:103BC0004102A180319213323100412203020103EC
:103BD000002203220102014011123395333101000A
:103BE000220103420322212201026100011100117E
:103BF0005213125312310041220322030023020305
:103C00000201022120321314161517161533112044
:103C1000016203020302032201A241401112531464
:103C20001314133211010002010203020302020005
:103C300002230203222120321416371817151312FB
:103C400011002122030243024301030203822120C7
:103C500011121314153415143211000162230203DA
:103C60000043020342012012131518193A171513C5
:103C70001100210203026304E302030203020102B2
:103C80004012131415171516341220212243020373
:103C900000A3220100111215181C1E1D1916131164
:103CA0000002010302030423040324030443042346
:103CB000040302034220111214151718361513318C
:103CC000210203022302030100454E41424C4500FC
:103CD0000000000000000000000003000000803F22
:103CE0000401524144495553000000000000000007
:103CF0000000000400000048430402414343454CD7
:103D000000000000000000000000000008000000AB
:103D10007A4400FF000000000000000000000000E6
:103D20000000000000000000000000B56206010372
:103D300000010601124F24505542582C34312C31C9
:103D40002C303030332C303030312C33383430306C
:103D50002C302A32360D0A004572726F723A2041B9
:103D6000505F48414C5F4156523A3A415652416E7B
:103D7000616C6F67496E206F7574206F6620636891
:103D8000616E6E656C730D0A0050414E49433A20D6
:103D90007363686564756C65723A3A7379737465B8
:103DA0006D5F696E697469616C697A6564206361CD
:103DB0006C6C65646D6F7265207468616E206F6EE7
:103DC000636500474F494E4720444F574E20464FAA
:103DD000522041205245424F4F540D0A0050414E4F
:103DE00049433A2041565253656D6170686F726560
:103DF0003A3A74616B6520757365642066726F6D05
:103E000020696E736964652074696D6572207072D3
:103E10006F636573730050414E49433A20535049D4
:103E200030207472616E7366657220636F6C6C69AA
:103E300073696F6E0050414E49433A2053504930E8
:103E400020777269746520636F6C6C6973696F6E3B
:103E500000040154435F58590000000000000000B6
:103E600000000000140000002040040254435F5A88
:103E700000000000000000000000000000650000DD
:103E800000A04000FF000000000000000000000053
:103E9000000000000000000000000000020050527E
:103EA0004F445543545F4944000000000000002681
:103EB000000000000005014143435343414C000012
:103EC00000000000000000002800000000000502C3
:103ED0004143434F464653000000000000000000ED
:103EE0000034000000000005034759524F46465376
:103EF0000000000000000000000040000000000082
:103F000001044D5055364B5F46494C544552000014
:103F10000000004C000000000000FF000000000056
:103F20000000000000000000000000000000000091
:103F30000000496E6974204779726F002A000A6791
:103F400079726F20646964206E6F7420636F6E767F
:103F5000657267653A20646966663D25662064700F
:103F6000730A00496E697420416363656C002A001E
:103F700020006F6E20697473204241434B00506CE7
:103F80006163652041504D20255320616E6420708F
:103F90007265737320616E79206B65792E0A004615
:103FA00061696C656420746F2067657420494E53A5
:103FB0002073616D706C650A004F6666736574737B
:103FC0003A20252E326620252E326620252E326696
:103FD0000A005363616C696E673A20252E326620B1
:103FE000252E326620252E32660A0043616C6962F6
:103FF000726174696F6E2073756363657373667540
:104000006C0A0043616C6962726174696F6E20466C
:1040100041494C45440A006C6576656C006F6E2022
:10402000697473204C4546542073696465006F6E53
:1040300020697473205249474854207369646500AD
:104040006E6F736520444F574E006E6F7365205539
:1040500050004D5055363030303A20556E61626C0C
:104060006520746F206765742073656D6170686F7B
:104070007265004D50553630303020737461727463
:104080007570206661696C65643A206E6F206461AA
:1040900074612072656164790050414E49433A2051
:1040A0006661696C656420746F20626F6F74204D67
:1040B00050553630303020352074696D65730050AE
:1040C000414E49433A2041505F496E6572746961BF
:1040D0006C53656E736F725F4D5055363030303AA9
:1040E0003A5F706F6C6C5F64617461206661696CCB
:1040F000656420746F2074616B6520535049207390
:10410000656D6170686F72652073796E6368726F38
:104110006E6F75736C79004D5055363030303A20E3
:10412000556E61626C6520746F20676574207365DD
:104130006D6170686F7265004661696C65642074BA
:104140006F20626F6F74204D5055363030302035FF
:104150002074696D65730054696D6564206F7574B2
:104160002077616974696E6720666F722075736568
:104170007220726573706F6E7365002D00256C641C
:104180002E2530376C640025535D200068656C7007
:10419000006578697400496E76616C696420636FAC
:1041A0006D6D616E642C2074797065202768656C74
:1041B000702700436F6D6D616E64733A0020202597
:1041C000530A000101544352565F454E41424C454B
:1041D00000000000000040000000803F0102544346
:1041E00052565F4D494450435400000000000041C6
:1041F00000000050420103544352565F4D41585055
:10420000435400000000000042000000BA420205D2
:104210005350494E5F41524D45440000000000009C
:1042200000430000008C4200FF000000000000007E
:10423000000000000000000000000000000000007E
:1042400041505F4D6F746F72733A206661696C659F
:104250006420746F20637265617465207468726F86
:1042600074746C6520637572766500454550524FD5
:104270004D2066756C6C0025733A2025640A002574
:10428000733A2025640A0025733A20256C640A00DD
:1042900025733A2025660A00556E6B6E6F776E2087
:1042A000636F6E76657273696F6E20272553270AD8
:1042B0000042616420636F6E76657273696F6E2071
:1042C0007479706520272553270A000100524F4C4E
:1042D0004C00000000000000000000000000000092
:1042E0000000803F01015049544348000000000095
:1042F0000000000000000001000000004001025426
:1043000048524F54544C450000000000000000008B
:104310000300000040400103594157000000000025
:1043200000000000000000000002000000804000CB
:10433000FF0000000000000000000000000000007E
:104340000000000000000000010050494E00000085
:10435000000000000000000000000000000000500D
:104360004100FF000000000000000000000000000D
:10437000000000000000000000000100444542551C
:1043800047000000000000000000000000000000E6
:1043900000000000FF00000000000000000000001E
:1043A000000000000000000000000000536368658A
:1043B00064756C657220736C6970207461736B5BDB
:1043C00025755D202825752F25752F2575290A004F
:1043D0005363686564756C6572206F76657272757B
:1043E0006E207461736B5B25755D202825752F2504
:1043F00075290A0050414E49433A20446174614690
:104400006C617368205350494465766963654472F2
:1044100069766572206E6F7420666F756E640050E9
:10442000414E49433A2044617461466C617368208F
:1044300053504944657669636544726976657220B4
:1044400073656D6170686F7265206973206E756C3D
:104450006C00554E4B4E2C2025750A0025532C2000
:1044600000256400257500256400257500256C6411
:1044700000256C7500256600252E326600252E323B
:104480006600252E326600252E3266002573002533
:1044900073002573002C2000464D542C2025752CCC
:1044A0002025752C2025532C2025532C2025530AFC
:1044B00000444620706167652C206C6F6720666938
:1044C0006C6520232C206C6F6720706167653A2033
:1044D00025752C090025752C090025750A004E6FDD
:1044E0002064617461666C61736820696E736572C3
:1044F000746564004D616E75666163747572657292
:104500003A2030782530327820202044657669635F
:10451000653A203078253034780A004E756D506148
:104520006765733A20257520205061676553697A65
:10453000653A2025750A000A4E6F206C6F67730A72
:104540000A000A2575206C6F67730A004C6F67209C
:1045500025752C2020202073746172742025752C01
:10456000202020656E642025750A00327C8900EDCC
:10457000D96877000000590000000000000000D654
:104580009FDCA81817AA90437327F6B968EDF4DEEC
:10459000D409FEE61C1C84DDE80B992927D6DF8DA3
:1045A000210F036418EFEE1EF0B78282009415000D
:1045B000F37C0000001400988F00007F6A00000068
:1045C00000000000E7B73F3600000000000000AF29
:1045D000669ED0385DD36C20B9EB5D7C7C7704009F
:1045E00000000000000000000000000000000000CB
:1045F00000000000000000000000000000002AF1A0
:104600000F86DBD0BC5416131586004E44BD7F9A2E
:1046100015159001EA49B51653A78AEA0000000073
:10462000000000000000000000000000000000008A
:10463000000000000000000000000000000000007A
:10464000000000000000000000000000000000006A
:10465000000000000000000000000000000000005A
:1046600000000000CC31AA2C532E000800000000EE
:10467000000000000000000000000000000000003A
:10468000B6460000010146554E4354494F4E0000C6
:10469000000000000000001D000000000000FF00FE
:1046A000000000000000000000000000000000000A
:1046B00000000000000002004D494E000000000014
:1046C0000000000000000000000A00008089440291
:1046D000015452494D00000000000000000000009D
:1046E00000000C000080BB4402024D415800000055
:1046F00000000000000000000000000E000080ED3F
:104700004401035245560000000000000000000074
:104710000000000010000000803F0205445A000025
:104720000000000000000000000000000011000078
:1047300000000000FF00000000000000000000007A
:10474000000000000000000000000000DCDFE1E3EA
:10475000E6E8EBEDEFF2F4F7F9FCFE000305080ADA
:104760000C0F111416181B1D202224272C76D88814
:10477000674F0823C1DFAE59B1B796E5E453C63A97
:1047800051997696E6C28426898C9B62407C6FFCA8
:10479000BC9C9F40BAA56FA590055A2A5C936B6C90
:1047A000676DC11BE0E40D47F520E6B5D0ED902E16
:1047B000009435770080841E0000204E000000C861
:1047C00033333333986E128341EF8D21893BE655A5
:1047D000CFFEE6DBD1844B38F77C1D90A4BBE424EC
:1047E0003284725E8100C9F1ECA1E53D6E616E001C
:1047F000696E660001021020200808102040102079
:104800004080020102010804020101020408102094
:104810004080804020100804020180040201804092
:1048200020100804020108040201010204081020FB
:10483000408001020408102040804005050505075E
:104840000508080808020202020A0A08080404040B
:104850000401010101010101010303030303030337
:1048600003040707070C0C0C0C0C0C0C0C020202C6
:104870000206060606060606060B0B0B0B0B0B0BB9
:104880000B05000020002300260029002C002F002B
:1048900032000001000003010601090100002200AE
:1048A000250028002B002E003100340002010000FA
:1048B000050108010B0100002100240027002A0047
:1048C0002D003000330001010000040107010A013E
:1048D000494E46494E4954594E414E000020410030
:1048E00000C84200401C4620BCBE4CCA1B0E5AAE3B
:1048F000C59D74CDCCCC3D0AD7233C17B7D13877B2
:10490000CC2B329595E6241FB14F0A000D94857883
:104910000D94DC0C0D94F0860D944B680D9493511E
:104920000D94FD0D0D9454210D94421A0D94485D83
:104930000D94793D0D94CF200D94E5770D94DA5CBC
:104940000D94A7210D94C7100D94EC4F0D94433D89
:104950000D947B210D94931A0D94FC190D943B50EA
:104960000D945D170D9462800D94FD7A0D94726420
:104970000D942E440D941D890D946E640D94AE65B6
:104980000D9431180D94177F0D94198D0D94E980B5
:104990000D94AB210D948A800D94B8590D943C3E32
:1049A0000D945B1A0D94E9640D947D210D94953B53
:1049B0000D9460220D94A11A0D94B7170D94C03573
:1049C0000D94A22D0D9477670D94C71D0D944B196E
:1049D0000D9424120D94FE450D94856D0D941A5D71
:1049E0000D94CC4D0D94B6430D944E5D0D948711EE
:1049F0000D944A170D940D1C0D94772D0D94F559B7
:104A00000D9425110D941C860D94842C0D94B611D3
:104A10000D94171F0D94CA640D94142A0D94977366
:104A20000D94B3800D9459110D940A510D944B655A
:104A30000D949D1F0D947D220D941D850D94276B63
:104A40000D944D520D94F2190D9437420D94366821
:104A50000D94AF820D94DC1B0D94620C0D94071B1A
:104A60000D947D100D9456800D94E6170D94D91178
:104A70000D943D7C0D94AA220D94B5820D94E48A88
:104A80000D9426120D94640A0D94E5140D94DC8F98
:104A90000D9404500D94C9210D94877F0D94A01995
:104AA0000D94F6860D949A190D9474510D94B401D9
:104AB0000D94C66F0D94A9140D94C5000D94C714E0
:104AC0000D94DB080D94A1520D9405890D949C1151
:104AD0000D948E5D0D94D51A0D94F9520D94941980
:104AE0000D945C520D9474610D9443770D94B481D0
:104AF0000D94471A0D943D1A0D94D41F0D948650B1
:104B00000D9441190D94F5880D9464050D942517A5
:104B10000D94B90F0D947E810D94037B0D94AE011D
:104B20000D94DD220D947E680D94405E0D94E7880F
:104B30000D94BA350D94787B0D94E21B0D94251AD3
:104B40000D94837E0D94DA190D94A20C0D94380106
:104B50000D94936C0D94706B0D945E330D948219CB
:104B60000D94C3210D94BA1A0D9498100D94865D7E
:104B70000D940C5B0D9437510D945D190D948914AF
:104B80000D94067E0D947A0C0D948B690D945A50F9
:104B90000D94AA1C0D94751A0D94137A0D94A60009
:104BA0000D94601A0D94A2590D9431520D94863BC8
:104BB0000D94AD7D0D949D080D94D5030D9466550F
:104BC0000D94F1420D942B170D946C840D94B37DCC
:104BD0000D948A290D94F90D0D94FE4C0D946B4B98
:104BE0000D9423830D94D6190D94EC190D94F9931B
:104BF0000D9423550D94377C0D94A13B0D94D183D6
:104C00000D94FE080D94C70E0D943C220D94561A77
:104C10000D9406810D94D2810D94E33D0D94BC65F5
:104C20000D94031B0D94E20C0D94B0430D94DE76AD
:104C30000D94C30B0D9409140D94852C0D94A408A8
:104C40000D94777E0D94FB190D948C140D94840CA7
:104C50000D94CA500D9437180D94B1140D94F28927
:104C60000D94AA500D9444210D948F850D940F1C22
:104C70000D946C6C0D94A90D0D94D1670D94B873BF
:104C80000D945E380D944A080D94B4840D94DC2381
:104C90000D94A41D0D943F110D94BF1A0D94F18134
:104CA0000D94FD150D94F7090D947E1B0D946F1A4C
:104CB0000D9483210D9423120D94B0590D94D26557
:104CC0000D94882C0D9444080D940F1B0D94E41939
:104CD0000D94AA490D94B8080D9435250D94FF4FF5
:104CE0000D9496240D9467150D9433770D948D16BD
:104CF0000D94E3220D94210D0D9463500D94B75043
:104D00000D942D500D9499190D9461190D94B714AB
:104D10000D94EE880D946F170D9422090D94CF65B4
:104D20000D9450190D94A8590D94D4500D94D90296
:104D30000D9471810D9429830D9419520D948E5AFE
:104D40000D949C1A0D949C0C0D9486190D94393970
:104D50000D94B1550D9444810D94DD210D94CE1A1E
:104D60000D946C100D94B51A0D94D7830D946C7D31
:104D70000D94C9700D9457850D9485140D94B259F6
:104D80000D940A1B0D9499810D94AE150D948220FB
:104D90000D9402060D94551E0D9451650D94231B20
:104DA0000D94651A0D94794A0D947B260D94242256
:104DB0000D94CA570D9422170D94D61F0D94E86CCC
:104DC0000D947F780D94A1510D94EB770D94C480D0
:104DD0000D9497480D94C3190D94C35B0D943F1B1C
:104DE0000D949C2D0D94CE650D947A830D94E25410
:104DF0000D9464380D94B40C0D94AA210D942B09D4
:104E00000D9457880D9419220D947C190D946E19E8
:104E10000D9474190D94E6100D94DB880D94C45A0A
:104E20000D94FD1A0D94F6190D9469640D94DF52DA
:104E30000D949B3B0D945E1F0D94111C0D94811ECF
:104E40000D941C6E0D947D670D9420120D94FE1A26
:104E50000D94DE200D94423E0D94D27E0D9454713B
:104E60000D9463210D94DB6D0D94A31C0D941E0213
:104E70000D94B01A0D94465E0D9448220D94435241
:104E80000D94C6100D941E520D94E3640D94D865D4
:104E90000D94F60D0D94DE190D94345C0D94C853E9
:104EA0000D94F71A0D94BB7C0D94F0180D94902C72
:104EB0000D948D1F0D94128F0D94131C0D94611F72
:104EC0000D948A2C0D9444510D94AB640D94AC86D2
:104ED0000D947F0C0D94002F0D94E2230D94A61ACF
:104EE0000D94360D0D94A6140D9425470D949C2217
:104EF0000D94D2200D94511A0D94A7680D94040DB1
:104F00000D94C6520D9446190D947B3B0D940611D9
:104F10000D94CD090D949C0D0D9490140D94C62FF5
:104F20000D94B1590D94B1450D944D390D94AD08C2
:104F30000D94A2790D94CC190D9447390D946D11EF
:104F40000D941D410D946E1A0D94B8520D940F4B93
:104F50000D94D1650D944B6A0D9439580D94747766
:104F60000D94753B0D9417410D947B1E0D948A1979
:104F70000D9476710D9446690D94C5880D945A89E7
:104F80000D9478190D946F520D942B390D947E7BEE
:104F90000D946A190D94081E0D949E100D94E25103
:104FA0000D94F7500D94C5710D94C41A0D94AB1A5D
:104FB0000D94A50B0D9421220D94EB420D94BC6A27
:104FC0000D94FA2E0D940E620D94817F0D94EF03D3
:104FD0000D94371E0D94D0190D9497880D94E321EC
:104FE0000D9463510D94897A0D94EF160D94E81980
:104FF0000D942C3C0D94ED100D9437220D94BF00B0
:105000000D9427800D9400220D94B1210D946E779C
:105010000D94444F0D944C1A0D9487520D942B6FA0
:105020000D94D8200D94BC6B0D9434220D948820DF
:105030000D946B440D9485860D94021E0D941E22D2
:105040000D94EB780D9436530D94023E0D94CC2FB5
:105050000D9431260D94945D0D9482050D94CB67CB
:105060000D948A0C0D94C91A0D946A1A0D94F109C5
:105070000D94AC790D9403220D94021A0D94E04F17
:105080000D942B810D94D5200D94541E0D94B51CB8
:105090000D94CB250D94A2800D9409220D948E6160
:1050A0000D94832C0D9490190D9438190D94599AE0
:1050B0000D94DB1A0D94C9080D944C160D94E42739
:1050C0000D944A090D94661B0D943E010D94BF8CFE
:1050D0000D94618A0D9414520D9464430D94B58817
:1050E0000D947D800D94CF510D94DB480D94C30C2D
:1050F0000D9482470D944E8F0D94C9650D948B507D
:105100000D945833AABDA2F41A2646289A2478276B
:10511000A024C6BF11241FBECFEFD1E2DEBFCDBF9A
:1051200000E00CBF15E0A0E0B2E0E4EDFFE303E037
:105130000BBF02C007900D92A039B107D9F716E155
:10514000A0E9B5E001C01D92A034B107E1F711E577
:10515000C2E1D1E500E006C022970109FE010BBFC4
:105160000F94D49BC430D10780E00807A9F70E94B0
:105170000FAB0D94D99F0C940000089508950895E5
:1051800060919710709198108091991090919A1059
:10519000609354087093550880935608909357086D
:1051A0002DEC3CEC4CEC5DE30F94CD9860935808EB
:1051B0007093590880935A0890935B0880919F10D0
:1051C0009091A010A091A110B091A21080935C08C2
:1051D00090935D08A0935E08B0935F088091A31040
:1051E0009091A410A091A510B091A61080935A0997
:1051F00090935B09A0935C09B0935D096091A7103F
:105200007091A8108091A9109091AA1060936E08D7
:1052100070936F0880937008909371082DEC3CECAC
:105220004CEC5DE30F94CD98609372087093730813
:1052300080937408909375088091AF109091B0108E
:10524000A091B110B091B210809376089093770836
:10525000A0937808B09379088091B3109091B4101E
:10526000A091B510B091B610809368099093690928
:10527000A0936A09B0936B09EFE1FEE080818D7F16
:10528000808308958091971090919810A091991023
:10529000B0919A108093540890935508A0935608A3
:1052A000B093570880919B1090919C10A0919D10F5
:1052B000B0919E108093580890935908A0935A0873
:1052C000B0935B0880919F109091A010A091A110C5
:1052D000B091A21080935C0890935D08A0935E0843
:1052E000B0935F088091A3109091A410A091A51095
:1052F000B091A61080935A0990935B09A0935C0922
:10530000B0935D098091A7109091A810A091A91069
:10531000B091AA1080936E0890936F08A0937008C4
:10532000B09371088091AB109091AC10A091AD102A
:10533000B091AE108093720890937308A093740894
:10534000B09375088091AF109091B010A091B110FA
:10535000B091B2108093760890937708A093780864
:10536000B09379088091B3109091B410A091B510CA
:10537000B091B6108093680990936909A0936A0967
:10538000B0936B09EFE1FEE080818D7F808308950B
:105390008F929F92AF92BF92CF92DF92EF92FF9245
:1053A0008090B7109090B810A090B910B090BA103B
:1053B00020E030E0A901C501B4010F9400968823D4
:1053C00009F477C0C090BB10D090BC10E090BD1025
:1053D000F090BE1020E030E0A901C701B6010F94A3
:1053E0000096882309F465C080925408909255086D
:1053F000A0925608B0925708809258089092590887
:10540000A0925A08B0925B088091BF109091C01092
:10541000A091C110B091C21080935C0890935D0878
:10542000A0935E08B0935F088091C3109091C41060
:10543000A091C510B091C61080935A0990935B0952
:10544000A0935C09B0935D09C0926E08D0926F087A
:10545000E0927008F0927108C0927208D0927308BE
:10546000E0927408F09275088091C7109091C8106E
:10547000A091C910B091CA108093760890937708D4
:10548000A0937808B09379088091CB109091CC10BC
:10549000A091CD10B091CE108093680990936909C6
:1054A000A0936A09B0936B0980911F0E8D7F809342
:1054B0001F0EFF90EF90DF90CF90BF90AF909F9026
:1054C0008F9008951092EC061092DC101092DB1071
:1054D0001092DD101092DE101092DF101092EE107C
:1054E00008950F931F930091C8061091C9068091EB
:1054F000011190910211A0910311B09104111016A5
:1055000011060CF009C0222717FD2095322F08172D
:1055100019072A073B0764F48C019D0101348FE1D0
:1055200018072105310524F000E41FE120E030E0F8
:10553000B801C9011F910F910895A091CD13B091A9
:10554000CE13ED91FC9111970280F381E02DCD01F6
:10555000199508958091CD139091CE13DC01ED91B2
:10556000FC910480F581E02D199508958091CD136B
:105570009091CE13DC01ED91FC910680F781E02D36
:105580001995089580918D0790918E078F3C24E0A6
:1055900092078CF0813525E092077CF0833D25E071
:1055A00092076CF0853526E092075CF0863D9640C8
:1055B00054F484E0089580E0089581E0089582E045
:1055C000089583E0089585E0089510920D111092DA
:1055D0000E1110920F111092101110921B111092B7
:1055E0001C1110921D1110921E1110921F11109279
:1055F0002011109221111092221110922311109259
:105600002411109225111092261110922711109238
:1056100028111092291110922A1110922B11109218
:105620002C1110922D1110922E110895CF93DF930B
:10563000FC01DB01C0918606D09187062881398163
:105640001B968C911B978F931A968C911A978F9318
:1056500019968C9119978F9318968C9118978F9310
:1056600017968C9117978F9316968C9116978F9308
:1056700015968C9115978F9314968C9114978F9300
:1056800013968C9113978F9312968C9112978F93F8
:1056900011968C9111978F938C918F9383858F9313
:1056A00082858F9381858F9380858F9387818F9358
:1056B00086818F9385818F9384818F9383818F934C
:1056C00082818F9381818F9380818F93EBEAF6E0C3
:1056D00083818F9382818F9381818F9380818F9338
:1056E000E5E5F7E081818F9380818F938CEC98E2E0
:1056F0009F938F93DF93CF93D9015096ED91FC91B7
:10570000519719958DB79EB782960FB6F8949EBFA4
:105710000FBE8DBFDF91CF91089580E00895E09195
:105720008606F0918706A081B18186EA96E29F9372
:105730008F93FF93EF935096ED91FC9151971995AC
:105740000F900F900F900F9008950F931F93CF938A
:10575000DF93E0918606F0918706A081B18187E012
:1057600097E29F938F93FF93EF935096ED91FC9167
:10577000519719950F900F900F900F90C0E0D0E0C7
:105780000091C3131091C413D801ED91FC910284D0
:10579000F385E02D40E0BE01C80119952196C115A1
:1057A000B0E1DB0789F7E0918606F0918706A081DA
:1057B000B18188E197E29F938F93FF93EF93509687
:1057C000ED91FC91519719950F900F900F900F90BC
:1057D00080E0DF91CF911F910F910895A0918606EF
:1057E000B0918706ED91FC9111970284F385E02D2D
:1057F000882319F06DE373E202C060E473E2CD0127
:1058000019958091860690918706DC01ED91FC91B7
:105810000284F385E02D64E473E219950895E09124
:105820008606F0918706A081B1818BEC92E29F936E
:105830008F93FF93EF935096ED91FC9151971995AB
:105840000F900F900F900F9080E008958091CD13EE
:105850009091CE13DC01ED91FC91068CF78DE02D3B
:1058600060E0199580E0089580916E1090916F101E
:105870000097B9F020911D0E20FF13C0FC01E95BD9
:10588000FF4F80819181039761F48091721081FDB7
:1058900008C08091901083FB882780F991E08927C8
:1058A000089580E00895CF93DF93262F30E0DC0148
:1058B000CD91DC912E30310508F047C02E583F4F76
:1058C000F9010D946E9BEA85FB8560E574E23BC0AF
:1058D000EA85FB856AE574E236C0EA85FB856FE5FB
:1058E00074E231C0EA85FB8568E674E22CC0EA8583
:1058F000FB856DE674E227C0EA85FB8564E774E208
:1059000022C0EA85FB856BE774E21DC0EA85FB8552
:105910006FE774E218C0EA85FB8566E874E213C09D
:10592000EA85FB856FE874E20EC0EA85FB8564E9D1
:1059300074E209C0EA85FB856EE974E204C0EA8579
:10594000FB8564EA74E2199511C01F926F932AEAED
:1059500034E23F932F939F938F93E889F9891995A8
:105960000F900F900F900F900F900F90DF91CF91AD
:10597000089580E0089580E00895E0918606F09112
:105980008706A081B1818CE591E29F938F93FF936D
:10599000EF935096ED91FC91519719950F900F90C0
:1059A0000F900F900895FC011282138214821582C9
:1059B0001682178210861186128613861486158623
:1059C00016861786108A118A128A138A148A158AF3
:1059D000168A178A108E118E128E138E148E158EC3
:1059E000168E0895FC01138212821582148217828A
:1059F000168210860895FC01E60FF11DE60FF11DD9
:105A00003296808191810895DC01CB0118962C910A
:105A10001897FD01E20FF11DE20FF11D3296608330
:105A200091832F5F233018F418962C9308951896BD
:105A30001C920895FF920F931F93CF93DF93FC0165
:105A4000868DDF0194E0899FA00DB11D1124F42EF5
:105A5000042F152F262F372F12960D931D932D935C
:105A60003C9315978F5F873010F4868F01C0168E98
:105A7000362F272F642F752F832F922FCDB7DEB7A8
:105A8000E5E00D94609B24E0629F800D911D112440
:105A9000FC013296DC0112965C91418132812381B6
:105AA000652F742F832F922F0895CF93DF93FC01DE
:105AB00042858085833018F48F5F808702C044233D
:105AC000E1F020852150DF0182E02802A00DB11D08
:105AD0001124129612165CF0DF0182E02802A00D5C
:105AE000B11D112413967C936E9312971DC09E9145
:105AF0008E91681779074CF1EFCFEF01A0E0B0E08D
:105B000090E001972C813D812617370744F01196CC
:105B1000AA0FBB1FAE0FBF1F6D937C9305C02296CB
:105B2000A817B907C4F0F3CF81E084278287808566
:105B3000833010F4869501C08185E80FF11DE80FD0
:105B4000F11D3296808191810AC013969C938E93A9
:105B500012972150BFCF398328831196D3CFDF917D
:105B6000CF9108950F931F93CF93DF9306DF68EED5
:105B700073E080E090E0E1DC07E411E2C1E5D1E20E
:105B8000E0918606F0918706A081B1811F930F9363
:105B9000FF93EF935096ED91FC915197199584E501
:105BA00091E10F94A77468EB7BE080E090E0C5DCA6
:105BB000A0918606B0918706ED91FC911197048023
:105BC000F581E02DCD0119950F900F900F900F905A
:105BD0001816190664F1E0918606F0918706A081F7
:105BE000B181DF93CF93FF93EF935096ED91FC91AA
:105BF0005197199584E591E10F94BA7468EB7BE0B5
:105C000080E090E09ADCA0918606B0918706ED9145
:105C1000FC9111970480F581E02DCD0119950F902D
:105C20000F900F900F90181619060CF0A9CF80E076
:105C3000DF91CF911F910F910895A5E0B0E0E3E2CD
:105C4000FEE20D94479BFE01319695E0DF011D9227
:105C50009A95E9F793EA998395E99A8393E19B836F
:105C60008C836D8345E050E0BF018DE89CE00F948C
:105C7000BB7C2596E2E00D94639BACE1B0E0E3E4ED
:105C8000FEE20D943D9BFE0131969CE1DF011D92E9
:105C90009A95E9F793EA998395E99A839EE09B8325
:105CA0008C834D835E836F83788709871A872B8760
:105CB0003C87CD86DE86EF86F88A898A9A8AAB8A07
:105CC000BC8A8CA59DA5AEA5BFA58D8B9E8BAF8BE9
:105CD000B88F88A999A9AAA9BBA9898F9A8FAB8FD8
:105CE000BC8F4CE150E0BF018DE89CE00F94BB7C81
:105CF0006C96ECE00D94599BA9E1B0E0E2E8FEE27D
:105D00000D943F9B99E1FE013196DF01792F1D92A1
:105D10007A95E9F773EA798375E97A839B838C83B3
:105D20006D832E833F8348875987EA86FB860C87DD
:105D30001D87AE86BF86C88AD98A8FA198A5A9A5D6
:105D4000BAA58A8B9B8BAC8BBD8B8BA59CA5ADA577
:105D5000BEA58E8B9F8BA88FB98F49E150E0BF0104
:105D60008DE89CE00F94BB7C6996EAE00D945B9B08
:105D7000A1E1B0E0EEEBFEE20D94479BBE016F5F48
:105D80007F4F81E1FB0111928A95E9F783EA8983CC
:105D900085E98A8381E08B838091710D9091720DEA
:105DA0009D838C838091BB099091BC099F838E83D6
:105DB0008091730D9091740D998788878091BF09A8
:105DC0009091C0099B878A87809172079091730791
:105DD0009D878C878091C3099091C4099F878E8786
:105DE0008091750D9091760D998B888B41E150E0F3
:105DF0008DE89CE00F94BB7C6196E2E00D94639B80
:105E0000A4E1B0E0E6E0FFE20D94479B9E012F5F26
:105E10003F4F94E1D9011D929A95E9F793EA99834E
:105E200095E99A8398E09B839091EB069C838D8300
:105E3000FB0180818E8381818F838281888783812A
:105E40009481A581B68189879A87AB87BC87878132
:105E50009085A185B2858D879E87AF87B88B838516
:105E60009485A585B685898B9A8BAB8BBC8B44E1D9
:105E700050E0B9018DE89CE00F94BB7C6496E2E0B1
:105E80000D94639BA6E0B0E0E8E4FFE20D94479B2D
:105E9000BE016F5F7F4F96E0FB0111929A95E9F783
:105EA00093EA998395E99A8393E09B838C8380910D
:105EB0000207909103079E838D8346E050E08DE8B2
:105EC0009CE00F94BB7C2696E2E00D94639BA8E1D6
:105ED000B0E0EDE6FFE20D94399BED86FE860F877C
:105EE000188B298B3A8B4B8B5C8B6D8B7E8B8F8BBE
:105EF000988F0091ED061091EE0684E6809FB00128
:105F0000819F700D1124882777FD8095982F0F941D
:105F1000A2962B013C01209107023091080240918A
:105F2000090250910A02752D972D0F94CD989B016F
:105F3000AC016D857E858F8598890F94239560933C
:105F4000C9057093CA058093CB059093CC05209129
:105F50002F11309130114091311150913211642D37
:105F6000752D862D972D0F94CD989B01AC016989D5
:105F70007A898B899C890F9423956093CD057093C2
:105F8000CE058093CF059093D005101611061CF115
:105F9000A0923311B0923411C0923511D0923611C3
:105FA0006091EF067091F0068091F1069091F206F3
:105FB0000F94E04460933711709338118093391136
:105FC00090933A1160933B1170933C1180933D1173
:105FD00090933E1101C12BED3FE049E450E4C6012E
:105FE000B5010F9422950F94B246609333117093CC
:105FF00034118093351190933611C090320ED090A9
:10600000330EE090340EF090350E20E030E040E0AA
:106010005FE36091420E7091430E8091440E909127
:10602000450E0F94CD984B015C016091ED06709187
:10603000EE06882777FD8095982F0F94A2969B01F6
:10604000AC01C501B4010F94CD9820E030E048ECDC
:1060500052E40F94CD980F9402449B01AC01C70108
:10606000B6010F94009687FF09C0C090320ED09001
:10607000330EE090340EF090350E2AC020E030E070
:1060800040E05FE36091420E7091430E8091440EB8
:106090009091450E0F94CD986B017C016091ED06B7
:1060A0007091EE06882777FD8095982F0F94A29621
:1060B0009B01AC01C701B6010F94CD9820E030E000
:1060C00048EC52E40F94CD980F9402446B017C018C
:1060D0006091ED067091EE06882777FD8095982FE8
:1060E0000F94A29620E030E048EC52E40F94CD9853
:1060F0009B01AC01C701B6010F9407964B015C01EF
:10610000AB01BC016A017B01C401D5018093371149
:1061100090933811A0933911B0933A116091EF0622
:106120007091F0068091F1069091F2060F94E04490
:10613000A70196015058740185010F94654460933E
:106140003711709338118093391190933A116091FF
:10615000ED067091EE06882777FD8095982F0F94B5
:10616000A29620E030E048EC52E40F94CD989B01D9
:10617000AC016091420E7091430E8091440E90915B
:10618000450E0F940796462F572F682F792F6A01D7
:106190007B0140933B1150933C1160933D117093F0
:1061A0003E1120E030E0A9016091EF067091F00609
:1061B0008091F1069091F2060F94009687FF0CC033
:1061C000F7FAF094F7F8F094C0923B11D0923C119A
:1061D000E0923D11F0923E1110923F111092401149
:1061E00010924111109242111092431110924411D9
:1061F000109245111092461119821A821B821C823C
:106200001D821E821F82188619861A861B861C868E
:10621000AE014F5F5F4FBE01635F7F4F81E29EE043
:106220000E9488C46896E0E10D94559BACE0B0E014
:10623000ECE1F1E30D943E9B982E19861A861B869D
:106240001C861D821E821F82188619821A821B825A
:106250001C8280911A119816E1F181E0981659F08C
:10626000981638F082E0981639F183E098122DC024
:106270002EC0ABD92CC09E012F5F3F4F46E65CE09D
:106280006EE77CE081E29EE00E9461C3A090B709C6
:10629000B090B809C090B909D090BA09E980FA80E5
:1062A0000B811C812D813E814F81588569857A85BE
:1062B0008B859C850CDE0BC046E65CE06EE77CE0DF
:1062C00081E29EE00E9488C402C080E003C09092F8
:1062D0001A1181E02C96EBE00D945A9B8091860672
:1062E00090918706DC01ED91FC910484F585E02D09
:1062F00061EB72E2199560918606709187068DE8D0
:106300009CE00F947A8380E00895A0E0B0E0EBE891
:10631000F1E30D943F9B31DB68EE73E080E090E0A9
:106320000CD905EC19E29BECE92E99E2F92E22ED4D
:10633000C22E29E2D22E64E670E080E090E0FDD823
:1063400080916E1090916F100F945E0AE0916E1024
:10635000F0916F1023A18091860690918706DC0151
:10636000ED91FC91222309F466C01F930F939F9334
:106370008F930088F189E02D1995E0916E10F091CE
:106380006F10408551856285738580918606909156
:1063900087060F941F47E0918606F0918706A0813B
:1063A000B181FF92EF92FF93EF935096ED91FC91A4
:1063B00051971995E0916E10F0916F1044855585B5
:1063C0006685778580918606909187060F941F4792
:1063D000C0918606D0918706E0916E10F0916F1003
:1063E000A880B98082A11F928F9360897189828968
:1063F000938924E630E040E050E00F94329A5F93B6
:106400004F933F932F93DF92CF92DF93CF93D5019A
:106410005096ED91FC9151971995E0916E10F09185
:106420006F1013A28DB79EB742960FB6F8949EBF19
:106430000FBE8DBF06C00284F385E02D6AEE79E2BF
:106440001995A0918606B0918706ED91FC91119760
:106450000480F581E02DCD011995181619060CF070
:106460006ACF80E0CDB7DEB7EAE00D945B9BCF93B7
:10647000DF93C8E2D0E08091860690918706DC0128
:10648000ED91FC910284F385E02D6DE57BE119959A
:10649000219789F780918606909187060F948B8EBD
:1064A000DF91CF910895CF93DF93EC0109C021973D
:1064B00065E075E080918606909187060F949F8E27
:1064C0001C161D06A4F3DF91CF910895E091860676
:1064D000F0918706A081B1811F9288E78F9389ECA4
:1064E0009CE19F938F93FF93EF935096ED91FC91D6
:1064F00051971995BCDF82E090E0D5DF0F900F90A7
:106500000F900F900F900F900895E0918606F091F4
:106510008706A081B1818DED93E29F938F93FF93C6
:10652000EF935096ED91FC9151971995A0DFE09172
:106530008606F0918706A081B18184EE93E29F9355
:106540008F93FF93EF935096ED91FC91519719958E
:10655000809115072DB73EB7285F3F4F0FB6F894CF
:106560003EBF0FBE2DBF813049F4E0918606F09109
:106570008706A081B18180EF93E215C0811109C027
:10658000E0918606F0918706A081B18188EF93E2C1
:106590000AC08230A9F4E0918606F0918706A081B6
:1065A000B18180E094E29F938F93FF93EF93509695
:1065B000ED91FC91519719950F900F900F900F90BE
:1065C00082E090E070CFCF93DF93E0918606F09168
:1065D0008706A081B18187EB94E29F938F93FF930D
:1065E000EF935096ED91FC915197199540DF81E022
:1065F0009091DD06911101C080E0F0D8E09186060F
:10660000F09187060190F081E02DC089D1898BE857
:106610009FE00E9476FD0F94E6442091860630911B
:1066200087069F938F937F936F9380EC94E29F9361
:106630008F933F932F93FE0119958BE89FE00E9463
:10664000F8FCFC01A0918606B0918706CD91DC9103
:10665000119783858F9382858F9381858F93808512
:106660008F9387818F9386818F9385818F93848188
:106670008F9383818F9382818F9381818F93808188
:106680008F9380ED94E29F938F93BF93AF93E889AC
:10669000F98919958091860690918706DC01ED9124
:1066A000FC910284F385E02D6EEE74E21995209141
:1066B0002910EDB7FEB77C960FB6F894FEBF0FBE5B
:1066C000EDBF809186069091870621110AC0DC01FA
:1066D000ED91FC910284F385E02D6BEF74E2199546
:1066E00059C0213049F4DC01ED91FC910284F3851D
:1066F000E02D60E075E2199580912910823069F4EF
:106700008091860690918706DC01ED91FC910284D0
:10671000F385E02D69E075E21995E0918606F09128
:106720008706A081B181809135108F9380913410BC
:106730008F93809133108F93809132108F9380913B
:1067400031108F93809130108F9380912F108F9301
:1067500080912E108F9380912D108F9380912C100B
:106760008F9380912B108F9380912A108F9381E1CA
:1067700095E29F938F93FF93EF935096ED91FC9149
:1067800051971995EDB7FEB770960FB6F894FEBF06
:106790000FBEEDBF81E090E086DEDF91CF910895DE
:1067A000CF93DF93E0918606F0918706A081B181B7
:1067B00088E59BE19F938F93FF93EF935096ED9124
:1067C000FC915197199553DEA0918606B0918706EA
:1067D000CD91DC911197E3E6FBE083818F93828179
:1067E0008F9381818F9380818F93EFE5FBE083818D
:1067F0008F9382818F9381818F9380818F93EBE53B
:10680000FBE083818F9382818F9381818F9380813D
:106810008F938FE59BE19F938F93BF93AF93E8890D
:10682000F9891995A0918606B0918706CD91DC91E2
:106830001197EBE4FBE083818F9382818F938181B9
:106840008F9380818F93E7E4FBE083818F93828134
:106850008F9381818F9380818F93E3E4FBE0838129
:106860008F9382818F9381818F9380818F93E7E5CE
:10687000FBE083818F9382818F9381818F938081CD
:106880008F93E3E5FBE083818F9382818F938181F6
:106890008F9380818F93EFE4FBE083818F938281DC
:1068A0008F9381818F9380818F938BE79BE19F935F
:1068B0008F93BF93AF93E889F98919958DB79EB7E8
:1068C000C0960FB6F8949EBF0FBE8DBF82E090E0D9
:1068D000EADDDF91CF910895E0918606F091870679
:1068E000A081B18181E193E29F938F93FF93EF9316
:1068F0005096ED91FC9151971995B9DD81E09091F9
:10690000CA06911101C080E00E94EE2BE09186063C
:10691000F0918706A081B1812091CB06822F992723
:1069200087FD90959F932F9388E193E29F938F9398
:10693000FF93EF935096ED91FC915197199582E05A
:1069400090E0B1DD8DB79EB70A960FB6F8949EBF62
:106950000FBE8DBF0895CF93DF93E0918606F0912F
:106960008706A081B18186E693E29F938F93FF9380
:10697000EF935096ED91FC915197199578DDE09148
:106980008606F0918706C081D181A7E2B7E0119613
:106990008C9111978F938C918F93A3E2B7E011960E
:1069A0008C9111978F938C918F938DE693E29F93A7
:1069B0008F93FF93EF93E889F9891995E091860603
:1069C000F0918706C081D181A4E4B7E011968C9143
:1069D00011978F938C918F93A0E4B7E011968C91CF
:1069E00011978F938C918F938BE793E29F938F9363
:1069F000FF93EF93E889F9891995E0918606F09164
:106A00008706C081D181A1E6B7E011968C911197DC
:106A10008F938C918F93ADE5B7E011968C91119780
:106A20008F938C918F9389E893E29F938F93FF9339
:106A3000EF93E889F9891995E0918606F091870628
:106A4000C081D181AEE7B7E011968C9111978F93F9
:106A50008C918F93AAE7B7E011968C9111978F9341
:106A60008C918F9387E993E29F938F93FF93EF939A
:106A7000E889F9891995E0918606F09187068DB726
:106A80009EB784960FB6F8949EBF0FBE8DBFC0818F
:106A9000D181ABE9B7E011968C9111978F938C91CE
:106AA0008F93A7E9B7E011968C9111978F938C91F2
:106AB0008F9385EA93E29F938F93FF93EF93E889F7
:106AC000F9891995E0918606F0918706C081D181F8
:106AD000A9EBB7E011968C9111978F938C918F93BE
:106AE000A5EBB7E011968C9111978F938C918F93B2
:106AF00083EB93E29F938F93FF93EF93E889F98958
:106B00001995E0918606F0918706C081D181A7EDA5
:106B1000B7E011968C9111978F938C918F93A3ED81
:106B2000B7E011968C9111978F938C918F9381EC94
:106B300093E29F938F93FF93EF93E889F9891995D7
:106B4000E0918606F0918706C081D181A5EFB7E07C
:106B500011968C9111978F938C918F93A1EFB7E041
:106B600011968C9111978F938C918F938FEC93E268
:106B70009F938F93FF93EF93E889F98919958DB7C8
:106B80009EB780960FB6F8949EBF0FBE8DBF82E071
:106B900090E089DCDF91CF910895A9E1B0E0E3EDC9
:106BA000F5E30D94459B86E09FE00E9431F286E07C
:106BB0009FE00E9452ED20E030E048EC52E40F9458
:106BC000CD980F946F9660933D1270933E12809310
:106BD0003F12909340121092421210924112209153
:106BE0000D0724FF59C02091C40C20FF55C08E0111
:106BF0000F5F1F4F29E1F80111922A95E9F723EA67
:106C0000298325E92A8324E02B832091550730919D
:106C100056073D832C83688779878A879B8720E086
:106C200030E048EC52E4609143127091441280913C
:106C30004512909146120F9407966C877D878E8738
:106C40009F876091471270914812809149129091EC
:106C50004A120F946F96798B688B80914B129091AA
:106C60004C129B8B8A8B80913B1290913C129D8B96
:106C70008C8B80915707909158079F8B8E8B8091BA
:106C80004D1290914E12998F888F49E150E0B801D2
:106C90008DE89CE00F94BB7C6996E4E00D94619BC9
:106CA00089E893E10F945B5980E0089585E793E1CB
:106CB0000F945B5980E00895E0918606F091870675
:106CC000A081B18180E499E29F938F93FF93EF932A
:106CD0005096ED91FC91519719950F900F900F9050
:106CE0000F90809123079091240784319540B4F14F
:106CF00068EE73E080E090E00E949D2AE0918606B5
:106D0000F0918706A081B1818EE499E29F938F93E1
:106D1000FF93EF935096ED91FC915197199568EE82
:106D200073E080E090E00E949D2AE0918606F09159
:106D30008706A081B1818FE699E29F938F93FF939D
:106D4000EF935096ED91FC91519719958DB79EB7A1
:106D500008960FB6F8949EBF0FBE8DBF8FE793E1E4
:106D60000F945B5980E00895809192099091930966
:106D7000DC01ED91FC910480F581E02D6091E3064A
:106D800019958091920990919309DC01ED91FC9104
:106D90000284F385E02D199520E030E048E452E4C8
:106DA0000F94CD980F946F96DC01CB014FEF50E01C
:106DB00060E070E00F94BD4480933A120895809192
:106DC000DD06882321F08BE89FE00C94EDF6089512
:106DD000A0E0B0E0EEEEF6E30D943B9BEC014B013E
:106DE0003A01E0918606F09187060190F081E02D4E
:106DF000008911890F94EE8C2091860630918706C8
:106E00009F938F9380ED9BE29F938F933F932F935C
:106E1000F80119958091860690918706DC01ED9125
:106E2000FC910484F585E02D66EF7BE21995A09036
:106E30008606B090870633E5C32E3CE2D32E40EBA6
:106E4000E42E41E1F42E0CE19301A401BE018DE892
:106E50009CE00F94AF820F900F900F900F900F90C7
:106E60000F90CDB7DEB7EEE00D94579BA4E0B0E0F5
:106E7000ECE3F7E30D943E9B982EFB01C484D5848C
:106E8000E684F78486018DE89CE00F94777E5C01B0
:106E9000FEEFCF16FFEFDF0649F460918606709192
:106EA00087068DE89CE00F94238341C01C141D04C9
:106EB000CCF0E0918606F0918706A081B18183EB4A
:106EC0009BE29F938F93FF93EF935096ED91FC91EC
:106ED0005197199540E050E061E070E080E090E06B
:106EE00077DF21C022E092120DC08DE89CE00F9464
:106EF000D27EF501E81BF90BEC15FD0518F4AC1476
:106F0000BD04B8F4E0918606F0918706A081B181B6
:106F100080EC9BE29F938F93FF93EF935096ED91BC
:106F2000FC91519719950F900F900F900F908FEF44
:106F300012C09E012F5F3F4FAE014D5F5F4FB60104
:106F40008DE89CE00F94817F49815A816B817C811F
:106F5000C6013EDF80E02496EBE00D945A9BE09161
:106F60008606F0918706A081B18188EA9AE29F9314
:106F70008F93FF93EF935096ED91FC915197199554
:106F800080910D0790910E070F900F900F900F902A
:106F9000E0918606F0918706009729F4A081B181DF
:106FA00087EB9AE274C180FF11C0A081B1818CEBA4
:106FB0009AE29F938F93FF93EF935096ED91FC91FC
:106FC000519719950F900F900F900F9080910D078A
:106FD00081FF15C0E0918606F0918706A081B181FE
:106FE0008BEC9AE29F938F93FF93EF935096ED91E2
:106FF000FC91519719950F900F900F900F908091E1
:107000000D0782FF15C0E0918606F0918706A081EA
:10701000B18189ED9AE29F938F93FF93EF935096FE
:10702000ED91FC91519719950F900F900F900F9043
:1070300080910D0783FF15C0E0918606F0918706C9
:10704000A081B1818EED9AE29F938F93FF93EF938E
:107050005096ED91FC91519719950F900F900F90CC
:107060000F9080910D0784FF15C0E0918606F09186
:107070008706A081B18182EE9AE29F938F93FF935E
:10708000EF935096ED91FC91519719950F900F90B9
:107090000F900F9080910D0785FF15C0E091860637
:1070A000F0918706A081B18188EE9AE29F938F9339
:1070B000FF93EF935096ED91FC91519719950F9096
:1070C0000F900F900F9080910D0787FF15C0E091F2
:1070D0008606F0918706A081B1818EEE9AE29F9399
:1070E0008F93FF93EF935096ED91FC9151971995E3
:1070F0000F900F900F900F9080910D0790910E07B9
:1071000090FF15C0E0918606F0918706A081B181BD
:1071100083EF9AE29F938F93FF93EF935096ED91B5
:10712000FC91519719950F900F900F900F908091AF
:107130000D0790910E0791FF15C0E0918606F09122
:107140008706A081B18188EF9AE29F938F93FF9386
:10715000EF935096ED91FC91519719950F900F90E8
:107160000F900F9080910D0790910E0792FF15C020
:10717000E0918606F0918706A081B18181E09BE2D3
:107180009F938F93FF93EF935096ED91FC915197BE
:1071900019950F900F900F900F9080910D0790917F
:1071A0000E0793FF15C0E0918606F0918706A08137
:1071B000B18189E09BE29F938F93FF93EF93509669
:1071C000ED91FC91519719950F900F900F900F90A2
:1071D00080910D0790910E0794FF15C0E0918606EF
:1071E000F0918706A081B18182E19BE29F938F930A
:1071F000FF93EF935096ED91FC91519719950F9055
:107200000F900F900F9080910D0790910E0795FFB2
:1072100015C0E0918606F0918706A081B18187E1D3
:107220009BE29F938F93FF93EF935096ED91FC9188
:10723000519719950F900F900F900F9080910D0717
:1072400090910E0796FF15C0E0918606F091870693
:10725000A081B18180E29BE29F938F93FF93EF9394
:107260005096ED91FC91519719950F900F900F90BA
:107270000F9080910D0790910E0797FF15C0E09138
:107280008606F0918706A081B18186E29BE29F93FA
:107290008F93FF93EF935096ED91FC915197199531
:1072A0000F900F900F900F90809186069091870617
:1072B0000F948B8E60918606709187068DE89CE016
:1072C0000F94D18381E00895CF92DF92EF92FF92E5
:1072D0000F931F938091CD139091CE13DC01ED910C
:1072E000FC910680F781E02D19952091871230914D
:1072F000881240911B1350911C132417350779F005
:1073000030931C1320931B1360931713709318135F
:107310008093191390931A1310921D133FC020915C
:1073200014022223D9F10091171310911813209100
:10733000191330911A136B017C01C01AD10AE20AA9
:10734000F30A9701860141E8C41644E8D4064EE1E9
:10735000E406F104F8F041E040931D131BC0013432
:1073600012442F403105D0F0609317137093181317
:107370008093191390931A138091C40C80FF0EC050
:1073800060E089EA9CE00F94785A89EA9CE00F94C7
:107390001F5C04C040911D134111E1CF1F910F915B
:1073A000FF90EF90DF90CF900895EF92FF920F93B0
:1073B000CF93DF9300D01F92CDB7DEB77C010F943F
:1073C000EE8C20913A1630913B163A8329839C83A8
:1073D0008B8300ED24E0AE014F5F5F4F68E9C7018A
:1073E0000F94EC890F900F900F900F90DF91CF9139
:1073F0000F91FF90EF9008952F923F924F925F92DE
:107400006F927F928F929F92AF92BF92CF92DF92B4
:10741000EF92FF920F93CF93DF93CDB7DEB7A8978C
:107420000FB6F894DEBF0FBECDBF1C0180913212A3
:1074300090913312A0913412B09135128D8F9E8F9E
:10744000AF8FB8A380912E1290912F12A09130127D
:10745000B091311289A39AA3ABA3BCA3C0902A1206
:10746000D0902B12E0902C12F0902D128090B70942
:107470009090B809A090B909B090BA094090B309AA
:107480005090B4096090B5097090B6098091AF0929
:107490009091B009A091B109B091B2098DA39EA3BA
:1074A000AFA3B8A70E94AA2A69837A838B839C839F
:1074B0008DA19EA1AFA1B8A58D839E83AF83B88710
:1074C00049865A866B867C868D869E86AF86B88A6C
:1074D000C98ADA8AEB8AFC8A89A19AA1ABA1BCA1EC
:1074E0008D8B9E8BAF8BB88F8D8D9E8DAF8DB8A100
:1074F000898F9A8FAB8FBC8F07E22CE1AE014F5F73
:107500005F4F6EE1C1010F94EC89A8960FB6F89415
:10751000DEBF0FBECDBFDF91CF910F91FF90EF90F7
:10752000DF90CF90BF90AF909F908F907F906F90A3
:107530005F904F903F902F900895A6E2B0E0E3EA6D
:10754000FAE30D94379B9AA389A3E0916E10F09112
:107550006F10DF01A95BBF4F8D919C9102972CF0BA
:1075600040A451A462A473A404C00E94AA2A2B01BF
:107570003C0100916E1010916F10D80158962D901B
:107580003C905997F801E95BFF4FE080F180B3E050
:10759000EB16F10444F0F801EB5AFF4F6081718162
:1075A0008281938103C060E070E0CB0120E030E095
:1075B00048EC52EC0F94CD980F946F967CA36BA37C
:1075C000E2E0EE16F10444F0F801EF5AFF4F60815B
:1075D00071818281938103C060E070E0CB0120E083
:1075E00030E048EC52E40F94CD980F946F967EA350
:1075F0006DA3F2E0EF16F10444F0F801E35BFF4FF6
:10760000C080D180E280F38003C0C12CD12C7601F0
:1076100020910111309102114091031150910411F8
:1076200080916F1190917011A0917111B0917211B0
:10763000281B390B4A0B5B0BAAE0B0E00F94BE99F4
:10764000698B7A8B8B8B9C8BD80150962D913D91B9
:107650004D915C915397AAE0B0E00F94BE990091D0
:10766000091110910A1120910B1130910C11809089
:10767000051190900611A0900711B0900811498251
:107680005A826B827C828D829E82AF82B886098705
:107690001A872B873C876D877E878F87988B20E0A2
:1076A00030E048EC52E4C701B6010F94CD980F9436
:1076B0006F967E8B6D8BADA0BEA0B88EAF8A8BA06F
:1076C0009CA09A8E898E3C8E2B8E08E62CE1AE0112
:1076D0004F5F5F4F61E289A19AA10F94EC89A69652
:1076E000E2E10D94539BA4E1B0E0E9E7FBE30D94E4
:1076F000379B7C0160913B1270913C12882777FD8B
:107700008095982F0F94A29620E030E048EC52E448
:107710000F9407963B016C01609101117091021169
:1077200080910311909104110F94A29620E030E013
:1077300048EC52E40F9407961B012C0180915707E7
:10774000909158076AE070E00F94FD998B01609169
:10775000C3097091C4098091C5099091C60924E6B6
:1077600030E040E050E00F94329ACA01B90128E6B7
:1077700031E040E050E00F94329A4B015C01E0911F
:107780006E10F0916F1064897589868997890F94BE
:10779000A09620E030E048EC52E40F9407969B015D
:1077A000F82FE92F462F532F682F792F49835A83BB
:1077B0006B837C83822F932FAF2FBE2F8D839E836D
:1077C000AF83B887422D532D642D752D49875A8775
:1077D0006B877C87462D572D6C2D7D2D4D875E87C1
:1077E0006F87788B9A8A898A0B8B1C8B04E124E142
:1077F000AE014F5F5F4F6AE4C7010F94EC89649656
:10780000E2E10D94539BAAE2B0E0E9E0FCE30D94C1
:10781000379B1C018091930F9091940F9C8F8B8FBD
:107820008091910F9091920F9E8F8D8F00918F0F6D
:107830001091900F20E030E04AE754E460913D0B56
:1078400070913E0B80913F0B9091400B0F94CD981F
:107850000F946F966F8F78A389A39AA320E030E0EE
:107860004AE754E46091390B70913A0B80913B0BDD
:1078700090913C0B0F94CD980F946F966BA37CA3C3
:107880008DA39EA320E030E04AE754E46091350BDD
:107890007091360B8091370B9091380B0F94CD98E7
:1078A0000F946F966B017C0120E030E04AE754E4CE
:1078B0006091250B7091260B8091270B9091280BDE
:1078C0000F94CD982AE038EE4CE151E40F940796DE
:1078D0000F946F964B015C0120E030E04AE754E4DE
:1078E0006091210B7091220B8091230B9091240BBE
:1078F0000F94CD982AE038EE4CE151E40F940796AE
:107900000F946F962B013C0120E030E04AE754E4ED
:1079100060911D0B70911E0B80911F0B9091200B9D
:107920000F94CD982AE038EE4CE151E40F9407967D
:107930000F946F966FA378A789A79AA70E94B62A7B
:107940009B01AC0129833A834B835C831D821E8299
:107950001F8218868FA198A59A8789875C864B8697
:107960009E868D86D88ACF868BA19CA19A8B898B87
:107970008F8D98A19C8B8B8B1E8B0D8B8D8D9E8DEF
:10798000988F8F8B8B8D9C8D9A8F898F00E92AE140
:10799000AE014F5F5F4F6BE1C1010F94EC89AA9676
:1079A000E2E10D94539BAEE0B0E0E9EDFCE30D9411
:1079B000399B7C0186E09FE00E9424F04B015C0132
:1079C00086E09FE00E9418F02091120F3091130F73
:1079D0004091140F5091150F0F9422952AE037ED26
:1079E00043E25CE30F94CD986B018C0186E09FE04D
:1079F0000E9418F02B013C010E94AA2A69837A8315
:107A00008B839C832AE037ED43E25CE3C301B20140
:107A10000F94CD986D837E838F8398874C2D5D2D39
:107A2000602F712F49875A876B877C8720E030E071
:107A300048EC52E4C501B4010F94CD980F946F96B1
:107A40007E876D8703E72EE0AE014F5F5F4F6DE1EC
:107A5000C7010F94EC892E96E0E10D94559BAEE49E
:107A6000B0E0E5E3FDE30D94379B1C018BE89FE05C
:107A70000E94F8FC8C0180914F0B9091500BA091CB
:107A8000510BB091520B8BA79CA7ADA7BEA78091BD
:107A9000530B9091540BA091550BB091560B8FA79F
:107AA00098ABA9ABBAAB8091570B9091580BA091B2
:107AB000590BB0915A0B8BAB9CABADABBEAB80916D
:107AC0005B0B90915C0BA0915D0BB0915E0B8FAB4B
:107AD00098AFA9AFBAAF80915F0B9091600BA09166
:107AE000610BB091620B8BAF9CAFADAFBEAF80911D
:107AF000630B9091640BA091650BB091660B23967C
:107B00008CAF9DAFAEAFBFAF239786E09FE00E94E2
:107B100024F06B017C0186E09FE00E9418F04B018D
:107B20005C018BE89FE00E9476FD2B013C01D801AF
:107B300018966D917D918D919C911B970F946F96E6
:107B400027966CAF7DAF8EAF9FAF2797F80164810A
:107B50007581868197810F946F962B966CAF7DAF60
:107B60008EAF9FAF2B97D8016D917D918D919C9198
:107B70000F946F962F966CAF7DAF8EAF9FAF2F9700
:107B800049825A826B827C82C501B4010F946F9640
:107B90006D837E838F83988720E030E048EC52E449
:107BA000C701B6010F94CD980F946F9669877A87B5
:107BB0008B879C878FA998ADA9ADBAAD8D879E871D
:107BC000AF87B88B8BAD9CADADADBEAD898B9A8BBD
:107BD000AB8BBC8B23968CAD9DADAEADBFAD23976B
:107BE0008D8B9E8BAF8BB88F8BA59CA5ADA5BEA5AD
:107BF000898F9A8FAB8FBC8F8FA598A9A9A9BAA995
:107C00008D8F9E8FAF8FB8A38BA99CA9ADA9BEA95C
:107C100089A39AA3ABA3BCA32D96AEADBFAD2D9700
:107C2000BEA3ADA32996EEADFFAD2997F8A7EFA3AC
:107C300025968EAD9FAD25979AA789A706E82AE2DB
:107C4000AE014F5F5F4F66E9C1010F94EC89C25BE3
:107C5000DF4FE2E10D94539B0F93CF93DF93CDB7AA
:107C6000DEB728970FB6F894DEBF0FBECDBF2091C8
:107C70009F05222349F1F091C205F0FF02C0E2E026
:107C800001C0E0E0F1FDE3E02091C7053091C805B7
:107C90004091C3055091C4056091C5057091C6051A
:107CA00049835A836B837C833E832D8321E0F111CA
:107CB00001C020E02F83E8870DEB28E0AE014F5F85
:107CC0005F4F62EA0F94EC8928960FB6F894DEBFF6
:107CD0000FBECDBFDF91CF910F9108950F93CF933A
:107CE000DF9300D0CDB7DEB769834A832B8309E9E0
:107CF00023E0AE014F5F5F4F6FE20F94EC890F906E
:107D00000F900F90DF91CF910F9108950F93CF9324
:107D1000DF93CDB7DEB7E3970FB6F894DEBF0FBEA3
:107D2000CDBF69834115510541F4FE01329622E32E
:107D3000DF011D922A95E9F708C022E3FA01DE016E
:107D4000129601900D922A95E1F703E523E3AE0127
:107D50004F5F5F4F6DEF0F94EC89E3960FB6F89489
:107D6000DEBF0FBECDBFDF91CF910F91089547E9E0
:107D700051E160919611CACF84E598E00E943BC31F
:107D80008EE698E00E943BC388E898E00C943BC3E1
:107D90008AE099E00E943BC384E299E00E943BC3E1
:107DA00010925D1110925E1110925F11109260118D
:107DB000109261111092621110926311109264116D
:107DC000089584E899E00E940AD880EF98E00C9426
:107DD0003BC3AF92BF92CF92DF92EF92FF920F938D
:107DE000CF93DF93CDB7DEB72C970FB6F894DEBFF5
:107DF0000FBECDBF5C018091CD139091CE13DC01FD
:107E0000ED91FC910480F581E02D19956B017C01C9
:107E100080916E1090916F100F94BD0B29833A835F
:107E20004B835C836D837E838F839887C986DA86D4
:107E3000EB86FC8609E82CE0AE014F5F5F4F62E005
:107E4000C5010F94EC892C960FB6F894DEBF0FBED7
:107E5000CDBFDF91CF910F91FF90EF90DF90CF904A
:107E6000BF90AF900895A0E0B0E0E9E3FFE30D9488
:107E7000399B2B013C01EA01C0908409D09085090F
:107E8000E0908609F09087094A0157FF04C08824D2
:107E90009924841A950AAA2497FCA094BA2CA701C5
:107EA000960160E070E08AE793E40F9407960F94E0
:107EB0006F9686169706A806B906E4F4C301B201C8
:107EC0000F94A2964B015C01BE01882777FD809537
:107ED000982F0F94A296A70196010F9407969B01E5
:107EE000AC01C501B4010F9423950F946F964B011B
:107EF0005C0142C0A7019601C701B6010F9423950A
:107F0000A70196010F94CD989B01AC0160E070E051
:107F10008AE793E40F9407960F946F966B017C01A8
:107F20001C161D06ACF4530142018C0C9D1CAE1CAA
:107F3000BF1C9E01DE010F94A69924EF31E040E0C2
:107F400050E00F94329A820E931EA41EB51E14C0E8
:107F50009E01DE010F94A6992CE03EEF4FEF5FEFFC
:107F60000F94329A49015A018C189D08AE08BF0837
:107F7000840C951CA61CB71C18ECE12EF12C00E01B
:107F800010E0E40CF51C061D171DA3019201285CEE
:107F9000310941095109C501B4010F94C744CDB756
:107FA000DEB7E0E10D94559BCF92DF92EF92FF9206
:107FB0000F931F936B017C01261B370B480B590B4A
:107FC000CA01B9010F947E46DC01CB0166277727F1
:107FD000601B710BA8010F94BD44BC01882777FD7D
:107FE0008095982F6C0D7D1D8E1D9F1D0F944E4604
:107FF0001F910F91FF90EF90DF90CF90089588E848
:1080000096E00D94F5638F929F92AF92BF92EF929C
:108010000F931F9380914F12882309F44FC0815012
:1080200080934F128091F31480648093F3146091D5
:108030001B0770911C07882777FD8095982F0F9458
:10804000A29620E030E04AE755E40F9407960F949B
:10805000E0444B015C016091380770913907882733
:1080600077FD8095982F0F94A29620E030E04AE7A4
:1080700055E40F9407960F94E0448B019C01809186
:10808000DE0982608093DE09EE24E39480914F1232
:108090008111E12CB501A4018DEA99E00E9437D944
:1080A00080914F1281110AC08091DE098D7F8093EB
:1080B000DE098091F3148F7B8093F3141F910F914D
:1080C000EF90BF90AF909F908F900895A2E0B0E0A6
:1080D000ECE6F0E40D94479BE0918606F09187066C
:1080E000A081B1811F928F9386E394E29F938F9337
:1080F000FF93EF935096ED91FC9151974A836983DA
:108100001995698180918606909187060E94532C6B
:10811000E0918606F0918706A081B1818FE394E219
:108120009F938F93FF93EF935096ED91FC9151970E
:1081300019950FB6F894DEBF0FBECDBFE09186064D
:10814000F09187064A81A081B181442319F083EB25
:1081500094E202C08BE494E29F938F93FF93EF939A
:108160005096ED91FC91519719950F900F900F90AB
:108170000F902296E2E00D94639B0F931F93CF9391
:10818000DF93E0918606F0918706A081B18188E2B5
:1081900094E29F938F93FF93EF935096ED91FC9110
:1081A000519719950E94373206E017E00F900F9013
:1081B0000F900F90C0E0D0E0F80161918F014091E5
:1081C0000C07552747FD50950C2E02C05695479534
:1081D0000A94E2F741708C2F79DF2196C630D105E1
:1081E00059F782E090E00E945332DF91CF911F91C6
:1081F0000F910895E0918606F0918706A081B181E4
:1082000089ED95E29F938F93FF93EF935096ED91B5
:10821000FC91519719950F900F900F900F90A0918E
:108220008606B0918706ED91FC9111970084F18547
:10823000E02DCD0119958F3F2FEF920781F38937FC
:10824000910519F089359105F1F40F944568E09195
:108250008606F0918706A081B18188E096E29F931F
:108260008F93FF93EF935096ED91FC915197199551
:1082700068EE73E080E090E00E949D2A0F900F90DE
:108280000F900F90FFCF8FEF08950F931F93809162
:10829000471190914811892B09F45FC00E94AA2AC6
:1082A0000091491110914A1120914B1130914C11BC
:1082B000601B710B820B930B00914D1110914E11AD
:1082C00020E030E0601771078207930708F445C08B
:1082D0003DC00E94AA2A6093491170934A1180936D
:1082E0004B1190934C1160914F11862F8450843024
:1082F000C0F4209147118091CB139091CC13DC01F5
:10830000ED91FC9120FF05C0409150115091511109
:1083100004C040915211509153110684F785E02D0D
:10832000199580914F11853021F484E591E10F94E6
:10833000E6748091471190914811181619066CF453
:108340000197909348118093471107C0809147117E
:1083500090914811892B09F0BCCF1F910F9108957E
:10836000CF92DF92EF92FF920F931F9300915511DE
:1083700010915611209157113091581180915B1234
:1083800090915C12A0915D12B0915E12801B910BD6
:10839000A20BB30BB7FF07C0B095A0959095819540
:1083A0009F4FAF4FBF4F853F9140A105B10594F15D
:1083B00000935B1210935C1220935D1230935E1257
:1083C000C901B801605B794B8F4F9F4F24E630E0C5
:1083D00040E050E00F94329ACA01B9010F94A2967E
:1083E0000F94E0446B017C010F9404966093190292
:1083F00070931A0280931B0290931C02C701B6016E
:108400000F94309960935F127093601280936112A1
:10841000909362121F910F91FF90EF90DF90CF9099
:108420000895A0E0B0E0E7E1F2E40D943E9BEC019A
:108430008091EB06992787FD90956817790714F0CE
:10844000188282C08FE0869F5001879FB00C112454
:108450008AEFB81A0091C3131091C413D801ED919B
:10846000FC910280F381E02DB501C8011995888344
:10847000D801ED91FC91B5016F5F7F4F0280F381D0
:10848000E02DC8011995982E8983D801ED91FC91B2
:10849000B5016E5F7F4F0280F381E02DC801199511
:1084A0008A83D801ED91FC91B5016D5F7F4F068005
:1084B000F781E02DC80119956B837C838D839E83A2
:1084C000D801ED91FC91B501695F7F4F0680F7817E
:1084D000E02DC80119956B017C01CF82D886E98611
:1084E000FA86D801ED91FC91B501655F7F4F06805A
:1084F000F781E02DC8011995AB01BC014B875C8762
:108500006D877E8794FE20C08091731190917411C5
:10851000A0917511B09176118C0D9D1DAE1DBF1DE2
:108520008F839887A987BA87809177119091781166
:10853000A0917911B0917A11840F951FA61FB71FD2
:108540008B879C87AD87BE87CE01CDB7DEB7EBE0CA
:108550000D945A9B892B79F48091C7139091C8137D
:10856000DC01ED91FC910088F189E02D19958823BB
:1085700011F080E0089581E00895A4E0B0E0E3EC1C
:10858000F2E40D94479B20910D0730910E07232BA9
:1085900081F093EA998395E99A839DE09B838C838C
:1085A00044E050E0BE016F5F7F4F8DE89CE00F9488
:1085B000BB7C2496E2E00D94639BA2E0B0E0E3EE86
:1085C000F2E40D94459B8B01823008F441C0BE015A
:1085D0006F5F7F4FD8011A968D919C911B970F94D6
:1085E0007F6D2091860630918706009739F5F90155
:1085F000408151818DB79EB70A970FB6F8949EBF00
:108600000FBE8DBFADB7BEB711968AE0F8013A969E
:1086100001900D928A95E1F78BE493E29F938F93FB
:108620003F932F93DA015096ED91FC915197199554
:108630000FB6F894DEBF0FBECDBF74C049815A811A
:10864000D8011A966D917C911B970F94C6726AC0DF
:1086500088E090E00E9453320E9466320E94AB3460
:108660000E948532E0918606F0918706A081B18153
:1086700088E094E29F938F93FF93EF935096ED9150
:10868000FC91519719950E9437320F900F900F90DF
:108690000F9080919406811102C00E94EE2B809170
:1086A00094068330A9F4E0918606F0918706A081B4
:1086B000B18184E194E29F938F93FF93EF9350965F
:1086C000ED91FC91519719950F900F900F900F908D
:1086D000809194068430A9F4E0918606F091870693
:1086E000A081B1818AE194E29F938F93FF93EF93EE
:1086F0005096ED91FC91519719950F900F900F9016
:108700000F9082E090E00E9453320E946C3435DD7D
:108710000E94D0330E94E3328091860690918706B2
:108720000F94917380E02296E4E00D94619B4F9248
:108730005F926F927F928F929F92AF92BF92CF92F1
:10874000DF92EF92FF92CF93DF93EC01009709F451
:1087500099C08091040790910507843F914009F0EA
:1087600073C090C08090FB069090FC06B4018827EF
:1087700077FD8095982F0F94A2966B017C01B5012F
:1087800068197909882777FD8095982F0F94A2960C
:108790002B013C01BE0168197909882777FD809576
:1087A000982F0F94A2969B01AC01C301B2010F94C4
:1087B000CD982B013C0164EF71E068197909882795
:1087C00077FD8095982F0F94A2969B01AC01C30171
:1087D000B2012EC084EFA81681E0B80609F452C099
:1087E000BE01882777FD8095982F0F94A2966B0184
:1087F0007C01B501645F7140882777FD8095982FD3
:108800000F94A2964B015C0168EE73E06C1B7D0B2C
:10881000882777FD8095982F0F94A2969B01AC0135
:10882000C501B4010F94CD9820E030E04AEF53E445
:108830000F9407969B01AC01C701B6010F942395D5
:108840000F946F96EB011EC048EE53E060E070E0BD
:10885000CE010F94BD445C014CEB52E06CE271E040
:1088600080910407909105070F94BD44EC0190930B
:1088700005078093040724EFA21621E0B2060CF44A
:1088800071CFA8CFCE01DF91CF91FF90EF90DF9015
:10889000CF90BF90AF909F908F907F906F905F90A0
:1088A0004F900895CF92DF92EF92FF92CF93DF9394
:1088B000EC0120E030E0A9016091ED127091EE1220
:1088C0008091EF129091F0120F940096811112C0D6
:1088D0006091020770910307882777FD8095982F94
:1088E0000F94A2966093ED127093EE128093EF12A4
:1088F0009093F0128091FB069091FC068C179D07D7
:108900000CF064C080913B1290913C12CB9687375B
:10891000910508F05BC08091BB099091BC09A091C2
:10892000BD09B091BE098D509E4FAF4FBF4F873EDE
:108930009340A105B10508F049C08091BF0990910D
:10894000C009A091C109B091C2098D509E4FAF4F8F
:10895000BF4F873E9340A105B105C0F524EA30E73B
:108960004DE75FE36091ED127091EE128091EF128E
:108970009091F0120F94CD986B017C01BE01882775
:1089800077FD8095982F0F94A2962AE037ED43E269
:108990005CE30F94CD989B01AC01C701B6010F9425
:1089A00023959B01462F532F682F792F4093ED126B
:1089B0005093EE126093EF127093F012622F732FA8
:1089C0000F946F967093030760930207DF91CF9126
:1089D000FF90EF90DF90CF900895A8E0B0E0E3EF34
:1089E000F4E40D94379B2B013C011A01890180911D
:1089F000011190910211A0910311B0910411481A34
:108A0000590A6A0A7B0AC0908409D0908509E090CF
:108A10008609F090870920E030E0A901C701B6017E
:108A20000F940096882309F466C0A7019601C70138
:108A3000B6010F942395A70196010F94CD989B0141
:108A4000AC0160E070E08AE793E40F9407960F941E
:108A50006F966B017C01D701C601880F991FAA1F71
:108A6000BB1F84159505A605B7058CF4A3019201DB
:108A70002C193D094E095F09A4EFB1E00F94BE998E
:108A80000F94A2960F9402444B015C0137C0AEEFE5
:108A9000BFEFA70196010F94CA99461657066806BC
:108AA0007906D4F422273327A90124193509460968
:108AB00057092C193D094E095F09A4EFB1E00F9445
:108AC000BE990F94A2960F9402444B015C01B7FA31
:108AD000B094B7F8B09412C0B301A20184E899E051
:108AE0000E94F8D70F94A296462F572F682F792F00
:108AF0004A015B0103C0812C912C5401B8018827E5
:108B000077FD8095982F0F94A2966B017C01B1019F
:108B1000882777FD8095982F0F94A2969B01AC0132
:108B200087017601C501B4010F9465446D837E838E
:108B30008F8398870E94AA2A6B017C018091F11291
:108B40009091F212A091F312B091F412A701960144
:108B5000281B390B4A0B5B0B2536310541055105A6
:108B6000C0F01092F5121092F6121092F7121092B5
:108B7000F8128D819E81AF81B8858093F912909310
:108B8000FA12A093FB12B093FC12812C912C540189
:108B90006BC08090F5129090F612A090F712B090F2
:108BA000F81260913B1270913C12882777FD8095F6
:108BB000982F0F94A2969B01AC016D817E818F81CD
:108BC00098850F942295A50194010F9422952FE981
:108BD0003BEA4DE45EE30F94CD989B01AC01C501E7
:108BE000B4010F9423956093F5127093F61280935D
:108BF000F7129093F8128090F9129090FA12A090C8
:108C0000FB12B090FC12A50194016D817E818F81D1
:108C100098850F9422952FE93BEA4DE45EE30F948B
:108C2000CD98162F272E382E092F762F272F322D4D
:108C3000432D502FC501B4010F9423956093F91271
:108C40007093FA128093FB129093FC1220E030E0B4
:108C500048E452E4612F722D832D902F0F94CD980C
:108C60000F946F964B015C01C092F112D092F212F8
:108C7000E092F312F092F4122091F5123091F61274
:108C80004091F7125091F8126091D6087091D70870
:108C90008091D8089091D9080F94CD980F946F9631
:108CA00069837A838B839C8369817A818B819C81A0
:108CB000680D791D8A1D9B1DE12C1DE7F12E00E03A
:108CC00010E020E033E84FEF5FEF0F94C7441B0143
:108CD000182F092F20910D0730910E0734FF38C04F
:108CE00020911007273009F453C0253289F550C070
:108CF0001092C4126091F5127091F6128091F712E1
:108D00009091F8120F946F96AB01BC018091D80539
:108D10008F938091D7058F938091D6058F93809103
:108D2000D5058F930F931F933F922F92812C912CF7
:108D30005401C12CD12C760109811A812B813C81EF
:108D400087E00E943D2E0FB6F894DEBF0FBECDBF68
:108D50002092FD123092FE1281E08093E61220E014
:108D600030E0A9016D817E818F8198850F940096F6
:108D7000811105C0809157079091580793DD40926B
:108D8000361250923712609238127092391208C01F
:108D90002091C4122F5F2093C4122A30C8F2A8CFAA
:108DA0002896E2E10D94539BA0E0B0E0EAEDF6E4F2
:108DB0000D943D9BBC0197FF05C08091C30C82FFC1
:108DC00007C026C0009721F18091C30C83FD20C00D
:108DD000882777FD8095982F0F94A2962AE037ED8B
:108DE00043EA5CE30F94CD989B01AC016091E712DC
:108DF0007091E8128091E9129091EA120F942395F4
:108E00006093E7127093E8128093E9129093EA124C
:108E1000C0900111D0900211E0900311F090041164
:108E2000C701B60162517D4F8F4F9F4F0F94A2969D
:108E30004B015C01C701B6016E5E72408109910968
:108E40000F94A2969B01AC016091E7127091E81219
:108E50008091E9129091EA12850174010F946544A2
:108E60006093E7127093E8128093E9129093EA12EC
:108E70008DE995E00E944AC080FF3AC02091AA0582
:108E80003091AB054091AC055091AD056091A205C4
:108E90007091A3058091A4059091A5050F9422954A
:108EA00020E030E048EC52E40F94CD987B01D82FBD
:108EB000C92F762FCE01272F3F2D492F582F609194
:108EC000E7127091E8128091E9129091EA120F94E2
:108ED0007D9818166CF49E018E2D9F2DA32FB22F16
:108EE0008093E7129093E812A093E912B093EA12EC
:108EF0006091E7127091E8128091E9129091EA1264
:108F000060934312709344128093451290934612DB
:108F10002091F9063091FA0679014AEFE40EF11C2E
:108F2000C6E0DFEFC21BD30B0F946F969701AE0123
:108F300054DDCDB7DEB7ECE00D94599BA0E0B0E076
:108F4000E4EAF7E40D94399BEA0169010F94A296D3
:108F50002091E7123091E8124091E9125091EA1203
:108F60000F9422954B015C0120E030E0A901792D9E
:108F70009B2D0F94009687FF04C08091C30C82FF45
:108F80000FC020E030E0A901682D792D8A2D9B2D9E
:108F90000F947D981816F4F58091C30C83FD3AC0A8
:108FA000B601882777FD8095982F0F94A2962AE026
:108FB00037ED43EA5CE30F94CD982B013C01BE01F1
:108FC000882777FD8095982F0F94A2962AE037ED99
:108FD00043EA5CE30F94CD989B01AC0183017201DD
:108FE000682D792D8A2D9B2D0F9465449B01AC0132
:108FF0006091E7127091E8128091E9129091EA1263
:109000000F9423956093E7127093E8128093E9120E
:109010009093EA128090011190900211A090031198
:10902000B0900411C501B40162517D4F8F4F9F4F25
:109030000F94A2962B013C01C501B4016E5E7240F3
:10904000810991090F94A2969B01AC016091E712EE
:109050007091E8128091E9129091EA1283017201F5
:109060000F9465446093E7127093E8128093E912BD
:109070009093EA122AEFC20ED11CCA5FD1090F9455
:109080006F969601AE01A9DCCDB7DEB7E0E10D9495
:10909000559B80910D0780FF04C08091C40C80FD1A
:1090A00009C080910D0787FF0EC08091C40C80FD20
:1090B00004C008950E94B82EF4CF6BE17BE08DE8E8
:1090C0009CE00D9416860895AFE0B0E0EAE6F8E47F
:1090D0000D94479B8091C40C80FF43C080910D0785
:1090E00081FD0E94B82E80910D0790910E0792FF8E
:1090F00038C0BE016F5F7F4F8FE0FB0111928A95F0
:10910000E9F783EA898385E98A838BE08B83809101
:10911000B30C9091B40C9D838C838091B50C90918D
:10912000B60C9F838E838091B70C9091B80C998771
:1091300088878091B90C9091BA0C9B878A8780911F
:10914000BB0C9091BC0C9D878C878091BD0C90913D
:10915000BE0C9F878E874FE050E08DE89CE00F9417
:10916000BB7C2F96E2E00D94639BADE3B0E0EBEBAC
:10917000F8E40D94379B80911D0E85FF7BC287E933
:109180009BE00F94CD248111C1C174C28091CD1395
:109190009091CE13DC01ED91FC910480F581E02DDE
:1091A00019950F94A0962B013C0120916C123091DF
:1091B0006D1240916E1250916F120F94229520E023
:1091C00030E04AE754E40F9407964B015C012CE52C
:1091D0003FE842EC5DE3792D9B2D0F947D9887FD50
:1091E0006EC12090ED063090EE061AAE1BAE1CAE9E
:1091F0001DAE1EAA1FAA18AE19AE1AAA1BAA1CAA37
:109200001DAA20E030E040E85FE3682D792D8A2D2B
:109210009B2D0F947D9887FD04C0812C912CA12C4F
:10922000B12C40926C1250926D1260926E1270923C
:109230006F1220E030E0A9016091EF067091F00616
:109240008091F1069091F2060F947D98C0904311A1
:10925000D0904411E0904511F090461140903711A4
:10926000509038116090391170903A11A301920119
:1092700087FD2DC0C701B6010F94009687FF5EC021
:1092800020913B1130913C1140913D1150913E1184
:10929000682D792D8A2D9B2D0F94CD989B01AC01C3
:1092A000C701B6010F942395FB01462F5F2F682F4E
:1092B000792F40934311509344116093451170935B
:1092C00046118301720120E030E0A9012CC0C701E2
:1092D000B6010F947D9818168CF520913B113091B2
:1092E0003C1140913D1150913E11682D792D8A2DF0
:1092F0009B2D0F94CD989B01AC01C701B6010F9433
:109300002395FB01462F5F2F682F792F4093431140
:10931000509344116093451170934611E12CF12C48
:109320008701A3019201BF010F946544609343112B
:1093300070934411809345119093461120914311ED
:10934000309144114091451150914611682D792D6D
:109350008A2D9B2D0F94CD9820913311309134118B
:1093600040913511509136110F9423959B01462F52
:10937000532F682F792F40933311509334116093FA
:10938000351170933611622F732F0F94B2462B0153
:109390003C01609333117093341180933511909395
:1093A0003611209143113091441140914511509153
:1093B0004611682D792D8A2D9B2D0F94CD989B01F8
:1093C000AC0160913F1170914011809141119091D9
:1093D00042110F94239560933F1170934011809335
:1093E0004111909342116091ED067091EE0688272D
:1093F00077FD8095982F0F94A29620E030E0A90188
:109400000F940096882309F45AC084E6829DB00127
:10941000839D700D1124882777FD8095982F0F94D8
:10942000A2966B018C01C301B20190580F9404966F
:109430009B01AC016C2D7D2D802F912F0F94CD9829
:109440009B01AC016091C9057091CA058091CB0563
:109450009091CC050F9423956AAB7BAB8CAB9DAB05
:10946000C301B2010F9430999B01AC016C2D7D2D8D
:10947000802F912F0F94CD989B01AC016091CD0569
:109480007091CE058091CF059091D0050F942395D2
:109490006EAB7FAB88AF99AF8091780E9091790ECB
:1094A000A0917A0EB0917B0E8AAF9BAFACAFBDAFEF
:1094B000BE016E5C7F4F81E29EE00E9470C481E23B
:1094C0009EE00E94F6D211C080911E0E81FFF7CF60
:1094D00046E65CE06EE77CE081E29EE00E9488C4A4
:1094E00004C081E29EE00E9447D280916B128F5FA0
:1094F00080936B128A3008F4BDC080910D0785FF00
:10950000B9C080911A1181110AC0B4C080911A119A
:109510008230D1F2833029F3813039F737CE10927F
:109520006B128E010F5F1F4F81E3F80111928A9534
:10953000E9F783EA898385E98A8385E08B838091D3
:109540001B1190911C11A0911D11B0911E118C83C3
:109550009D83AE83BF8360910D1170910E11809138
:109560000F119091101124E630E040E050E00F948C
:10957000329A398728878091EA0E9091EB0EA0915C
:10958000EC0EB091ED0E8A879B87AC87BD878091EA
:10959000EE0E9091EF0EA091F00EB091F10E8E872D
:1095A0009F87A88BB98B8091F20E9091F30EA091BA
:1095B000F40EB091F50E8A8B9B8BAC8BBD8B80919A
:1095C000F60E9091F70EA091F80EB091F90E8E8BD9
:1095D0009F8BA88FB98F8091660C9091670CA0919A
:1095E000680CB091690C8A8F9B8FAC8FBD8F809176
:1095F0006A0C90916B0CA0916C0CB0916D0C8E8FDD
:109600009F8FA8A3B9A38091FA0E9091FB0EA09111
:10961000FC0EB091FD0E8AA39BA3ACA3BDA38091C9
:10962000FE0E9091FF0EA091000FB091010F8EA33E
:109630009FA3A8A7B9A78091680E9091690EA091E9
:109640006A0EB0916B0E8AA79BA7ACA7BDA78091AD
:109650006C0E90916D0EA0916E0EB0916F0E8EA754
:109660009FA7A8ABB9AB41E350E0B8018DE89CE0FF
:109670000F94BB7CED96E2E10D94539B21E0FC013D
:109680003081361301C020E0FC016083622F0D940D
:10969000BF71CF93DF93FB01C285D38562EF76E282
:1096A000CE010F947A9D892B11F461E018C064EF0C
:1096B00076E2CE010F947A9D892B11F460E00FC001
:1096C00066EF76E2CE010F947A9D892BB9F368EFAD
:1096D00076E2CE010F947A9D892B29F462E085E130
:1096E00097E0CCDF18C0E0918606F0918706A08154
:1096F000B1818AEF96E29F938F93FF93EF935096F9
:10970000ED91FC91519719950E9485320F900F9021
:109710000F900F9002C00E94853280E0DF91CF91C0
:109720000895AFE0B0E0E7E9FBE40D943B9BA9822C
:10973000BA82CB82DC82ED82FE820F831887298772
:109740003A874B875C876D877E878F87C401CC8083
:10975000DD80EE80FF804091EB06552747FD509558
:1097600060E070E00F94BD443C01009729F4A0E153
:10977000AA2EC12CD12C76018FE0869D4001879DB9
:10978000900C11248AEF981A0091C3131091C413FE
:10979000D801ED91FC910284F385E02D4A2DB401AE
:1097A000C8011995D801ED91FC91B4016F5F7F4F0D
:1097B0000284F385E02D4A81C8011995D801ED9105
:1097C000FC91B4016E5F7F4F0284F385E02D4B81E5
:1097D000C8011995D801ED91FC91B4016D5F7F4FDF
:1097E0000684F785E02DA7019601C8011995D801D7
:1097F000ED91FC91288539854A855B85B401695FC7
:109800007F4F0684F785E02DC8011995D801ED91A9
:10981000FC912C853D854E855F85B401655F7F4F4A
:109820000684F785E02DC80119958091EB069927EC
:1098300087FD9095681679062CF0662D6F5F8BEE8C
:1098400096E01CDF2F96EEE00D94579BFF920F934E
:109850001F93CF93DF93F82EEB010A851B8566EFEC
:1098600072E2C8010F947A9D892B11F461E008C05F
:1098700069EF72E2C8010F947A9D892B21F460E0B0
:109880008AEC96E012C081E08F1588F48C859D8566
:10989000AE85BF850497A105B10548F461E08AEC67
:1098A00096E0ECDE6C858BEC96E0E8DE18C0E0918B
:1098B0008606F0918706A081B1818DEF92E29F9399
:1098C0008F93FF93EF935096ED91FC9151971995DB
:1098D0000E946C340F900F900F900F9002C00E9466
:1098E0006C3480E0CDB7DEB7E5E00D94609BCF929D
:1098F000DF92EF92FF921F93CF93DF93EC016A0107
:109900007B0111E09A01AB01688179818A819B8199
:109910000F940096811101C010E0C882D982EA82BA
:10992000FB82612FCE010F94BF71DF91CF911F9108
:10993000FF90EF90DF90CF9008959B0161E0FC01D4
:10994000408151814217530709F460E0FC013183E3
:1099500020830D94BF71FF920F931F93CF93DF93DA
:10996000EB01E0918606F0918706A081B18184E148
:1099700096E29F938F93FF93EF935096ED91FC9116
:10998000519719956C857D8583E197E0D6DF6E89C7
:109990007F8981E197E0D1DFE0918606F09187062B
:1099A000A081B18183E496E29F938F93FF93EF931D
:1099B0005096ED91FC91519719950E943732F09095
:1099C00010078DB79EB708960FB6F8949EBF0FBECE
:1099D0008DBFF11004C080E00E94EE2B48C0C09102
:1099E0008606D091870608811981609111077091D0
:1099F0001207882777FD8095982F0F94A29620E074
:109A000030E04AE754E40F9407969F938F937F9337
:109A10006F936091130770911407882777FD8095E5
:109A2000982F0F94A29620E030E04AE754E40F9478
:109A300007969F938F937F936F938F2D992787FD21
:109A400090959F93FF928BE496E29F938F93DF9381
:109A5000CF93D8015096ED91FC91519719958DB700
:109A60009EB70E960FB6F8949EBF0FBE8DBF82E0D4
:109A700090E00E94533280E0CDB7DEB7E5E00D9470
:109A8000609BEF92FF920F931F93CF93DF937B0125
:109A90008230B9F0E0918606F0918706A081B1810D
:109AA0008EE29BE29F938F93FF93EF935096ED91FD
:109AB000FC91519719950F900F900F900F908FEF89
:109AC000AAC0FB010285138560E47BE2C8010F9404
:109AD000679D892B09F484C064E47BE2C8010F947C
:109AE000679DC1E0D0E0892B11F0C0E0D0E062E5D5
:109AF0007BE2C8010F94679D892B09F4C2606FE572
:109B00007BE2C8010F94679D892B09F4C46063E66A
:109B10007BE2C8010F94679D892B09F4C86066E653
:109B20007BE2C8010F94679D892B09F4C0616BE645
:109B30007BE2C8010F94679D892B09F4C06260E73E
:109B40007BE2C8010F94679D892B09F4C06465E727
:109B50007BE2C8010F94679D892B09F4C06869E70F
:109B60007BE2C8010F94679D892B09F4D1606DE7F2
:109B70007BE2C8010F94679D892B09F4D26065E8E8
:109B80007BE2C8010F94679D892B09F4D4606CE8CF
:109B90007BE2C8010F94679D892B09F4D86064E9C2
:109BA0007BE2C8010F94679D892B09F4D06168E9B5
:109BB0007BE2C8010F94679D892B09F4D06260EAAB
:109BC0007BE2C8010F94679D892B09F4D06465EA94
:109BD0007BE2C8010F94679D892B21F4D06802C0F5
:109BE000CFEFDFEF6CEA7BE2F701808191810F9488
:109BF000679D20910D0730910E07BE01892B19F446
:109C0000622B732B04C060957095622373238DE0E3
:109C100097E093DE80E0CDB7DEB7E6E00D945F9B82
:109C2000A2E0B0E0E6E1FEE40D94419B8B018330BD
:109C300049F0E0918606F0918706A081B18181E329
:109C400095E26EC0BE016F5F7F4FD8011A968D916D
:109C50009C911B970F947F6DFC010097B1F4E091EC
:109C60008606F091870620813181D8011B968C9160
:109C70001B978F931A968C918F938DE595E29F9306
:109C80008F93FF93EF93D9018FC089819A8182309E
:109C9000910569F12CF48130910509F077C009C074
:109CA0008330910509F44DC08430910509F06EC0F0
:109CB00063C0D80156966D917D918D919C91599775
:109CC000062F112707FD1095212F312F60177107DF
:109CD0008207930749F0E0918606F0918706A081FC
:109CE000B18182E795E21CC0CF01C8DC68C0D80111
:109CF00056966D917D918D919C9159978B0122275C
:109D000017FD2095322F6017710782079307B1F076
:109D1000E0918606F0918706A081B18184E995E201
:109D20009F938F93FF93EF935096ED91FC915197F2
:109D300019950F900F900F900F9041C0CF01FDDD4E
:109D40003EC0D8015696CD90DD90ED90FC9059978D
:109D500021E040815181628173814C155D056E0562
:109D60007F0509F420E0C082D182E282F382622F73
:109D7000CF010F94BF7123C0D8015A964D915D91C8
:109D80006D917C915D97CF01B2DD19C0E09186069F
:109D9000F0918706A081B1819F938F9387EB95E225
:109DA0009F938F93FF93EF935096ED91FC91519772
:109DB00019950F900F900F900F900F900F9080E0DB
:109DC0002296E8E00D945D9BA0E0B0E0EAEEFEE4B0
:109DD0000D94419BEB0144E951E16CE67EEE0F945A
:109DE000BD448C0144E951E16CE67EEECE010F9456
:109DF000BD44EC016091E5067091E606643981E1AD
:109E0000780749F41093720D0093710DD093740D7F
:109E1000C093730D49C08091B2129091B31268172C
:109E20007907C1F07093B3126093B212882777FD5F
:109E30008095982F0F94A29620E030EA4CE855E4E4
:109E40000F94079660932A0270932B0280932C0242
:109E500090932D02C0902A02D0902B02E0902C0209
:109E6000F0902D02B801882777FD8095982F0F94E8
:109E7000A296A70196010F94CD980F946F967093B8
:109E8000720D6093710DBE01882777FD8095982F24
:109E90000F94A296A70196010F94CD980F946F96F8
:109EA0007093740D6093730DCDB7DEB7E8E00D9439
:109EB0005D9B8091C7139091C813DC01ED91FC91DB
:109EC0000088F189E02D199520911E0E27FB992716
:109ED00090F9891709F458C080FB27F920931E0ECA
:109EE0008091B7139091B813DC01ED91FC91068835
:109EF000F789E02D27FD39C02091C606233131F1C5
:109F00005CF42230E1F11CF42130A1F510C02430C2
:109F100099F0293079F515C0293361F11CF4263206
:109F200049F519C02F36E1F0233721F51EC040EB6B
:109F300054E060E070E027C040EC52E160E070E087
:109F400022C040E855E260E070E01DC040E05BE404
:109F500060E070E018C040E056E960E070E013C0D7
:109F60004CEF51EB61E070E00EC040E052EC61E07C
:109F700070E009C040E051EE60E070E004C040E6EF
:109F800059E060E070E0199508950F93CF93DF9347
:109F9000CDB7DEB729970FB6F894DEBF0FBECDBFA1
:109FA00020911E0E21FF02C023E001C024E0E091B9
:109FB0006D104E2F552747FD5095652F752F309109
:109FC00090103E7109F025E0E350E53010F030E1EB
:109FD00001C038E1E091C40CE0FD02C0306401C072
:109FE000306C49835A836B837C834DE04D8343E01F
:109FF0004E8331603F832887498702E329E0AE0121
:10A000004F5F5F4F60E00F94EC8929960FB6F8948C
:10A01000DEBF0FBECDBFDF91CF910F910895A4E2B7
:10A02000B0E0E5E1F0E50D94379B1C012091DD06E1
:10A03000211107C09BE0492E9CEF592E612C712CF9
:10A0400006C08FE0482E8CEF582E612C712C809129
:10A050006E1090916F10009749F0FC01E95BFF4F83
:10A0600080819181181619060CF4CDC080911F0EC5
:10A0700082FF02C0689460F888248A940FE9902EC9
:10A08000A82CB82C84209520A620B72080916D1094
:10A09000883061F01CF4823074F005C08B301CF005
:10A0A0008D3049F406C080E6982A05C0689496F879
:10A0B00002C0689495F8222309F4A8C08091990FF2
:10A0C000882309F4A3C08DEA99E00E944DDE88231D
:10A0D00009F49CC01FE0C12E1CEFD12EE12CF12C05
:10A0E00080916E1090916F10009761F0FC01E95B18
:10A0F000FF4F808191811816190624F48091721007
:10A1000081FF8BC080911F0E82FF06C0809190104E
:10A1100081FD02C06894E0F880917B0B90917C0BEC
:10A12000059710F09CEFC922809194068430B9F411
:10A1300084E996E00E94A5F588A320E030E048EC91
:10A1400052E46091AB067091AC068091AD0690919F
:10A15000AE060F94CD980F946F968B0104C08FEFCD
:10A1600088A30FEF1FEF20E030E04AE754E460914E
:10A17000A7067091A8068091A9069091AA060F944F
:10A18000CD980F94749669A37AA38BA39CA340E106
:10A1900057E260E070E086E999E00F94A576498285
:10A1A0005A826B827C828D829E82AF82B886C986FB
:10A1B000DA86EB86FC8620E030E04AE754E40F9430
:10A1C000CD980F9474967E876D8789A19AA1988BFC
:10A1D0008F871A8B098B1C8A1B8A1E8A1D8A188EF0
:10A1E0001F8A1A8E198E1C8E1B8E1E8E1D8E98A194
:10A1F0009F8F0CE72FE1AE014F5F5F4F61E0C10120
:10A200000F94EC890DC0689445F830CFBBE0CB2E9D
:10A21000BCEFDB2EE12CF12C63CF6894C5F872CF34
:10A22000A496E2E10D94539BACE1B0E0EAE1F1E5E4
:10A230000D94379B5C0160913612709137128091BA
:10A240003812909139120F94A29620E030E048EC39
:10A2500052E40F9407968B018B8F9C8F60911B119A
:10A2600070911C1180911D1190911E110F94A09658
:10A2700020E030E048EC52E40F9407960F94749677
:10A280002B013C0160910D1170910E1180910F1105
:10A29000909110110F94A29620E030E048EC52E427
:10A2A0000F9407960F946F966B017C0160912B11B0
:10A2B00070912C1180912D1190912E110F94A296D6
:10A2C00020E030E048EC52E40F9407961B014C016B
:10A2D00060912711709128118091291190912A1174
:10A2E0000F94A29620E030E048EC52E40F940796D9
:10A2F00069837A838B839C83822D932DA82DB92D1E
:10A300008D839E83AF83B8873B8D2C8D802F912FBB
:10A31000A32FB22F89879A87AB87BC871D861E869D
:10A320001F86188A198A1A8A1B8A1C8ADE8ACD8A95
:10A33000D88ECF8A5A8E498E07EB2AE1AE014F5F45
:10A340005F4F6EE3C5010F94EC896C96E2E10D94CA
:10A35000539BA0E3B0E0EFEAF1E50D94379B98AB97
:10A360008FA7E0916E10F0916F1082A18F8FA08D5A
:10A37000B18DB9A3A8A3848995899BA38AA3A0A121
:10A38000B1A1BDA3ACA32089318942895389AAE038
:10A39000B0E00F94BE99698B7A8B8B8B9C8B8485F4
:10A3A0009585A685B7858EA39FA3A8A7B9A7808505
:10A3B0009185A285B3858AA79BA7ACA7BDA7DF011E
:10A3C000A95BBF4F9C919EA780A591A5A2A5B3A50F
:10A3D0001C012D01612C712C43019C01A20160E044
:10A3E00070E080E090E002E00F94749B59016A01F4
:10A3F0007B01E82F192F05E00F94749B0E2F0F940B
:10A40000B69B51016201E12CF12C00E010E00F94A9
:10A41000A19B03E00F94749B29833A834B835C8355
:10A420006D837E838F8398878AA59BA5ACA5BDA5E8
:10A4300089879A87AB87BC878EA19FA1A8A5B9A55C
:10A440008D879E87AF87B88BACA1BDA1BE8BAD8B2E
:10A450008FEF9FEF988F8F8B8AA19BA19A8F898F07
:10A46000A8A1B9A1BC8FAB8FBEA5BD8F8F8D8E8FDC
:10A4700008E12EE1AE014F5F5F4F68E18FA598A91B
:10A480000F94EC89E096E2E10D94539BA9E1B0E0D2
:10A49000ECE4F2E50D94379B988F8F8B20913A1264
:10A4A0002090E7073090E8074090C9075090CA070E
:10A4B0000091AB071091AC07E0908D07F0908E07EC
:10A4C000C0907007D0907107A0905307B0905407C8
:10A4D00080903607909037076090190770901A07A0
:10A4E000298F0E94AA2A69837A838B839C837E8228
:10A4F0006D8298868F82BA86A986DC86CB86FE8698
:10A50000ED86188B0F875A8A498A3C8A2B8A1D8AC6
:10A51000298D2E8B04EF26E1AE014F5F5F4F63E282
:10A520008F89988D0F94EC896996E2E10D94539B85
:10A53000A7E1B0E0EEE9F2E50D94379B9F8B8E8B9F
:10A540002090C10C3090C20C4090BF0C5090C00CB9
:10A550000091BD0C1091BE0CE090BB0CF090BC0CB7
:10A56000C090B90CD090BA0CA090B70CB090B80CB9
:10A570008090B50C9090B60C6090B30C7090B40CB9
:10A580000E94B62A69837A838B839C837E826D8244
:10A5900098868F82BA86A986DC86CB86FE86ED8673
:10A5A000188B0F875A8A498A3C8A2B8A1D8A0EED9E
:10A5B00025E1AE014F5F5F4F64E28E899F890F9462
:10A5C000EC896796E2E10D94539B2F923F924F9254
:10A5D0005F926F927F928F929F92AF92BF92CF9233
:10A5E000DF92EF92FF920F93CF93DF93CDB7DEB759
:10A5F000A0970FB6F894DEBF0FBECDBF1C0120910F
:10A60000630A3091640A4091650A5091660A2D8F61
:10A610003E8F4F8F58A34090670A5090680A609011
:10A62000690A70906A0A80906B0A90906C0AA090F8
:10A630006D0AB0906E0A8DEA99E00E948CDA6B0187
:10A640007C018DEA99E00E9448DA2D8D3E8D4F8D78
:10A6500058A129833A834B835C834D825E826F824B
:10A66000788689869A86AB86BC86812C912C20E8D8
:10A67000A22E2FE3B22E8D869E86AF86B88A198AC7
:10A680001A8A1B8A1C8A6D8B7E8B8F8B988FC98E42
:10A69000DA8EEB8EFC8E0FE72CE1AE014F5F5F4F41
:10A6A00063EAC1010F94EC89A0960FB6F894DEBF5F
:10A6B0000FBECDBFDF91CF910F91FF90EF90DF9054
:10A6C000CF90BF90AF909F908F907F906F905F9052
:10A6D0004F903F902F900895EF92FF920F931F930A
:10A6E0000091BB091091BC092091BD093091BE09B0
:10A6F000601B710B820B930B0F947E460F94A296F6
:10A7000020915A0930915B0940915C0950915D0993
:10A710000F94CD980F946F9620911F0E21FD11C0BC
:10A72000E090E706F090E8060091E9061091EA064D
:10A7300022273327A9012E193F09400B510B0F94F3
:10A74000C74410929B126093B8127093B912809311
:10A75000BA129093BB121F910F91FF90EF90089542
:10A76000A2E0B0E0E6EBF3E50D94379B4090C3091F
:10A770005090C4096090C5097090C60964197509A4
:10A78000860997090F947E4614E9E12E11E1F12E16
:10A7900000E010E02CE63EEE4FEF5FEF0F94C74471
:10A7A0002B013C010F94A2962091760930917709F4
:10A7B00040917809509179090F94CD980F946F9634
:10A7C000262E7A83382E20910D0730910E0734FF04
:10A7D0002DC080911007833049F534C01092C41207
:10A7E0008091D8058F938091D7058F938091D6055E
:10A7F0008F938091D5058F931F921F921F921F9266
:10A80000812C912C5401C12CD12C7601022D1A815E
:10A81000232D392FB301A20183E099830E943D2E9D
:10A820000FB6F894DEBF0FBECDBF998110929B1278
:10A830002092A0123A813093A1123092A2129093EA
:10A84000A31208C08091C4128F5F8093C4128A3013
:10A8500068F3C4CF2296E2E10D94539BEF92FF92EE
:10A860000F931F930091BF091091C0092091C10956
:10A870003091C209601B710B820B930B0F947E46C3
:10A880000F94A296209168093091690940916A0954
:10A8900050916B090F94CD980F946F9620911F0ED5
:10A8A00021FD11C0E090E706F090E8060091E9066E
:10A8B0001091EA0622273327A9012E193F09400BE0
:10A8C000510B0F94C74410929B126093C012709367
:10A8D000C1128093C2129093C3121F910F91FF90E7
:10A8E000EF9008958F929F92AF92BF92CF92DF9296
:10A8F000EF92FF920F931F930F94A2962091470817
:10A90000309148084091490850914A080F94CD98D9
:10A910000F946F964B015C016091750D7091760DEF
:10A920008091770D9091780D0F94A2966B017C0128
:10A93000C501B4010F94A29620911E0230911F020E
:10A9400040912002509121020F94CD989B01AC01BF
:10A95000C701B6010F9423950F946F966093750D00
:10A960007093760D8093770D9093780D0F944E46EB
:10A970006093750D7093760D8093770D9093780D9D
:10A98000C090C309D090C409E090C509F090C609F1
:10A990006C197D098E099F090F947E4618EEE12EF1
:10A9A00013E0F12E00E010E028E13CEF4FEF5FEF05
:10A9B0000F94C7446B017C018091C40C80FF07C0D9
:10A9C0008091570790915807892B09F003C0C12C3B
:10A9D000D12C76016091C3097091C4098091C50999
:10A9E0009091C6096C0D7D1D8E1D9F1D0F944E46C6
:10A9F0006093750D7093760D8093770D9093780D1D
:10AA0000B701A60186E799E00E94F8D710929B1241
:10AA1000680D791D8A1D9B1D6093A0127093A11271
:10AA20008093A2129093A3121F910F91FF90EF9029
:10AA3000DF90CF90BF90AF909F908F9008950F932D
:10AA4000CF93DF931F921F92CDB7DEB72091EC0614
:10AA5000332727FD30953A8329830CE122E0AE01AC
:10AA60004F5F5F4F6AE20F94EC890F900F90DF9178
:10AA7000CF910F910895CF92DF92EF92FF920F93B3
:10AA8000CF93DF93CDB7DEB769970FB6F894DEBFEB
:10AA90000FBECDBF29833A834B835C83FE82ED8258
:10AAA000D886CF82098F6115710541F4FE01399670
:10AAB00020E1DF011D922A95E9F708C020E1FB01A2
:10AAC000DE01199601900D922A95E1F70CED29E12E
:10AAD000AE014F5F5F4F66E10F94EC8969960FB648
:10AAE000F894DEBF0FBECDBFDF91CF910F91FF90E5
:10AAF000EF90DF90CF9008955093F9144093F8149D
:10AB00006093F5147093F614FB0180E090E001C0AF
:10AB10000196249179962111FBCF8093F7140D941F
:10AB20006A6BCF93DF93EC018EE792E09983888381
:10AB30008AE992E09AA389A31FAECE0181960E9472
:10AB4000D32C8CE892E09AA389A36EE47FE2CE0135
:10AB50000F94C96EDF91CF910895ACE0B0E0E3EBC4
:10AB6000F5E50D94479BFC01E256FF4F2081233011
:10AB7000DCF42617C9F06083FC01E954FF4F108212
:10AB800011821282138219821A821B821C821D82F8
:10AB90001E821F82188619861A861B861C86BE0195
:10ABA0006F5F7F4F0E94FDFC2C96E2E00D94639B4B
:10ABB000FC01A2ADB3ADA35BBF4F86A5992787FD6E
:10ABC00090958D939C9382A993A9009749F0DC01FD
:10ABD000A554BF4F26A5332727FD30952D933C93D1
:10ABE00008958BE89FE00E94D2F9882379F08BE8E2
:10ABF0009FE00E94B7F7882349F08BE89FE090938D
:10AC0000E0098093DF098DEA99E0D2CF8091860632
:10AC100090918706DC01ED91FC910484F585E02D8F
:10AC20006EE17EE1199561E083E00C941D2EACE0AD
:10AC3000B0E0EDE1F6E50D94459BFB01028513853F
:10AC400068E179E2C8010F947A9D892B39F461E0BB
:10AC50008DED96E00E943E4BC4DF3CC06BE179E293
:10AC6000C8010F947A9D892BE9F419821A821B82FC
:10AC70001C821D821E821F82188619861A861B86D8
:10AC80001C86BE016F5F7F4F8BE89FE00E94EBFC4C
:10AC90008BE89FE00E94F4FC60E08DED96E00E945E
:10ACA0003E4B18C0E0918606F0918706A081B181E5
:10ACB0008FE199E29F938F93FF93EF935096ED91DD
:10ACC000FC91519719950E94E3320F900F900F90CD
:10ACD0000F9007C060E08DED96E00F94BF710E9469
:10ACE000E33280E02C96E4E00D94619BAEE0B0E0AE
:10ACF000ECE7F6E50D94379B19861A861B861C86B1
:10AD00001D821E821F82188619821A821B821C8253
:10AD10000E94BD2CE0918606F0918706A081B1814A
:10AD200085E899E29F938F93FF93EF935096ED916F
:10AD3000FC915197199568EE73E080E090E00E94D5
:10AD40009D2A8DEA99E034DF41E050E060E070E058
:10AD50008BE19BE00F945E38E0918606F0918706C8
:10AD6000A081B1818AE899E29F938F93FF93EF933B
:10AD70005096ED91FC915197199562E370E080E057
:10AD800090E00E949D2A0FB6F894DEBF0FBECDBFA3
:10AD900053E9E52E59E2F52E8BE19BE00F943C3E02
:10ADA0002090350B9091360B9D87A091370BAE8785
:10ADB000B090380BA090390B90903A0B80903B0BE1
:10ADC00070903C0B60903D0B50903E0B40903F0BC1
:10ADD0003090400BEDE1FBE0DE0111968CE001903C
:10ADE0000D928A95E1F7CE0101960F9418530091C8
:10ADF000860610918706F801C080D1802AE038EEDF
:10AE00004CE151E40F9407969F938F937F936F9338
:10AE10003F924F925F926F927F928F929F92AF92EA
:10AE2000BF92FE85FF938D858F932F928C858F9394
:10AE30008B858F938A858F9389858F9388858F9350
:10AE40008F818F938E818F938D818F938C818F9340
:10AE50008B818F938A818F9389818F93FF92EF9259
:10AE60001F930F93D6015096ED91FC915197199530
:10AE70000FB6F894DEBF0FBECDBF68E270E080E091
:10AE800090E00E949D2AA0918606B0918706ED91E0
:10AE9000FC9111970480F581E02DCD0119951816CC
:10AEA00019060CF079CF80E02E96E2E10D94539BC9
:10AEB000AFE0B0E0EEE5F7E50D94379B8091DD065D
:10AEC000811119C0E0918606F0918706A081B181B9
:10AED0008CEE99E29F938F93FF93EF935096ED91B1
:10AEE000FC915197199580E00E94EE2B0F900F90E6
:10AEF0000F900F9051C18BE89FE00E94D2F9811111
:10AF00000EC08091860690918706DC01ED91FC9140
:10AF10000484F585E02D66EF79E219953DC18DEA4F
:10AF200099E046DE8091DE0984608093DE098BE83B
:10AF30009FE09093E0098093DF098DEA99E038DE85
:10AF40000E94E33241E050E060E070E08BE19BE082
:10AF50000F945E3860E08DEA99E00E9425DB0E9444
:10AF6000BD2CC12CD12C7601212C312C10E064E6B3
:10AF7000862E912CA12CB12C64E170E080E090E051
:10AF80000E949D2A0E94AA2A409083125090841207
:10AF90006090851270908612641975098609970968
:10AFA000643171058105910508F4D5C00E94AA2A73
:10AFB00080918312681B70E080E090E00F94A0966F
:10AFC00020E030E04AE754E40F94079660931E02B5
:10AFD00070931F0280932002909321020E94AA2A5C
:10AFE00060938312709384128093851290938612DB
:10AFF0008DEA99E00E942AEB1F5F153099F48BE8E7
:10B000009FE00E94B7F7882361F067E27AE08BE85F
:10B010009FE00E9480FD6B017C018BE89FE00E9415
:10B0200087FE10E0BFEF2B1A3B0AE5E12E16310434
:10B030000CF491C08091990F882309F47DC08BE8AE
:10B040009FE00E94F8FCFC0120812B8381818C838E
:10B0500092819D83A381AE83B481BF830581768075
:10B0600067805084418432842384E0918606F09185
:10B0700087060190F081E02D808991899A838983E8
:10B080009091930F9887A091940FA987B091910FF9
:10B09000BA87E091920FEB87F0918F0FFC87209198
:10B0A000900F2D87C701B6010F94E64420E030E0F1
:10B0B00048EC52E40F94CD980F946F960F944E463F
:10B0C000A0918606AE87B0918706BF872F923F92E8
:10B0D0004F925F926F927F920F93EF81EF93FE8179
:10B0E000FF932D812F93AC81AF93BB81BF93E985F3
:10B0F000EF93F885FF932B852F93AA85AF93BD859A
:10B10000BF93EC85EF93A50194010F94329A5F935E
:10B110004F933F932F9385E19AE29F938F93BF853F
:10B12000BF93EE85EF93E981FA8119950FB6F894F4
:10B13000DEBF0FBECDBF0DC0809186069091870601
:10B14000DC01ED91FC910484F585E02D61E57AE266
:10B150001995212C312CA0918606B0918706ED918E
:10B16000FC9111970480F581E02DCD0119951816F9
:10B1700019060CF001CF8091860690918706DC01BC
:10B18000ED91FC910484F585E02D65E67AE2199550
:10B190008BE89FE00E94F4FC80E02F96E2E10D94A2
:10B1A000539BA8E1B0E0E7EDF8E50D94419B809159
:10B1B000860690918706DC01ED91FC910484F5856B
:10B1C000E02D6DE279E219958DEA99E0F1DC41E03C
:10B1D00050E060E070E08BE19BE00F945E3880917E
:10B1E000C5139091C61320E035E03E872D87988BDC
:10B1F0008F879E012F5E3F4FAE014B5E5F4FBE01BA
:10B20000635F7F4F8BE19BE00F944739882361F1A7
:10B2100029896A895B894C893D89FE89EF89788D06
:10B22000C32E832F9F2FAE2FB72F89839A83AB8393
:10B23000BC83022F822F962FA52FB42F8D839E8340
:10B24000AF83B88719861A861B861C86DA80EB8046
:10B25000FC801E812F81388540E05A856B857C8576
:10B260008DEA99E00E94C4D90E94D03380E06896AC
:10B27000E8E00D945D9B0F931F93CF93DF93EC0158
:10B280008B0184EA92E0998388837BAF6AAF5DAFDC
:10B290004CAFFE01EA5BFF4F1082118212821382D3
:10B2A000FE01EE5BFF4F1082118212821382FE01BB
:10B2B000FE961082118212821382FE01E25BFF4F22
:10B2C00010861186128613861482158216821782C2
:10B2D0001082118212821382FE01E65AFF4F1482FD
:10B2E0001582168217821082118212821382FE0149
:10B2F000EE59FF4F14821582168217821082118236
:10B3000012821382FE01E659FF4F148215821682C3
:10B31000178210821182128213826BE37EE2CE01C9
:10B320000F94C96ED801ED91FC910088F189E02D50
:10B33000C8011995FE01E65BFF4F6083718382832C
:10B34000938389A9886089AB84EC92E09983888390
:10B35000FE01E658FF4F108611861286138614826E
:10B36000158216821782DE01AA57BF4F18961D92CA
:10B370001D921D921C921B971D921D921D921C9254
:10B380001397DE01AE56BF4F14961D921D921D926B
:10B390001C9217971D921D921D921C921397DE010D
:10B3A000A256BF4F18961D921D921D921C921B977C
:10B3B00014961D921D921D921C9217971D921D921C
:10B3C0001D921C921397DE01A655BF4F18961D9231
:10B3D0001D921D921C921B9714961D921D921D92F8
:10B3E0001C9217971D921D921D921C921397DE01BD
:10B3F000AA54BF4F18961D921D921D921C921B9726
:10B4000014961D921D921D921C9217971D921D92CB
:10B410001D921C921397DE01AE53BF4F18961D92DA
:10B420001D921D921C921B9714961D921D921D92A7
:10B430001C9217971D921D921D921C921397DE016C
:10B44000AE52BF4F18961D921D921D921C921B97D3
:10B4500014961D921D921D921C9217971D921D927B
:10B460001D921C921397DE01B39518961D921D92A2
:10B470001D921C921B9714961D921D921D921C9258
:10B4800017971D921D921D921C921397DE01A45FC7
:10B49000BE4F18961D921D921D921C921B971496DA
:10B4A0001D921D921D921C9217971D921D921D9226
:10B4B0001C921397DE01A05EBE4F1D921D921D923D
:10B4C0001C921397DE01AC5DBE4F40E050E060E897
:10B4D0007FE34D935D936D937C93139714961D9228
:10B4E0001D921D921C921797DE01A25CBE4F18960A
:10B4F0001D921D921D921C921B9714961D921D92D7
:10B500001D921C9217971D921D921D921C921397CB
:10B51000DE01A65BBE4F18961D921D921D921C92D5
:10B520001B9714961D921D921D921C9217971D92A7
:10B530001D921D921C921397DE01AE59BE4F1896B4
:10B540001D921D921D921C921B9714961D921D9286
:10B550001D921C9217971D921D921D921C9213977B
:10B5600040A351A362A373A3408B518B628B738B57
:10B570004083518362837383FE01EE58FF4F42E79D
:10B580005AE86EE07CE34083518362837383CA5838
:10B59000DF4F4AE057ED63E27CE3488359836A83D7
:10B5A0007B83DF91CF911F910F910895A0E0B0E0D0
:10B5B000ECEDFAE50D943F9BEC015B016A0179012A
:10B5C0006BEA7CE20F94C96EF50180819181A281C2
:10B5D000B38188839983AA83BB83F601808191819B
:10B5E000A281B3818C839D83AE83BF83F701808169
:10B5F0009181A281B38188879987AA87BB87F80147
:10B600008081918197FF03C09195819591099D87D4
:10B610008C8740E050E060EC7FE74E8B5F8B688F5B
:10B62000798FCDB7DEB7EAE00D945B9B1F93CF9384
:10B63000DF93EC01162F81E090E09D8B8C8B6C8F5B
:10B6400066EB76E4CE010F94C96E1E3040F4E12F14
:10B65000F0E0EE0FFF1FEA5EF94ED183C083DF9169
:10B66000CF911F910895CF93DF93EC01DFDF6BE65D
:10B6700076E4CE010F94C96EDF91CF910895AEE0CC
:10B68000B0E0E5E4FBE50D94379B5C0160E0865A91
:10B690009F4FCCDF61E0C50189589F4FC7DF62E053
:10B6A000C5018C569F4FC2DF63E0C5018F549F4F89
:10B6B000BDDF64E0C50182539F4FD5DF65E0C50162
:10B6C00084519F4FD0DF66E0C501865F9E4FCBDF80
:10B6D00067E0C501885D9E4FC6DF69E0C5018A5BF2
:10B6E0009E4FC1DF6AE0C5018C599E4FBCDFE4EF7D
:10B6F0008E2E992493949E868D868FE692E1A3E800
:10B70000BBE389839A83AB83BC83FDEC4F2EFCECB7
:10B710005F2E652CFDE37F2E4D825E826F827886E0
:10B72000AAE9CA2EA9E9DA2EA9E1EA2EAEE3FA2E99
:10B73000C986DA86EB86FC868E01035F1F4F9E0169
:10B740002F5F3F4FAE014B5F5F4FBE01675F7F4F83
:10B75000C5018B569E4F2ADF9E868D868FE692E12D
:10B76000A3E8BBE389839A83AB83BC834D825E826B
:10B770006F827886C986DA86EB86FC868E01035F47
:10B780001F4F9E012F5F3F4FAE014B5F5F4FBE01CA
:10B79000675F7F4FC50181559E4F08DF80E293E0D0
:10B7A0009E878D8719821A821B821C828AE097ED00
:10B7B000A3EABCE38D839E83AF83B8878DEC9CECBA
:10B7C000ACE4BEE389879A87AB87BC878E01035FB1
:10B7D0001F4F9E012F5F3F4FAE014B5F5F4FBE017A
:10B7E000675F7F4FC50187539E4FE0DEB0E92B2E88
:10B7F000332433943E862D8619821A821B821C8242
:10B80000C12CD12CE12C1FE3F12ECD82DE82EF8200
:10B81000F886412C512C00E8602E0FE3702E4986EB
:10B820005A866B867C868E01035F1F4F9E012F5FB9
:10B830003F4FAE014B5F5F4FBE01675F7F4FC5015A
:10B840008D519E4FB3DE3E862D8619821A821B8251
:10B850001C82CD82DE82EF82F88649865A866B860C
:10B860007C868E01035F1F4F9E012F5F3F4FAE010D
:10B870004B5F5F4FBE01675F7F4FC50183509E4F97
:10B8800095DE8CE2282E332433943E862D86198251
:10B890001A821B821C821D821E821F82188680E0F3
:10B8A00090E0A0ECB0E489879A87AB87BC878E01D3
:10B8B000035F1F4F9E012F5F3F4FAE014B5F5F4FF6
:10B8C000BE01675F7F4FC501895E9D4F6FDE9E861B
:10B8D0008D8619821A821B821C8280E090E0A0EC87
:10B8E000BFE38D839E83AF83B88780E090E0A0E4C0
:10B8F000BFE389879A87AB87BC878E01035F1F4FA1
:10B900009E012F5F3F4FAE014B5F5F4FBE01675FF0
:10B910007F4FC5018F5C9D4F49DE94E6892E912CA7
:10B920009E868D868FE892ECA5EFBDE389839A838E
:10B93000AB83BC83CD82DE82EF82F88680E090E02C
:10B94000A0E2B0E489879A87AB87BC878E01035F4A
:10B950001F4F9E012F5F3F4FAE014B5F5F4FBE01F8
:10B96000675F7F4FC501855B9D4F20DE9E868D867C
:10B970008FE892ECA5EFBDE389839A83AB83BC8308
:10B98000CD82DE82EF82F88680E090E0A0E2B0E433
:10B9900089879A87AB87BC878E01035F1F4F9E0103
:10B9A0002F5F3F4FAE014B5F5F4FBE01675F7F4F21
:10B9B000C5018B599D4FFADD750191E8E91A9DEF9C
:10B9C000F90A67ED7DE2C7010F94C96ED7014D9268
:10B9D0005D926D927C921397F501ED57FD4F1082A9
:10B9E000118212821382F501E957FD4F11821082F4
:10B9F0007501B3E7EB1ABDEFFB0A67ED7DE2C70106
:10BA00000F94C96EF7014082518262827382F50100
:10BA1000EF56FD4F1082118212821382F501EB5610
:10BA2000FD4F118210824501F5E68F1AFDEF9F0A46
:10BA300067ED7DE2C4010F94C96EC12CD12C20E9C1
:10BA4000E22E20E4F22ED401CD92DD92ED92FC9212
:10BA50001397F501E156FD4F108211821282138275
:10BA6000F501ED55FD4F118210824501B7E58B1AA6
:10BA7000BDEF9B0A67ED7DE2C4010F94C96EF4012E
:10BA8000C082D182E282F382F501E355FD4F10823C
:10BA9000118212821382F501EF54FD4F1182108240
:10BAA0004501F9E48F1AFDEF9F0A67ED7DE2C401BD
:10BAB0000F94C96ED401CD92DD92ED92FC92139752
:10BAC000F501E554FD4F1082118212821382F501B7
:10BAD000E154FD4F118210827501BBE3EB1ABDEFFB
:10BAE000FB0A67ED7DE2C7010F94C96EF701408242
:10BAF000518262827382F501E753FD4F10821182F9
:10BB000012821382F501E353FD4F318220822E967B
:10BB1000E2E10D94539B9091E406923029F093302A
:10BB200039F0913019F406C0882321F080E008959F
:10BB300087E0089582E00895873061F480911F0EB8
:10BB40008D7F80931F0E10929B120E9442298FE1DD
:10BB50000C94BD420895A8E0B0E0E1EBFDE50D9442
:10BB6000379B80911D0E867009F4E3C090911E0EE4
:10BB700092FFDFC060911B0770911C07009138078E
:10BB800010913907823031F5882777FD8095982FFD
:10BB90000F94A2964B015C018091150290911602C0
:10BBA000A0911702B09118028D839E83AF83B8874E
:10BBB000B801882777FD8095982F0F94A2966B0186
:10BBC0007C0140905712509058126090591270901A
:10BBD0005A1225C0882777FD8095982F0F94A2963A
:10BBE0004B015C018091190290911A02A0911B02F5
:10BBF000B0911C028D839E83AF83B887B8018827DC
:10BC000077FD8095982F0F94A2966B017C01409050
:10BC10005F125090601260906112709062122D81DC
:10BC20003E814F815885C501B4010F94CD98698339
:10BC30007A838B839C83A3019201C701B6010F9481
:10BC4000CD989B01AC0169817A818B819C810F9495
:10BC50002295462F572F682F792F49835A836B835C
:10BC60007C83A3019201C501B4010F94CD984B01CF
:10BC70005C012D813E814F815885C701B6010F942B
:10BC8000CD989B01AC01C501B4010F942395162FEB
:10BC9000072F1C018090070290900802A0900902D3
:10BCA000B0900A02C0902F11D0903011E090311165
:10BCB000F0903211A501940169817A818B819C8178
:10BCC0000F94CD982B013C01A7019601D8016B2F51
:10BCD0007A2F822D932D0F94CD989B01AC01C30137
:10BCE000B2010F9423950F946F9670931C07609385
:10BCF0001B0769817A818B819C819058A7019601ED
:10BD00000F94CD986B017C01A5019401F8016F2F70
:10BD10007E2F822D932D0F94CD989B01AC01C701EE
:10BD2000B6010F9423950F946F9670933907609323
:10BD300038072896E2E10D94539B811112C080913F
:10BD40001D0E8670843079F48091CF109091D010C0
:10BD5000A091D110B091D210893E9340A105B105B8
:10BD600014F00C94B0410895982F81E0923020F0A7
:10BD7000953011F080E00895089590911D0E292FBF
:10BD80002170281749F080FB90F990931D0E8823AD
:10BD900019F089E10C94BD4208958F929F92AF9261
:10BDA000BF92CF92DF92EF92FF920F931F9381E0A9
:10BDB000E4DF80E180936C11E0916E10F0916F10E0
:10BDC0008485358526859785582F80937711309304
:10BDD00078112093791190937A118085318522858D
:10BDE0009385182F809373113093741120937511DC
:10BDF0009093761110926F11109270111092711130
:10BE000010927211812C912C40E1A42EB0906D11F2
:10BE1000C0906E11D12CE0907011F09071110091D2
:10BE20007211232F30917511492F60917811709103
:10BE3000791180917A110E94914BE0916E10F091EE
:10BE40006F1000851185228533854485558566856B
:10BE5000778587E99BE00F942F2580910D079091BE
:10BE60000E0790FF05C06CE671E180E00E94002F94
:10BE70008CE691E10F9456459B01AC0160930C0256
:10BE800070930D0280930E0290930F0260E070E0B9
:10BE900080E89FE30F94079660931002709311025D
:10BEA00080931202909313021F910F91FF90EF90D5
:10BEB000DF90CF90BF90AF909F908F90089590911A
:10BEC0001D0E95FB222720F9281749F080FB95F9D4
:10BED00090931D0E882319F08FE00C94BD420895B5
:10BEE000CF93C82F40911D0E4695437050E0282FE8
:10BEF00030E042175307A9F0811102C08BE107C05F
:10BF0000813011F48AE103C00E94B0418DE10E94AA
:10BF1000BD42C370CC0F90911D0E997F9C2B9093C6
:10BF20001D0ECF910895CF93C82F80911E0E817062
:10BF30008C1759F0CC2319F080E10E94BD4280910A
:10BF40001E0EC0FB80F980931E0ECF910895809144
:10BF5000C40C80FFC2C060E089EA9CE00F94785A6C
:10BF60008091A30B8E608093A30B8BE89FE00E94CF
:10BF7000F4FC60E082E097E00F94BF7180919A0535
:10BF80008370823009F095C00E94C82984E598E04A
:10BF90000E9449C38EE698E00E9449C38AE599E071
:10BFA0000E9410D888E699E00E9410D88091540829
:10BFB00090915508A0915608B0915708809397101A
:10BFC00090939810A0939910B0939A10809158086C
:10BFD00090915908A0915A08B0915B0880939B10EA
:10BFE00090939C10A0939D10B0939E1080915C083C
:10BFF00090915D08A0915E08B0915F0880939F10BA
:10C000009093A010A093A110B093A21080915A0910
:10C0100090915B09A0915C09B0915D098093A31098
:10C020009093A410A093A510B093A61080916E08D1
:10C0300090916F08A0917008B09171088093A7103B
:10C040009093A810A093A910B093AA1080917208A1
:10C0500090917308A0917408B09175088093AB100B
:10C060009093AC10A093AD10B093AE108091760871
:10C0700090917708A0917808B09179088093AF10DB
:10C080009093B010A093B110B093B2108091680952
:10C0900090916909A0916A09B0916B098093B310DE
:10C0A0009093B410A093B510B093B61085E20E949F
:10C0B000BD4280919A058C7F80939A0580E033DFA2
:10C0C0008091DE0982608093DE098BE00E94BD4290
:10C0D0008091DE09877F8093DE090895CF93C82F72
:10C0E00080911E0E869581708C1769F0CC2311F01B
:10C0F00082E101C08CE10E94BD4280911E0EC0FB16
:10C1000081F980931E0ECF910895CF93C82F80910F
:10C110002E02C81709F483C0C43018F4C23080F46A
:10C1200004C0C43009F06FC04FC01092E6121092E4
:10C13000361210923712109238121092391265C0CE
:10C1400040913B1250913C1260910111709102118B
:10C1500080910311909104110E94333F0F94A29695
:10C160006093E7127093E8128093E9129093EA12B9
:10C170006093780E7093790E80937A0E90937B0E75
:10C1800080912E02F1DD882309F43FC00E94E13E38
:10C1900080915507909156070E949743209102077E
:10C1A00030910307821B930BBC01882777FD809594
:10C1B000982F0F94A2966093FE087093FF088093C7
:10C1C00000099093010921C080E088DF1092751268
:10C1D0001092741240913B1250913C1260910111E7
:10C1E0007091021180910311909104110E94333FCC
:10C1F0000F94A2966093E7127093E8128093E9126D
:10C200009093EA1202C080E00BC0C0932E021092FD
:10C210004E1210924D121092EC121092EB1281E01D
:10C22000CF91089590911D0E94FB222720F9281795
:10C2300051F080FB94F990931D0E9091F31480FBC4
:10C2400095F99093F314089590911D0E93FB222776
:10C2500020F9281721F080FB93F990931D0E089583
:10C2600080911D0E83FD52C0809118078130E9F145
:10C2700086FF4AC03AC081E697E00F94166E882385
:10C2800009F444C08091230790912407853195409B
:10C29000ECF58091270790912807843A9640B4F1F5
:10C2A0008091400790914107853195407CF58091C0
:10C2B000440790914507843A964044F11DC080910F
:10C2C000610790916207843A964004F180917A0761
:10C2D00090917B0785319540CCF480917E079091B9
:10C2E0007F07843A964094F00FC08DE597E00F9455
:10C2F000166E8111C7CFBFCF80915D0790915E0709
:10C30000853195401CF4DBCF81E09ECF08954F929C
:10C310005F926F927F928F929F92AF92BF92CF92D5
:10C32000DF92EF92FF92CF93DF93CDB7DEB72C97DA
:10C330000FB6F894DEBF0FBECDBF80919B12811166
:10C34000B1C06091A0127091A1128091A21290913F
:10C35000A3120F94A2966B017C016091B8127091A8
:10C36000B9128091BA129091BB120F94A2964B0110
:10C370005C012091891230918A1240918B12509168
:10C380008C12C701B6010F94CD989B01AC01C50179
:10C39000B4010F9422950F946F966093B41270932A
:10C3A000B5128093B6129093B712809126029091A5
:10C3B0002702A0912802B091290289839A83AB8336
:10C3C000BC836091C0127091C1128091C212909191
:10C3D000C3120F94A2962B013C0180908D12909075
:10C3E0008E12A0908F12B0909012809122029091A4
:10C3F0002302A0912402B09125028D839E83AF83F6
:10C40000B887A301920169817A818B819C810F9405
:10C41000CD9869877A878B879C872D813E814F8154
:10C420005885C501B4010F94CD98A70196010F94CA
:10C43000CD989B01AC0169857A858B859C850F948D
:10C4400023950F946F966093BC127093BD128093E6
:10C45000BE129093BF1229813A814B815C816D811C
:10C460007E818F8198850F94CD98A70196010F94B6
:10C47000CD986B017C01A3019201C501B4010F9419
:10C48000CD989B01AC01C701B6010F9422950F9482
:10C490006F9660939C1270939D1280939E1290935E
:10C4A0009F12B3C0823009F0B0C06091A0127091A9
:10C4B000A1128091A2129091A3120F94A2966B01E7
:10C4C0007C016091B8127091B9128091BA1290916A
:10C4D000BB120F94A2964B015C01209189123091FE
:10C4E0008A1240918B1250918C12C701B6010F94A1
:10C4F000CD989B01AC01C501B4010F9422950F9416
:10C500006F966093C5127093C6128093C712909372
:10C51000C8128091260290912702A0912802B09122
:10C52000290289839A83AB83BC836091C012709186
:10C53000C1128091C2129091C3120F94A2962B0146
:10C540003C0180908D1290908E12A0908F12B0902E
:10C5500090128091220290912302A0912402B09126
:10C5600025028D839E83AF83B887A30192016981E1
:10C570007A818B819C810F94CD9869877A878B878C
:10C580009C872D813E814F815885C501B4010F9450
:10C59000CD98A70196010F94CD989B01AC016985B8
:10C5A0007A858B859C850F9423950F946F96609365
:10C5B000C9127093CA128093CB129093CC12298126
:10C5C0003A814B815C816D817E818F8198850F944A
:10C5D000CD98A70196010F94CD986B017C01A30122
:10C5E0009201C501B4010F94CD989B01AC01C70124
:10C5F000B6010F9422950F946F96609393127093E7
:10C60000941280939512909396122C960FB6F894EC
:10C61000DEBF0FBECDBFDF91CF91FF90EF90DF90D7
:10C62000CF90BF90AF909F908F907F906F905F90D2
:10C630004F900895A0E0B0E0E0E2F3E60D94379B60
:10C64000EC01662309F4A7C020912602309127024D
:10C650004091280250912902609122027091230298
:10C6600080912402909125020F94CD98E12CF12C19
:10C6700000E81FE320E030E040E05FE30F94654412
:10C680004B015C014091BB095091BC096091BD090F
:10C690007091BE0977FF07C07095609550954195E0
:10C6A0005F4F6F4F7F4F8091BF099091C009A0915C
:10C6B000C109B091C209B7FF07C0B095A095909588
:10C6C00081959F4FAF4FBF4F6A017B0148175907B4
:10C6D0006A077B0714F46C017D0168E273E280E075
:10C6E00090E06C197D098E099F090F94A296E12CA8
:10C6F00010E8F12E0BE315E420E030E0A9010F94DF
:10C7000065442B013C01A8019701C501B4010F94B8
:10C71000CD981B018C01E090FB06F090FC06B70160
:10C72000882777FD8095982F0F94A2964B015C0186
:10C73000BE016E197F09882777FD8095982F0F9489
:10C74000A2966B017C01222D332D402F512FC30166
:10C75000B2010F9407969B01AC01C701B6010F947B
:10C76000CD98A50194010F942395E12CF12C0AE7B3
:10C7700014E4A50194010F9465440F946F969B01F6
:10C780002C1B3D0B30934C1220934B127093580787
:10C790006093570708C090935807809357071092EB
:10C7A0004C1210924B12609157077091580780916C
:10C7B00029108130A1F4882777FD8095982F0F9458
:10C7C000A29620E030E04AE754E40F940796609385
:10C7D0004210709343108093441090934510CDB74E
:10C7E000DEB7E2E10D94539BA0E1B0E0EAEFF3E69F
:10C7F0000D94379B20EA3CE043EB55E460912A120C
:10C8000070912B1280912C1290912D120F94CD9833
:10C810000F946F964090B4125090B5126090B6127B
:10C820007090B712461A570A680A790AB301A20132
:10C8300084E598E00E94ACC16D837E838F839887E6
:10C840006091620870916308809164089091650816
:10C850002091C30C20FF1FC00F946F9669837A83C9
:10C860008B839C8329813A814B815C81121613064C
:10C87000140615061CF477FE20C00DC089819A812C
:10C88000AB81BC81892B8A2B8B2BB9F01414150436
:10C890001604170494F400911E0210911F022091B7
:10C8A000200230912102B301A20184E598E00E94A8
:10C8B000BEC169837A838B839C8300911E02109191
:10C8C0001F022091200230912102B301A20184E5D0
:10C8D00098E00E944DC24B015C016D817E818F8189
:10C8E000988529813A814B815C81620F731F841F77
:10C8F000951F680D791D8A1D9B1D18E8E12E13E117
:10C90000F12E00E010E028E73CEE4FEF5FEF0F94D0
:10C91000C7441B0120910D0730910E0734FF2FC033
:10C9200020911007243009F440C3253009F43DC399
:10C93000253129F53AC31092C4122091D8052F93BE
:10C940002091D7052F932091D6052F932091D505BF
:10C950002F939F938F933F922F92C980DA80EB8021
:10C96000FC800D811E812F813885B301A20184E0F6
:10C970000E943D2E0FB6F894DEBF0FBECDBF2092B1
:10C980001D0730921E0720EA3CE043EB55E460911E
:10C990002E1270912F1280913012909131120F94BB
:10C9A000CD980F946F964090BC125090BD1260903D
:10C9B000BE127090BF12461A570A680A790AB3016C
:10C9C000A2018EE698E00E94ACC16D837E838F83C6
:10C9D000988760917C0870917D0880917E08909185
:10C9E0007F082091C30C20FF1FC00F946F966983AE
:10C9F0007A838B839C8389819A81AB81BC81181651
:10CA000019061A061B061CF477FE20C00DC02981EA
:10CA10003A814B815C81232B242B252BB9F01414F4
:10CA200015041604170494F400911E0210911F02BD
:10CA30002091200230912102B301A2018EE698E0FC
:10CA40000E94BEC169837A838B839C8300911E02FE
:10CA500010911F022091200230912102B301A20106
:10CA60008EE698E00E944DC24B015C016D817E8193
:10CA70008F81988529813A814B815C81620F731F78
:10CA8000841F951F680D791D8A1D9B1D18E8E12ED6
:10CA900013E1F12E00E010E028E73CEE4FEF5FEFEE
:10CAA0000F94C7441B0120910D0730910E0734FFEE
:10CAB0002DC020911007243009F480C2253009F4DC
:10CAC0007DC2253119F57AC22091D8052F93209186
:10CAD000D7052F932091D6052F932091D5052F931D
:10CAE0009F938F933F922F92C980DA80EB80FC80D6
:10CAF0000D811E812F813885B301A20188E60E9435
:10CB00003D2E0FB6F894DEBF0FBECDBF20923A0780
:10CB100030923B0760919C1270919D1280919E1201
:10CB200090919F120F94A2966B017C0120EA3CE049
:10CB300043EB55E4609132127091331280913412BC
:10CB4000909135120F94CD989B01AC01C701B601AD
:10CB50000F9422950F946F962B013C01B301A20113
:10CB600088E898E00E94ACC16D837E838F839887AC
:10CB70006091960870919708809198089091990813
:10CB80002091C30C21FF1FC00F946F9669837A8395
:10CB90008B839C8389819A81AB81BC81181619068D
:10CBA0001A061B061CF477FE20C00DC029813A81AD
:10CBB0004B815C81232B242B252BB9F014141504F5
:10CBC0001604170494F400911E0210911F02209184
:10CBD000200230912102B301A20188E898E00E946E
:10CBE000BEC169837A838B839C8300911E0210915E
:10CBF0001F022091200230912102B301A20188E896
:10CC000098E00E944DC24B015C016D817E818F8155
:10CC1000988529813A814B815C81620F731F841F43
:10CC2000951F680D791D8A1D9B1D14E9E12E11E1E8
:10CC3000F12E00E010E02CE63EEE4FEF5FEF0F9498
:10CC4000C7441B0120910D0730910E0734FF29C006
:10CC500020911007263029F5B6C11092C4122091F8
:10CC6000D8052F932091D7052F932091D6052F9388
:10CC70002091D5052F939F938F933F922F92C98038
:10CC8000DA80EB80FC800D811E812F813885B30115
:10CC9000A20186E00E943D2E0FB6F894DEBF0FBEC3
:10CCA000CDBF20927407309275078091E6128823D9
:10CCB00009F49AC10091FD121091FE120E94AA2A55
:10CCC0004B015C014090030A5090040A6090050AF1
:10CCD0007090060A8091FF1290910013A0910113A9
:10CCE000B0910213A5019401281B390B4A0B5B0B71
:10CCF000253631054105510548F010920313109275
:10CD00000413109205131092061348C0B801882727
:10CD100077FD8095982F0F94A2966B017C012AE0F5
:10CD200038EE4CE151E4C301B2010F9423959058C1
:10CD300020E030E048EC52E40F94CD989B01AC0128
:10CD4000C701B6010F942295E12CF12C0AEF16E4ED
:10CD500020E030E04AEF56EC0F946544C090031396
:10CD6000D0900413E0900513F0900613A7019601EC
:10CD70000F94229523E833EA44EE5DE30F94CD98B7
:10CD80009B01AC01C701B6010F9423956093031377
:10CD90007093041380930513909306138092FF12EF
:10CDA00090920013A0920113B092021360910313AA
:10CDB0007091041380910513909106130F946F9650
:10CDC000AB01BC0180EF98E00E94ACC169837A831B
:10CDD0008B839C836091FE087091FF08809100090D
:10CDE000909101092091C30C2C7069F10F946F96FA
:10CDF0002B013C01141415041604170484F420E0DC
:10CE000030E0A90160910313709104138091051320
:10CE1000909106130F94009687FF2BC014C0411405
:10CE200051046104710429F120E030E0A90160910E
:10CE300003137091041380910513909106130F94BE
:10CE40007D981816B4F460910313709104138091C7
:10CE50000513909106130F946F96AB01BC010AE085
:10CE600017ED23E23CE380EF98E00E94BEC12B0166
:10CE70003C0160910313709104138091051390910C
:10CE800006130F946F96AB01BC010AE017ED23E285
:10CE90003CE380EF98E00E944DC24B015C01609141
:10CEA000FD067091FE06882777FD8095982F0F94D8
:10CEB000A2966B017C016091FB067091FC068827AD
:10CEC00077FD8095982F0F94A2966D877E878F8728
:10CED000988B69817A818B819C81640D751D861D7B
:10CEE000971D680D791D8A1D9B1DE0910207F09129
:10CEF00003079F01442737FD4095542F620F731F8E
:10CF0000841F951F0F94A296870176012D853E857B
:10CF10004F8558890F9465440F946F961B0180913B
:10CF20000D0790910E0794FF3CC08091100782324C
:10CF300009F452C0833209F44FC0843291F54CC0D9
:10CF40001092C41260910313709104138091051321
:10CF5000909106130F946F96AB01BC018091D80598
:10CF60008F938091D7058F938091D6058F93809171
:10CF7000D5058F93C101AA2797FDA095BA2FBF931E
:10CF8000AF939F938F937301620109811A812B8163
:10CF90003C8182E20E943D2E0FB6F894DEBF0FBEA8
:10CFA000CDBF61E0C10146DB1FC02091C4122F5FDD
:10CFB0002093C4122A3008F4E2CCBDCC2091C412D4
:10CFC0002111A4CD81CD2091C4122F5F2093C412D2
:10CFD0002A3008F466CE41CE8091C4128F5F8093D0
:10CFE000C4128A30F0F2ACCF6096E2E10D94539B0C
:10CFF000CF92DF92EF92FF92CF93DF9300D01F92F8
:10D00000CDB7DEB790911D0E97FD77C18091C40C0E
:10D0100080FF0DC180912E02823009F43DC030F4B2
:10D02000882359F0813009F068C114C0833009F4B5
:10D03000B4C0843009F061C101C18091550790915D
:10D040005607181619060CF00CC00E9497437C0175
:10D0500060E010C080915507909156071816190688
:10D060002CF060E080E090E0E5DA05C10E94974393
:10D070007C0161E0C701DEDAC7010E945244809161
:10D080001E0E80FDF8C08091C40C80FDFDC0F3C071
:10D0900081E00E94935FEFC095FFC9C08091550762
:10D0A000909156072091901021FD2EC048EE53E03C
:10D0B00060E070E00F94BD44803921E0920744F4B1
:10D0C0002091F9063091FA06DC01A059B1400BC05D
:10D0D000893542E094078CF02091F9063091FA06E8
:10D0E000DC01A855B2400F94A69920E931E040E058
:10D0F00050E00F94329A790102C0E12CF12CF092A9
:10D100004E12E0924D1202C0E12CF12C80911E0EC5
:10D1100081FF3BC01E141F0494F580E00E946E60E6
:10D12000609101117091021180910311909104118D
:10D130006C5E7F4F8F4F9F4F0F94A2966093E712C4
:10D140007093E8128093E9129093EA1220E030E0A5
:10D15000A9016091FE087091FF08809100099091EB
:10D1600001090F94009687FF04C080EF98E00E94A9
:10D170003BC361E089EA9CE00F94C55B06C060E0B8
:10D1800080E090E057DA1092E61280911E0E81FD49
:10D19000B4C0C7010E94D446B0C095FF48C080917A
:10D1A0001E0E81FF05C061E089EA9CE00F94C55B1B
:10D1B0006091360E7091370E8091380E9091390E35
:10D1C0000F946F969B01AC0180913A0E90913B0EAB
:10D1D000A0913C0EB0913D0EBC01CD019058298329
:10D1E0003A834B835C830F946F966B017C01609153
:10D1F000780E7091790E80917A0E90917B0E0F943B
:10D200006F9629813A81A6010E949E478091780EEF
:10D210009091790EA0917A0EB0917B0E809343127B
:10D2200090934412A0934512B093461266C060E0FA
:10D2300080E090E0FFD91092E6121DC080910111AC
:10D2400090910211A0910311B09104113091F70651
:10D250002091F806883E9340A105B10574F51CC0E5
:10D260008091550790915607892B19F08091901065
:10D2700081FD0E94A75F10924312109244121092F7
:10D2800045121092461239C080910207909103070F
:10D290008E159F0584F7FCCE832F922F97FF03C036
:10D2A0009195819591099195819591090E94D44616
:10D2B00080911E0E81FDD4CFDECFE32EF22EF7FE3D
:10D2C00003C0F194E194F108F194E194F1088091A4
:10D2D0003A0E90913B0EA0913C0EB0913D0EBC01D8
:10D2E000CD0190580F946F969701AB0168EE73E0F3
:10D2F00080E090E00E949E47BECF0F900F900F906D
:10D300000F90DF91CF91FF90EF90DF90CF90089535
:10D310006091860C7091870C8091880C9091890C9B
:10D320000F946F9660930111709302118093031113
:10D330009093041160916E0C70916F0C8091700C41
:10D340009091710C0F946F9670933C1260933B1206
:10D350004FDE80913B1290913C1243968797E8F400
:10D360008091C30C82FF19C080911E0E81FD20C0E8
:10D3700080917412909175128233910530F4019668
:10D38000909375128093741213C081E00E946E60B6
:10D3900010927512109274120BC0109275121092A6
:10D3A000741280911E0E81FF03C080E00E946E60A7
:10D3B00090911D0E8091C40C95FF17C080FF1EC078
:10D3C000E0916D10EE30F8F4F0E0E35BFD4F80810A
:10D3D0008823C9F08091550790915607892B99F4BD
:10D3E0008091901081FF0AC0089580FF0CC0809149
:10D3F000550790915607892B19F4089580E001C0D4
:10D4000081E00C945F5F0895FC01148A138A28EE72
:10D4100033E037A726A731AB20AB65E87EE00D945B
:10D42000C96E0F931F93CF93DF938C01CB016930AB
:10D43000710508F03FC09B0120583F4FF9010D9442
:10D440006E9BF80162A91AC0F80164A917C0F8011F
:10D4500066A914C0F80160AD11C0F80162AD0EC03C
:10D46000F80164AD0BC0F80166AD08C0D801A05C3E
:10D47000BF4F03C0D801AE5BBF4F6C916623D1F0A4
:10D48000800F911FEC01CC5BDF4F8881811110C0B0
:10D49000633308F062E382E390E070E00F94FD995B
:10D4A000F801E35BFF4F8081860F888381E003C032
:10D4B0008150888380E0DF91CF911F910F91089573
:10D4C000A4E0B0E0E6E6FAE60D94439B8C01FC0193
:10D4D00087859089892BC1F460E070E0EE24E394A5
:10D4E000F12CEC0EFD1EC7010F94A26FF8012785E9
:10D4F00030892F5F3F4F308B278760E070E0C70196
:10D500000F944E71892B91F7F801878590892496A5
:10D51000E6E00D945F9B4F925F926F927F928F92A5
:10D520009F92AF92BF92CF92DF92EF92FF920F93B2
:10D53000CF93DF93CDB7DEB760970FB6F894DEBF19
:10D540000FBECDBF5C01FC01E380F480E114F10467
:10D55000B9F165817681C7010F9490712B013C016F
:10D560004501F7E08F0E911C01E020E130E0AE01B3
:10D570004F5F5F4FB401C7010F948D6CF501C384F9
:10D58000D484E584F684858196810F94C489082F1C
:10D59000A3019201BE016F5F7F4FF50181899289DE
:10D5A0000E943B55B5016B5F7F4FC4010F944E71D4
:10D5B000F50194838383838594850196948783877B
:10D5C00060960FB6F894DEBF0FBECDBFDF91CF914E
:10D5D0000F91FF90EF90DF90CF90BF90AF909F9012
:10D5E0008F907F906F905F904F9008950F93CF939F
:10D5F000DF9300D01F92CDB7DEB7FC01878D882363
:10D60000B9F026893789808D918D8217930780F034
:10D61000448D528D818992893A8329835B834C831F
:10D6200006EE24E0AE014F5F5F4F68E20F94EC8995
:10D630000F900F900F900F90DF91CF910F91089561
:10D64000CF93DF93EC010E94AA2AC25BDF4F68836D
:10D6500079838A839B83DF91CF910895FC01728344
:10D66000618381E080838091B7139091B81368172C
:10D67000790739F47093FD146093FC14128A118AAF
:10D6800008C07093FB146093FA1481E090E0928BD1
:10D69000818B14821382CF01D3CF81E08093140257
:10D6A0000E94B62A6093171370931813809319136E
:10D6B00090931A13089580911D0E87FD17C08068FE
:10D6C00080931D0E109298058091BB099091BC0922
:10D6D000A091BD09B091BE09B7FD02C081E001C0B3
:10D6E0008FEF80931E1385E10C94BD420895CF9275
:10D6F000DF92EF92FF92C0901E13DD24C7FCD094FE
:10D70000ED2CFD2C6091BB097091BC098091BD0985
:10D710009091BE09A70196010F94CE99209198058A
:10D72000213059F120F0223009F079C055C0643918
:10D73000714181059105ECF4A0E4BCE9A7019601D3
:10D740000F94BE996093B4127093B5128093B61281
:10D750009093B71280912E020E94B45E882309F440
:10D760005EC0809155079091560760E086559F4FA7
:10D770002AC081E08093980552C0DC01CB01885D0E
:10D780009C4DAF4FBF4F8C3B9443A105B105F0F0CA
:10D79000A0E4BCE9A70196010F94BE996093B4126E
:10D7A0007093B5128093B6129093B71280912E02A7
:10D7B0000E94B45E882399F1809155079091560795
:10D7C00060E0885791090E941A6329C082E0809323
:10D7D00098051092990523C0809199058436A8F484
:10D7E00080912E020E94B45E882349F080915507F3
:10D7F0009091560760E086559F4F0E941A63809172
:10D8000099058F5F809399050AC086E10E94BD4209
:10D8100080911D0E8F7780931D0E10929805FF90BA
:10D82000EF90DF90CF900895109297051092960593
:10D8300010929205109293051092940510929505FE
:10D8400010929105109290050895A3E1B0E0EBE2EB
:10D85000FCE60D94459B80910D0783FF4EC08E0121
:10D860000F5F1F4F83E1D8011D928A95E9F783EA84
:10D87000898385E98A8386E08B838091C7098C83BD
:10D880008091C8098D8380919005909191059F8327
:10D890008E838091960590919705998788878091CE
:10D8A000920590919305A0919405B09195058A8772
:10D8B0009B87AC87BD878091AB099091AC099F870E
:10D8C0008E878091BD139091BE13DC01ED91FC9188
:10D8D0000488F589E02D1995888B80917B0B9091B8
:10D8E0007C0B9A8B898B80918C0C8B8B43E150E065
:10D8F000B8018DE89CE00F94BB7C80919609882349
:10D9000071F1E0918606F0918706A081B181809146
:10D9100095058F93809194058F93809193058F93B4
:10D92000809192058F93809197058F9380919605B2
:10D930008F93809191058F93809190058F938FE0C5
:10D9400090E19F938F93FF93EF935096ED91FC910D
:10D95000519719950FB6F894DEBF0FBECDBF64DFA7
:10D960001092AC091092AB096396E4E00D94619BB0
:10D970000F931F9320919605309197052F5F3F4F8E
:10D980003093970520939605009192051091930589
:10D990002091940530919505061717072807390738
:10D9A00040F460939205709393058093940590934F
:10D9B0009505653079428105910548F08091900583
:10D9C00090919105019690939105809390051F91F8
:10D9D0000F910895AFE0B0E0E0EFFCE60D94399BC5
:10D9E0004C01BC82CD82DE82EF82F88609871A87DD
:10D9F0002B873C874D875E876F876C817D818E8109
:10DA00009F810F94A2966B017C016C857D858E852C
:10DA10009F850091771110917811209179113091A3
:10DA20007A11601B710B820B930B0F94A2962CE260
:10DA30003DE74EE85FE30F94CD9820910C023091C2
:10DA40000D0240910E0250910F020F94CD985B0190
:10DA50008C01688579858A859B85409073115090EB
:10DA600074116090751170907611641975098609AA
:10DA700097090F94A2962CE23DE74EE85FE30F94DE
:10DA8000CD98F40160837183828393838A2D9B2DCB
:10DA9000A02FB12F84839583A683B783C086D186B8
:10DAA000E286F386C4012F96E0E10D94559BA0E039
:10DAB000B0E0EDE5FDE60D94419B8C01EB01FC012E
:10DAC00024813581468157816C817D818E819F8142
:10DAD0000F9422956B017C01F801208131814281F4
:10DAE0005381688179818A819B810F942295905816
:10DAF000A70196010F94AD9520EA3CE043EB55E475
:10DB00000F94CD9820E030EA4CE056E40F94239532
:10DB10008B01D82FC92F20E030E0A901FE01712F21
:10DB20008F2F9E2F0F94009687FF0EC020E030EAC3
:10DB30004CE057E4FE01602F712F8F2F9E2F0F9422
:10DB400023958B01D82FC92F9E01602F712F832F12
:10DB50009C2FCDB7DEB7E8E00D945D9BCF93C82F27
:10DB600080919212C81709F45FC0EC2FF0E0EA3000
:10DB7000F10508F055C0E757FF4F0D946E9B1092CA
:10DB800093121092941210929512109296124AC00B
:10DB900080911D0E80FF44C06BE771E18EE79CE031
:10DBA00086DF0F946F96609397127093981280930C
:10DBB000991290939A1236C080911D0E80FF30C04A
:10DBC0008CE0E9ECF5E0ABE7B1E101900D928A95CC
:10DBD000E1F74091C3095091C4096091C509709162
:10DBE000C6094093971250939812609399127093BC
:10DBF0009A1218C080911D0E80FD14C011C0409172
:10DC0000C3095091C4096091C5097091C609409338
:10DC1000750D5093760D6093770D7093780D02C05B
:10DC200080E003C0C093921281E0CF910895A8E1F3
:10DC3000B0E0EDE1FEE60D94479B8CE0EEE7FCE002
:10DC4000DE011D9601900D928A95E1F780911A11DF
:10DC5000982F9150923098F481E29EE00E94C4C8BF
:10DC60000F94749660931B1170931C1180931D1177
:10DC700090931E1181E29EE00E941CD214C083305A
:10DC8000D9F481E29EE00E94AFCD0F947496609328
:10DC90001B1170931C1180931D1190931E1181E232
:10DCA0009EE00E9411D260930D1170930E1180932B
:10DCB0000F119093101110C010921B1110921C1193
:10DCC00010921D1110921E1110920D1110920E1132
:10DCD00010920F11109210110E94342C882399F188
:10DCE00029893A894B895C896D857E858F859889DC
:10DCF0000F94EC440F946F966093CF107093D010F4
:10DD00008093D1109093D21019821A821B821C82A8
:10DD10001D821E821F82188619861A861B861C8603
:10DD2000BE016F5F7F4FCE010D96C1DE0F946F96DF
:10DD30006093551170935611809357119093581119
:10DD400080E00E949D5E6896E2E00D94639BA9E0EE
:10DD5000B0E0EDEAFEE60D94379BC0907207D090DC
:10DD600073078091901081FF02C0C12CD12CE091EB
:10DD70009212F0E0EA30F10508F008C4ED56FF4FCA
:10DD80000D946E9B80911E0E81FF10C08091C3097F
:10DD90009091C409A091C509B091C6098093750DF1
:10DDA0009093760DA093770DB093780DB6018827E8
:10DDB00077FD8095982F0E947254E8C3B60188279A
:10DDC00077FD8095982F0F94A29620914708309167
:10DDD00048084091490850914A080F94CD980F94F3
:10DDE0006F962B013C0180915308823069F480903A
:10DDF000931290909412A0909512B0909612840C69
:10DE0000951CA61CB71C53C060919312709194127C
:10DE100080919512909196120F94A2962091A4123F
:10DE20003091A5124091A6125091A7120F94CD984F
:10DE30000F946F966093931270939412809395123F
:10DE4000909396129301820177FE07C00027112755
:10DE5000980104191509260937094B015C0197FF40
:10DE600007C0882499245401861A970AA80AB90A77
:10DE700078018901E818F9080A091B0917FF08C089
:10DE800010950095F094E094E11CF11C011D111D0A
:10DE9000640D751D861D971D22273327A9012E1994
:10DEA0003F09400B510B0F94C7444B015C0160913B
:10DEB000A8127091A9128091AA129091AB120F949E
:10DEC0006F96AB01BC0186E799E00E94F8D721E08C
:10DED00020939B12680D791D8A1D9B1D60939C12D7
:10DEE00070939D1280939E1290939F12C501B4016E
:10DEF0000F94A2966B017C0120EA3CE043EB55E4D1
:10DF000060913212709133128091341290913512D7
:10DF10000F94CD989B01AC01C701B6010F942295D7
:10DF200020911E0230911F02409120025091210247
:10DF30000F94CD982091A8123091A9124091AA1265
:10DF40005091AB120F942395FB01462F5F2F682F42
:10DF5000792F4093A8125093A9126093AA1270933C
:10DF6000AB12E12CF12C0AE714E420E030E04AE7A0
:10DF700054EC6F01BF010F9465446093A812709335
:10DF8000A9128093AA129093AB128091C40C80FFC7
:10DF9000F5C28091570790915807892B09F4EEC27A
:10DFA000F5C280911E0E81FDCFC2209111113091DA
:10DFB000121140911311509114116091750D7091CF
:10DFC000760D8091770D9091780D0CE310E00E9412
:10DFD000D43F6093750D7093760D8093770D909379
:10DFE000780D6091750D7091760D8091770D9091FF
:10DFF000780D0E94B053C114D10409F4C7C280E067
:10E00000ADDDC4C280911E0E81FF10C08091C30996
:10E010009091C409A091C509B091C6098093750D6E
:10E020009093760DA093770DB093780D8091AC12FC
:10E030008F5F8A3018F48093AC1211C01092AC122A
:10E040006BE771E18EE79CE032DD0F946F96609391
:10E050009712709398128093991290939A1220912C
:10E060009712309198124091991250919A126091A2
:10E07000750D7091760D8091770D9091780D0CE370
:10E0800010E00E94D43F6093750D7093760D8093DD
:10E09000770D9093780DADCF80911E0E81FF10C04B
:10E0A0008091C3099091C409A091C509B091C60996
:10E0B0008093750D9093760DA093770DB093780DA6
:10E0C0008091ED069091EE06892BA9F460913311B1
:10E0D0007091341180913511909136110F94E6446E
:10E0E00020E030E048EC52E40F94CD980F946F9606
:10E0F0009B01AC0162CF8091AD128F5F8A3018F422
:10E100008093AD1211C01092AD126BE771E18EE7F2
:10E110009CE0CDDC0F946F966093971270939812E9
:10E120008093991290939A1220919712309198129D
:10E130004091991250919A1240CF80911E0E81FD0C
:10E1400003C22091551130915611409157115091B1
:10E15000581133CF80911E0E81FF11C08091C309E9
:10E160009091C409A091C509B091C6098093750D1D
:10E170009093760DA093770DB093780D1EC000910B
:10E1800093111091941120918F1130919011409121
:10E190009111509192116091750D7091760D809151
:10E1A000770D9091780D0E94D43F6093750D709318
:10E1B000760D8093770D9093780D6091750D709129
:10E1C000760D8091770D9091780D86C080911E0E0E
:10E1D00081FF10C08091C3099091C409A091C50925
:10E1E000B091C6098093750D9093760DA093770D2D
:10E1F000B093780DE0916E10F0916F1084A195A10D
:10E20000EE24D7FCE094FE2C892B41F1848995897A
:10E21000A689B78985369105A105B105F8F0208D4D
:10E22000318D428D538D6091750D7091760D809179
:10E23000770D9091780D0CE310E00E94D43F60932D
:10E24000750D7093760D8093770D9093780D6C0D0E
:10E250007D1D8E1D9F1D0F944E463EC06091750D15
:10E260007091760D8091770D9091780D0F94A29614
:10E270004B015C01C701B6010F94A296209147089B
:10E28000309148084091490850914A080F94CD9820
:10E2900020911E0230911F024091200250912102D4
:10E2A0000F94CD989B01AC01C501B4010F94239547
:10E2B0000F946F966093750D7093760D8093770D24
:10E2C0009093780D0F944E466093750D7093760D74
:10E2D0008093770D9093780D0E94B05357C1809131
:10E2E0001E0E81FF10C08091C3099091C409A091B6
:10E2F000C509B091C6098093750D9093760DA093D2
:10E30000770DB093780D609138077091390780913F
:10E310001B0790911C070E94E44E8091660C90911F
:10E32000670CA091680CB091690C89839A83AB83C8
:10E33000BC8340906A0C50906B0C60906C0C709099
:10E340006D0C8090070290900802A0900902B09096
:10E350000A02C0902F11D0903011E0903111F0904E
:10E360003211A5019401C301B2010F94CD986D83C0
:10E370007E838F839887A701960169817A818B813B
:10E380009C810F94CD989B01AC016D817E818F8122
:10E3900098850F9422956D837987382E292EA701B1
:10E3A0009601C301B2010F94CD986B017C01A501C8
:10E3B000940169817A818B819C810F94CD989B0116
:10E3C000AC01C701B6010F942395462F572F682F34
:10E3D000792F4A015B0175016401E894F7F820E0A8
:10E3E00030E048E454E4C701B6010F94009687FD7D
:10E3F00006C0C12CD12CA8E4EA2EA4E4FA2E809108
:10E40000710D9091720D97FD0196BC017595679500
:10E41000882777FD8095982F0F94A2962B013C01B9
:10E4200020E030E046E155E4C701B6010F940796BD
:10E430009B01AC0160E070E080E89FE30F942295BF
:10E440009B01AC01C301B2010F94CD980F946F965C
:10E450000E947254E12CF12C01EA13E420E030E038
:10E4600041EA53ECFD81E985D1016F2F7E2F8B2F7F
:10E47000922D0F9465442B013C0120E030E041EAED
:10E4800053ECC501B4010F9465444B015C0120E0DD
:10E4900030E040E651ECC301B2010F94CD980F94E7
:10E4A0006F960E946C536091730D7091740D61159D
:10E4B0007105B9F52FE832EC45EF5CE36091AE12DF
:10E4C0007091AF128091B0129091B1120F94239578
:10E4D0008B017C0120E030E040E651E4712F9F2D5C
:10E4E0000F94009687FD06C000E010E050E6E52E90
:10E4F00061E4F62E402F512F6E2D7F2D4093AE12EA
:10E500005093AF126093B0127093B112202F312F3D
:10E510004E2D5F2DC501B4010F94CD980F946F96C9
:10E520000CC01092AE121092AF121092B012109254
:10E53000B112882777FD8095982F0E942E5426C00F
:10E5400080911E0E81FF11C08091C3099091C40972
:10E55000A091C509B091C6098093750D9093760D71
:10E56000A093770DB093780D3CCD2091521230914D
:10E57000531240915412509155121FCD1092A8126F
:10E580001092A9121092AA121092AB122996E2E1EF
:10E590000D94539B89EA9CE00F941A5D89EA9CE0F4
:10E5A0000D94485DAF92BF92CF92DF92EF92FF92AF
:10E5B0000F931F93A12CB12CC12CD12CE12CF12C49
:10E5C00000E010E023E238E045E058E067EE77E055
:10E5D00089EC97E00F945B8A1F910F91FF90EF9069
:10E5E000DF90CF90BF90AF90089580919409909163
:10E5F0009509DC01ED91FC910484F585E02D1995D8
:10E6000020E030E04AE754E40F94CD980F947496DC
:10E61000CB010895A3E0B0E0E0E1F3E70D94439B64
:10E620007C018091BD139091BE13DC01ED91FC91B2
:10E630000488F589E02D1995182FD7DF9A838983EF
:10E640001B8305E123E0AE014F5F5F4F65EAC70121
:10E650000F94EC892396E6E00D945F9B8F929F9236
:10E66000AF92BF92EF92FF920F931F93CF93DF93DE
:10E67000EC017B01009721F081309105A9F405C0E0
:10E68000A091FC14B091FD1404C0A091FA14B091B3
:10E69000FB14ED91FC9111970680F781E02DCD01DF
:10E6A00019958C0197FF02C000E010E00E94AA2A91
:10E6B0002AE096958795779567952A95D1F780906A
:10E6C000C706992487FC9094A92CB92C8616970626
:10E6D000A806B90640F486E999E00F9477768A3F58
:10E6E000910538F0C7C0CE010E94AA42882399F351
:10E6F000BFC08091C40C80FDB8C0BCC009301105FA
:10E700000CF4B6C0CE010E94C54FADC00F3111054B
:10E710000CF4AEC0CE010E940F50A5C0043011050C
:10E720000CF4A6C0CE010E94D5399DC00C31110554
:10E730000CF49EC0CE010E94FC3995C00C3111052D
:10E740000CF496C0CE010E949D3A8DC00A3111058D
:10E750000CF48EC0CE010E94145185C00E311105FB
:10E760000CF486C0CE010E94A9517DC00C30110569
:10E770000CF47EC0CE010E94E93E75C00631110541
:10E780000CF476C0CE010E9446526DC005311105D1
:10E790000CF46EC0CE010E94985265C00431110580
:10E7A0000CF466C0CE010E94733B5DC00A311105B6
:10E7B0000CF45EC0CE010E94033C55C00E30110522
:10E7C0000CF456C0CE010E94D33C4DC00A32110554
:10E7D0000CF44EC0CE010E942F3D45C00230110501
:10E7E0000CF446C0CE010E941F553DC009311105F1
:10E7F0000CF43EC0CD2B19F489E79DE006C0809152
:10E80000CB0D882381F18BEC9DE00E948B6A2BC09D
:10E81000043011056CF1CD2B19F489E79DE006C099
:10E820008091CB0D8823F9F08BEC9DE00E94F66A75
:10E830001AC003331105E4F0CE010E94B73E13C0A5
:10E8400006311105ACF0CE010E942C3E0CC00C31FB
:10E85000110574F0CE010E94E55205C00330110588
:10E860003CF0CE01D7DE81E010C081E08093291218
:10E8700080E00BC00850110987E1E816F10498F711
:10E88000F701E356FF4F0D946E9BDF91CF911F91DF
:10E890000F91FF90EF90BF90AF909F908F90089551
:10E8A000EF92FF920F931F93CF93DF93F82EE92EF1
:10E8B0008B0180E3F89EE0011124C753DE4E1BC09C
:10E8C0008EA5FE01E80FF11DE80FF11D6081718139
:10E8D0008F2D9E2DC3DE811104C00731110579F4FF
:10E8E0003EC02EA52F5F273111F02EA701C01EA616
:10E8F0008FA581508FA78FA58111E2CFEECF4EA5B6
:10E900008FA550E00FC0FE01E40FF11DE40FF11DD3
:10E91000208131812017310711F14F5F473109F410
:10E9200040E05F5F5813EFCF511116C0B8018F2D33
:10E930009E2D94DE811113C00FC08EA5890F8731E3
:10E9400008F08751FE01E80FF11DE80FF11D11835A
:10E9500000839F5F9FA703C09FA5973171F7CDB735
:10E96000DEB7E6E00D945F9BA0E0B0E0EAEBF4E7F1
:10E970000D94459BFE0138962191319181E0809361
:10E9800096118F0142E350E067E971E18091CF1366
:10E990009091D0130F94FE0C62E170E080E090E063
:10E9A0007FDF8091CB0D882329F062E170E081E068
:10E9B00090E076DFE4E00D94619BFC01818992890F
:10E9C0006FCFCF93DF93EC01BC0189E79DE0F5DFCA
:10E9D0008091CB0D882321F0BE018BEC9DE0EDDF13
:10E9E000DF91CF91089587E190E0EBCF80E090E058
:10E9F000E8CFCF93DF93EC018F8D8111C4C08E8D52
:10EA00008111C1C0109229128B819C81892BB9F090
:10EA1000FE01EE5BFF4F808191811816190624F0EC
:10EA200082E390E09183808368E070E0CE010E94F1
:10EA3000116A882309F4A7C061E170E0A2C0809147
:10EA400076128111A0C060E070E0CE010E94116AD0
:10EA5000882361F06AE070E0CE01AFDF6BE070E028
:10EA6000CE01ABDF6CE070E0CE01A7DF8091291210
:10EA7000811189C061E070E0CE010E94116A882393
:10EA8000C1F063E070E0CE0198DF64E070E0CE0199
:10EA900094DF66E070E0CE0190DF6DE070E0CE01C3
:10EAA0008CDF65E070E0CE0188DF63E170E0CE01CD
:10EAB00084DF80912912811166C064E070E0CE018C
:10EAC0000E94116A882321F062E070E0CE0175DFB8
:10EAD00080912912811157C063E070E0CE010E943D
:10EAE000116A882321F06FE070E0CE0166DF80912B
:10EAF0002912811148C062E070E0CE010E94116AC3
:10EB0000882341F068E070E0CE0157DF69E070E0F3
:10EB1000CE0153DF80912912811135C065E070E08C
:10EB2000CE010E94116A882341F061E070E0CE01BD
:10EB300044DF65E170E0CE0140DF80912912811150
:10EB400022C066E070E0CE010E94116A882321F0A5
:10EB500067E070E0CE0131DF80912912811113C08E
:10EB600067E070E0CE010E94116A882361F064E1E1
:10EB700070E0CE0122DF66E170E0CE011EDF6EE0C4
:10EB800070E0CE011ADFDF91CF91089589E79DE013
:10EB900030DF8091CB0D882319F08BEC9DE029CFDD
:10EBA00008958F929F92AF92BF92EF92FF920F9330
:10EBB0001F93CF93DF93EC018B017A010E94AA2A65
:10EBC0003AE096958795779567953A95D1F7809035
:10EBD000C706992487FC9094A92CB92C8616970611
:10EBE000A806B90620F401301105B1F406C0CE0123
:10EBF0000E94AA42811115C0F6CF81E08093961140
:10EC000042E350E0B70187E991E10F94D19D62E1C1
:10EC100070E0CE0145DE05C0A701602FCE010E9445
:10EC2000863EDF91CF911F910F91FF90EF90BF90A3
:10EC3000AF909F908F900895A3E3B0E0E2E2F6E7F3
:10EC40000D94479BDE01129620E030E0FA01E20FBE
:10EC5000F31FE491ED93EE2369F02F5F3F4F2233D2
:10EC60003105A1F7AE014E5F5F4FFC0181899289AA
:10EC700098DF05C0FE01E20FF31F1282F3CFE39687
:10EC8000E2E00D94639B0F931F93CF93DF93EC010E
:10EC90008B01AB01BC0189E79DE0CEDF8091CB0DFC
:10ECA000882329F0A801BE018BEC9DE0C5DFDF9130
:10ECB000CF911F910F91089564EB7BE181E090E08B
:10ECC000E2DF86E09FE00E9479EB6AEC7BE181E085
:10ECD00090E0D9CFA0E0B0E0E0E7F6E70D943B9BF1
:10ECE0000E94BD2CE9DFC0E8DAE264E670E080E073
:10ECF00090E00E949D2A86E09FE00E9431F286E02B
:10ED00009FE00E9452ED6B017C012091080F8091E1
:10ED1000860690918706DC01ED91FC91211107C0D8
:10ED20000484F585E02D64E77AE219953EC00089F8
:10ED3000118986E09FE00E9424F0962E872E782E7F
:10ED4000692E86E09FE00E9418F0B0908606A090A1
:10ED500087066F927F928F929F929F938F937F935C
:10ED60006F9320E030E048EC52E4C701B6010F9405
:10ED7000CD980F946F960F94A29620E030E048EC67
:10ED800052E40F9407969F938F937F936F93DF9333
:10ED9000CF93AF92BF92F80119958DB79EB7409669
:10EDA0000FB6F8949EBF0FBE8DBFA0918606B0919E
:10EDB0008706ED91FC9111970480F581E02DCD013E
:10EDC0001995181619060CF090CF80E0CDB7DEB774
:10EDD000EEE00D94579B62E97DE181E090E053DF26
:10EDE0008DE89CE00F94377C60EA7DE181E090E063
:10EDF0004ACF81E080937612EEDF1092761280E0A7
:10EE000008958091C40C80FF86C080915507909131
:10EE10005607892B09F482C08091901081FF7BC036
:10EE20007DC080911D0E87FD76C04091E506509112
:10EE3000E6064053584F662757FD6095762F809120
:10EE4000BB099091BC09A091BD09B091BE09B7FF63
:10EE500007C0B095A095909581959F4FAF4FBF4F3C
:10EE6000481759076A077B07BCF08091BF0990914A
:10EE7000C009A091C109B091C209B7FF07C0B09500
:10EE8000A095909581959F4FAF4FBF4F4817590759
:10EE90006A077B070CF03FC0209112132F5F20936D
:10EEA000121380913D1290913E12A0913F12B091A9
:10EEB0004012213049F48093131390931413A093BC
:10EEC0001513B09316130895409113135091141312
:10EED0006091151370911613841B950BA60BB70B3D
:10EEE000B7FF07C0B095A095909581959F4FAF4F04
:10EEF000BF4FC397A105B1050CF00DC02431A0F0A0
:10EF000061E08CE00E941D2E64EF7EE183E090E0E2
:10EF1000BADE0C94A75F10921213089580916D10C1
:10EF2000813009F07ECFF7CF0895CF92DF92EF9234
:10EF3000FF92CF93C82F86E69CE00F9418536B0185
:10EF40007C010E94342C882361F1E0916E10F091D5
:10EF50006F1040A151A12091DB063091DC062417EF
:10EF60003507FCF08091721081FD1BC020E030E07D
:10EF7000A901C701B6010F940096882391F020E003
:10EF800030E048E452E4C701B6010F947D981816AA
:10EF900044F081E009C068E871E183E090E073DE4D
:10EFA00002C0C111F8CF80E0CF91FF90EF90DF90C9
:10EFB000CF9008956BE47BE181E090E064DE8DEA20
:10EFC00099E00E94D85541E050E060E070E08BE1AC
:10EFD0009BE00F945E380E94D033EEEDF9E0808123
:10EFE0008260808381E00C946E6080911807882392
:10EFF000A9F18130A9F183FD33C00EC0F0E0EC5BD4
:10F00000FD4F8081811104C08091D906833021F4A5
:10F0100081E08BDF8823A9F180911807813031F1DD
:10F0200085FD24C00BC02091530730915407809177
:10F0300000079091010728173907ECF08091CF1352
:10F040009091D013DC01ED91FC910280F381E02DD1
:10F050001995019719F46BEF7BE10FC081E00895DA
:10F06000E0916D10E350E93048F2CECF8091FF0679
:10F070008111D9CFE3CF69EE7BE183E090E003DE3D
:10F0800080E00895813039F018F0823061F406C0D4
:10F0900064E57EE105C061E37EE102C063E47EE1F8
:10F0A00083E090E0F0CD08954F925F926F927F924F
:10F0B0008F929F92AF92BF92CF92DF92EF92FF9288
:10F0C0000F931F93CF93C82F80916812C81709F42C
:10F0D00026C1C53050F4C23008F01BC1CC2309F45E
:10F0E00018C1C13009F02BC108C0C63009F411C1E4
:10F0F000A8F0C73009F023C116C01092C5121092B3
:10F10000C6121092C7121092C8121092C912109211
:10F11000CA121092CB121092CC12FBC080911D0E1D
:10F1200080FDF7C00CC181110AC18091C40C80FF21
:10F1300006C180911E0E81FFF4C001C180919A0525
:10F14000877880939A050E94AA2A6093CD127093C3
:10F15000CE128093CF129093D01280919A058F7720
:10F1600080939A0580919B058E7F80939B0580916B
:10F17000540890915508A0915608B0915708809373
:10F18000971090939810A0939910B0939A10409173
:10F1900058085091590860915A0870915B08409343
:10F1A0009B1050939C1060939D1070939E10409004
:10F1B0005C0850905D0860905E0870905F08409217
:10F1C0009F105092A0106092A1107092A210809097
:10F1D0005A0990905B09A0905C09B0905D098092FB
:10F1E000A3109092A410A092A510B092A610C09067
:10F1F0006E08D0906F08E0907008F0907108C0928F
:10F20000A710D092A810E092A910F092AA104091F5
:10F21000720850917308609174087091750840935A
:10F22000AB105093AC106093AD107093AE10009182
:10F23000760810917708209178083091790800932A
:10F24000AF101093B0102093B1103093B2104091D2
:10F2500068095091690960916A0970916B0940933E
:10F26000B3105093B4106093B5107093B6108093A0
:10F27000B7109093B810A093B910B093BA10409201
:10F28000BF105092C0106092C1107092C210809254
:10F29000C3109092C410A092C510B092C610C09234
:10F2A000BB10D092BC10E092BD10F092BE10009343
:10F2B000C7101093C8102093C9103093CA10409300
:10F2C000CB105093CC106093CD107093CE108EE184
:10F2D0000E94BD4264E57EE183E090E0D4DC809151
:10F2E0009A058C7F816080939A0513C00E94C02884
:10F2F00080E20E94BD4264E57EE183E090E0C3DCF1
:10F3000008C00E94C82984E201C082E20E94BD4276
:10F3100016C0809168120E949C5DC093681281E0C3
:10F320000FC080919A05837090E08230910549F377
:10F330008330910551F3019709F000CFD7CF80E0DA
:10F34000CF911F910F91FF90EF90DF90CF90BF90E2
:10F35000AF909F908F907F906F905F904F900895A7
:10F36000ACE0B0E0E6EBF9E70D943B9B3C01009785
:10F3700009F469C0FC0187819085A185B285892B3C
:10F380008A2B8B2B49F483859485A585B685892B9B
:10F390008A2B8B2B09F457C01092FD1082E084DE7B
:10F3A00080E00E948B5D0E94AE6D83E00E948560CC
:10F3B00083E00E941631F30180809180A280B380A7
:10F3C000C480D580E680F78000851185228533854D
:10F3D000448555856685CE0101960E94EA6C609150
:10F3E0000111709102118091031190910411613407
:10F3F000FFE17F078105910524F060E47FE180E073
:10F4000090E00F94A29669877A878B879C87BE01CC
:10F410006F5F7F4F81E29EE00E94ACD781E29EE069
:10F420000E9411D260930D1170930E1180930F11F1
:10F430009093101160931111709312118093131116
:10F440009093141116C081E08093FD100E94342C1B
:10F45000882321F085E028DE82E003C080E024DEFE
:10F4600080E00E94163180E00E94AE6D84E00E9430
:10F4700085602C96EEE00D94579BA1E2B0E0E3E4AA
:10F48000FAE70D94399B80916812833009F4ADC37B
:10F4900028F4813071F008F06AC3A7C3863009F4FC
:10F4A00022C4873009F40CC6853011F00C9488888A
:10F4B000BBC330911B0720911C073093710D209323
:10F4C000720D90913807809139079093730D809356
:10F4D000740D692F782F77FF03C0719561957109BD
:10F4E000809172079091730797FF03C09195819562
:10F4F0009109681779070CF4BC01832F922F97FFAD
:10F5000003C0919581959109681779070CF4BC01A6
:10F51000882777FD8095982F0F94A29620E030EAF7
:10F520004CE855E40F9407969B01AC0160E070E055
:10F5300080E89FE30F942295E12CF12C00E81FE373
:10F5400020E030E0A9010F9465442091220230911F
:10F55000230240912402509125020F94CD985B0123
:10F560008C01982F4A2D5B2D692F712F4093A41287
:10F570005093A5126093A6127093A71260911B0777
:10F5800070911C07882777FD8095982F0F94A2967D
:10F590002091430830914408409145085091460815
:10F5A0000F94CD980F946F962B013C0180915308D6
:10F5B000823069F48090C5129090C612A090C71254
:10F5C000B090C812840C951CA61CB71C51C0609149
:10F5D000C5127091C6128091C7129091C8120F94F3
:10F5E000A2962A2D3B2D402F512F0F94CD980F948A
:10F5F0006F966093C5127093C6128093C712909352
:10F60000C8127301620177FE07C0CC24DD247601A5
:10F61000C418D508E608F7088B019C0197FF07C0BE
:10F62000002711279801061B170B280B390B4601E1
:10F630005701801A910AA20AB30A85017401B7FE24
:10F6400008C010950095F094E094E11CF11C011D98
:10F65000111D640D751D861D971D22273327A901D5
:10F660002E193F09400B510B0F94C7444B015C010D
:10F670006091D1127091D2128091D3129091D412D4
:10F680000F946F96AB01BC018AE599E00E94F8D710
:10F6900021E020939B12680D791D8A1D9B1D6093AC
:10F6A000B4127093B5128093B6129093B712C5013D
:10F6B000B4010F94A2966B017C0120EA3CE043EB7D
:10F6C00055E460912A1270912B1280912C12909126
:10F6D0002D120F94CD989B01AC01C701B6010F9478
:10F6E000229520911E0230911F02409120025091DC
:10F6F00021020F94CD982091D1123091D2124091D5
:10F70000D3125091D4120F942395FB01462F5F2FF3
:10F71000682F792F4093D1125093D2126093D31255
:10F720007093D412E12C10E8F12E0BE315E420E0E5
:10F7300030E84BE355ECBF010F9465446093D11260
:10F740007093D2128093D3129093D4128091C40CF0
:10F7500080FD02C00C949C888091570790915807B7
:10F76000892B11F40C949C886091380770913907AB
:10F77000882777FD8095982F0F94A29620914308B3
:10F780003091440840914508509146080F94CD9817
:10F790000F946F962B013C0180915308823069F4DD
:10F7A0008090C9129090CA12A090CB12B090CC1247
:10F7B000840C951CA61CB71C55C06091C912709191
:10F7C000CA128091CB129091CC120F94A2962091E4
:10F7D000A4123091A5124091A6125091A7120F9435
:10F7E000CD980F946F966093C9127093CA1280934C
:10F7F000CB129093CC127301620177FE07C0CC2428
:10F80000DD247601C418D508E608F7088B019C01B1
:10F8100097FF07C0002711279801061B170B280B1D
:10F82000390B46015701801A910AA20AB30A8501D1
:10F830007401B7FE08C010950095F094E094E11CA7
:10F84000F11C011D111D640D751D861D971D2227BC
:10F850003327A9012E193F09400B510B0F94C744C0
:10F860004B015C016091D5127091D6128091D71234
:10F870009091D8120F946F96AB01BC0188E699E085
:10F880000E94F8D721E020939B12680D791D8A1DF4
:10F890009B1D6093BC127093BD128093BE12909317
:10F8A000BF12C501B4010F94A2966B017C0120EA3E
:10F8B0003CE043EB55E460912E1270912F12809141
:10F8C0003012909131120F94CD989B01AC01C70179
:10F8D000B6010F94229520911E0230911F02409193
:10F8E0002002509121020F94CD982091D512309191
:10F8F000D6124091D7125091D8120F942395FB0144
:10F90000462F5F2F682F792F4093D5125093D61230
:10F910006093D7127093D812E12C10E8F12E0BE30C
:10F9200015E420E030E84BE355EC6F01BF010F9484
:10F9300065446093D5127093D6128093D71290933A
:10F94000D8128091C40C80FD02C00C94A6888091CE
:10F95000570790915807892B11F40C94A688809131
:10F960005308811114C082E080939B121092B81248
:10F970001092B9121092BA121092BB121092C012C9
:10F980001092C1121092C2121092C312E6C060917E
:10F99000BB097091BC098091BD099091BE090F947B
:10F9A0007E464B015C0180915308823049F52091DD
:10F9B000E5063091E606C901AA2797FDA095BA2F62
:10F9C00088159905AA05BB050CF40DC08827992751
:10F9D000821B930BAA2797FDA095BA2F881699062C
:10F9E000AA06BB066CF4AC01BD01481959096A09A5
:10F9F0007B098AE599E00E94F8D72B013C0103C0FE
:10FA0000412C512C320118EBE12E1BE0F12E00E0CD
:10FA100010E028E434EF4FEF5FEFC501B4010F941D
:10FA2000C7444B015C01C301B2010F94A2966B0164
:10FA30007C01C501B4010F94A29620914B0830912E
:10FA40004C0840914D0850914E080F94CD989B0161
:10FA5000AC01C701B6010F94229522E020939B12BE
:10FA60000F946F966093B8127093B9128093BA1284
:10FA70009093BB126091BF097091C0098091C10938
:10FA80009091C2090F947E464B015C01809153080E
:10FA9000823049F52091E5063091E606C901AA2792
:10FAA00097FDA095BA2F88159905AA05BB050CF4FA
:10FAB0000DC088279927821B930BAA2797FDA09535
:10FAC000BA2F88169906AA06BB066CF4AC01BD01D4
:10FAD000481959096A097B0988E699E00E94F8D714
:10FAE0002B013C0103C0412C512C320118EBE12EBB
:10FAF0001BE0F12E00E010E028E434EF4FEF5FEF61
:10FB0000C501B4010F94C7444B015C01C301B201AC
:10FB10000F94A2966B017C01C501B4010F94A296CB
:10FB200020914F083091500840915108509152084F
:10FB30000F94CD989B01AC01C701B6010F9422959B
:10FB400022E020939B120F946F966093C0127093E3
:10FB5000C1128093C2129093C3121092A0121092FD
:10FB6000A1121092A2121092A3120C948888609194
:10FB7000680E7091690E80916A0E90916B0E609381
:10FB80002711709328118093291190932A110091C5
:10FB90006C0E10916D0E20916E0E30916F0E0093D1
:10FBA0002B1110932C1120932D1130932E110E94A4
:10FBB0006C5360912B1170912C1180912D119091AB
:10FBC0002E110E942E5480911B0790911C07909338
:10FBD000720D8093710D8091380790913907909341
:10FBE000740D8093730D0C9488880E94AB5D6091B6
:10FBF00038077091390780911B0790911C070E946C
:10FC0000E44E6091710D7091720D882777FD80959B
:10FC1000982F0E946C536091730D7091740D88271A
:10FC200077FD8095982F5BC00E94AB5D00911B070C
:10FC300010911C071093720D0093710D609138079D
:10FC4000709139077093740D6093730D882777FD59
:10FC50008095982F0F94A2964B015C01B8018827DC
:10FC600077FD8095982F0F94A296AB01BC01EAE036
:10FC7000CE2EE7EDDE2EE3E2EE2EECE3FE2E950136
:10FC8000840181E29EE00E941CC56091680E709123
:10FC9000690E80916A0E90916B0E6093271170939C
:10FCA00028118093291190932A1100916C0E1091C4
:10FCB0006D0E20916E0E30916F0E00932B111093EC
:10FCC0002C1120932D1130932E110E946C536091B2
:10FCD0002B1170912C1180912D1190912E110E9459
:10FCE0002E540C9488880E94AB5D00911B071091E4
:10FCF0001C071093720D0093710D8091380790913D
:10FD000039079093740D8093730D6091D3107091A7
:10FD1000D4108091D5109091D6100F94A2966B01BB
:10FD20007C01B801882777FD8095982F0F94A296C3
:10FD3000209143083091440840914508509146086D
:10FD40000F94CD984B015C0120914B0830914C08E9
:10FD500040914D0850914E08C701B6010F94CD98BF
:10FD60009B01AC01C501B4010F9422950F946F96CD
:10FD70004B015C01C501B4010F94A29620911E02B3
:10FD800030911F0240912002509121020F94CD9892
:10FD90009B01AC01C701B6010F9423950F946F9698
:10FDA0006093D3107093D4108093D5109093D61095
:10FDB0000F947E466093D3107093D4108093D51027
:10FDC0009093D6104091E5065091E6067A010027FF
:10FDD000F7FC0095102F2B013C0197FF07C044242E
:10FDE00055243201461A570A680A790AE414F504C0
:10FDF000060517050CF522273327241B350B44274E
:10FE000037FD4095542F0F94C7446093D3107093DF
:10FE1000D4108093D5109093D6100091BB09109107
:10FE2000BC092091BD093091BE09601B710B820B8A
:10FE3000930B0F947E461AC00091BB091091BC0928
:10FE40002091BD093091BE09601B710B820B930B91
:10FE50000F947E4618EBE12E1BE0F12E00E010E03F
:10FE600028E434EF4FEF5FEF0F94C7446B017C0140
:10FE70008091C40C80FD04C0C12CD12C760106C039
:10FE80008091570790915807892BB1F36091BB0976
:10FE90007091BC098091BD099091BE096C0D7D1DCA
:10FEA0008E1D9F1D0F947E466093D3107093D410C7
:10FEB0008093D5109093D610B701A6018AE599E0FA
:10FEC0000E94F8D710929B12680D791D8A1D9B1D08
:10FED0006093B8127093B9128093BA129093BB12C8
:10FEE0006091D7107091D8108091D9109091DA104C
:10FEF0000F94A2966B017C016091380770913907CD
:10FF0000882777FD8095982F0F94A296209143081B
:10FF10003091440840914508509146080F94CD987F
:10FF20004B015C0120914F083091500840915108DD
:10FF300050915208C701B6010F94CD989B01AC01B6
:10FF4000C501B4010F9422950F946F964B015C018B
:10FF5000C501B4010F94A29620911E0230911F0298
:10FF600040912002509121020F94CD989B01AC0149
:10FF7000C701B6010F9423950F946F966093D71025
:10FF80007093D8108093D9109093DA100F947E4616
:10FF90006093D7107093D8108093D9109093DA1093
:10FFA0004091E5065091E6067A010027F7FC00959E
:10FFB000102F2B013C0197FF07C044245524320128
:10FFC000461A570A680A790AE414F5040605170563
:10FFD0000CF522273327241B350B442737FD40958A
:10FFE000542F0F94C7446093D7107093D810809308
:10FFF000D9109093DA100091BF091091C009209197
:020000021000EC
:10000000C1093091C209601B710B820B930B0F94D5
:100010007E461AC00091BF091091C0092091C10904
:100020003091C209601B710B820B930B0F947E46BB
:1000300018EBE12E1BE0F12E00E010E028E434EF95
:100040004FEF5FEF0F94C7446B017C018091C40CAC
:1000500080FD04C0C12CD12C760106C080915707C9
:1000600090915807892BB1F36091BF097091C00935
:100070008091C1099091C2096C0D7D1D8E1D9F1D3F
:100080000F947E466093D7107093D8108093D91048
:100090009093DA10B701A60188E699E00E94F8D79C
:1000A00010929B12680D791D8A1D9B1D6093C012D2
:1000B0007093C1128093C2129093C3120C948888DB
:1000C00080911D0E867029F080911E0E82FD0E9487
:1000D000AB5D609138077091390780911B07909153
:1000E0001C070E94E44E6091710D7091720D88277B
:1000F00077FD8095982F0E946C536091730D7091DD
:10010000740D882777FD8095982F0E942E5480913A
:100110007207909173072091380730913907409109
:100120001B0750911C0760919A05762F737011F090
:100130000C94B088EDC7232B11F4892B99F062FF42
:100140000E94422980919A05846080939A050E94BA
:10015000AA2A6093D9127093DA128093DB129093DB
:10016000DC1224C062FF22C00E94AA2A0091D91288
:100170001091DA122091DB123091DC12601B710BAE
:10018000820B930B653F71408105910578F080915A
:100190009A058B7980939A050E94AA2A6093CD12C2
:1001A0007093CE128093CF129093D01220919A0523
:1001B00022FDAEC7822F82958695837090E08130B4
:1001C000910509F428C18230910509F457C3892BA0
:1001D00009F09EC78091BB099091BC09A091BD090F
:1001E000B091BE09B7FF07C0B095A09590958195D5
:1001F0009F4FAF4FBF4F8D329140A105B105B4F471
:100200008091BF099091C009A091C109B091C20924
:10021000B7FF07C0B095A095909581959F4FAF4FC0
:10022000BF4F8D329140A105B10554F00E94AA2A1A
:100230006093CD127093CE128093CF129093D01210
:100240000E94AA2A0091CD121091CE122091CF12B5
:100250003091D012601B710B820B930B6A3F7105BA
:100260008105910508F454C780919A058F798062C1
:1002700080939A051092DD121092DE121092DF1216
:100280001092E0121092E1121092E2121092E31218
:100290001092E4120E94AA2A6093CD127093CE129B
:1002A0008093CF129093D0128091B4129091B51296
:1002B000A091B612B091B7128093C5129093C61256
:1002C000A093C712B093C8128091BC129091BD1236
:1002D000A091BE12B091BF128093C9129093CA121E
:1002E000A093CB12B093CC1280919C1290919D124E
:1002F000A0919E12B0919F128093931290939412AA
:10030000A0939512B093961280919A0583FD3FC0F9
:100310006091B7107091B8108091B9109091BA1097
:10032000609354087093550880935608909357082B
:100330002AE037ED43E25CE30F94CD9860935808D0
:100340007093590880935A0890935B088091BF106E
:100350009091C010A091C110B091C21080935C0820
:1003600090935D08A0935E08B0935F088091C310DE
:100370009091C410A091C510B091C61080935A09F5
:1003800090935B09A0935C09B0935D093EC06091B6
:10039000BB107091BC108091BD109091BE10609305
:1003A0006E0870936F0880937008909371082AE02C
:1003B00037ED43E25CE30F94CD986093720870933D
:1003C000730880937408909375088091C71090917A
:1003D000C810A091C910B091CA108093760890936C
:1003E0007708A0937808B09379088091CB1090910A
:1003F000CC10A091CD10B091CE108093680990934D
:100400006909A0936A09B0936B0980911F0E8260FD
:1004100080931F0E7DC6922F991F9927991F809157
:100420009B058170880F892B322F387020718330A3
:1004300071F5311116C0222319F080ED97E002C04A
:1004400080E398EF9093720D8093710D6091710D20
:100450007091720D882777FD8095982F0E946C53BC
:1004600072C0222319F080ED97E002C080E398EF7C
:100470009093740D8093730D6091730D7091740D52
:10048000882777FD8095982F0E942E545CC080911C
:10049000931290919412A0919512B09196123111ED
:1004A00024C0222329F048E253E260E070E004C057
:1004B00048ED5CED6FEF7FEF4093B4125093B512AF
:1004C0006093B6127093B7124091C9125091CA123C
:1004D0006091CB127091CC124093BC125093BD121C
:1004E0006093BE127093BF1223C0222329F048E20A
:1004F00053E260E070E004C048ED5CED6FEF7FEF29
:100500004093BC125093BD126093BE127093BF1201
:100510004091C5125091C6126091C7127091C812D5
:100520004093B4125093B5126093B6127093B71201
:1005300080939C1290939D12A0939E12B0939F1251
:1005400082E080939B1280919A054BE45AE06FE71A
:100550007AE083FD27C0CE0101960F94605547E5F0
:100560005AE0BE016F5F7F4FCE010D960F9460552C
:100570008D859E85AF85B889BC01CD019F770F948D
:10058000E64420E030E048EC52E40F94CD983B0183
:100590008C01C090BB09D090BC09E090BD09F090DF
:1005A000BE0926C0CE0101960F94605547E55AE07A
:1005B000BE016F5F7F4FCE010D960F946055898904
:1005C0009A89AB89BC89BC01CD019F770F94E64421
:1005D00020E030E048EC52E40F94CD983B018C01D0
:1005E000C090BF09D090C009E090C109F090C20945
:1005F000F7FE08C0F094E094D094C094C11CD11CC4
:10060000E11CF11C90919A05991F9927991F8091DF
:100610009B058170880F892B833009F04AC0C70180
:10062000B6010F94A2964B015C012091DD1230912E
:10063000DE124091DF125091E0120F947D9818164F
:1006400084F48092DD129092DE12A092DF12B092BA
:10065000E0128092E1129092E212A092E312B09224
:10066000E4122091E1123091E2124091E312509194
:10067000E412C501B4010F94009687FF6AC020E020
:1006800030E041EE54E46091DD127091DE12809111
:10069000DF129091E0120F947D9818160CF059C05B
:1006A0008092E1129092E212A092E312B092E412D0
:1006B00050C02091DD123091DE124091DF12509136
:1006C000E012662D772D802F912F0F947D981816AC
:1006D000A4F4862D972DA02FB12F8093DD12909337
:1006E000DE12A093DF12B093E0128093E112909398
:1006F000E212A093E312B093E4122091E112309140
:10070000E2124091E3125091E412662D772D802F72
:10071000912F0F94009687FF1CC020E030E041EE3F
:1007200055E46091DD127091DE128091DF1290919C
:10073000E0120F947D98181664F4862D972DA02F43
:10074000B12F8093E1129093E212A093E312B09341
:10075000E4120E94AA2A8090CD129090CE12A0900E
:10076000CF12B090D012681979098A099B09643FA9
:1007700071408105910530F080919A058F798064F0
:1007800080939A0590919A05292F221F2227221FD4
:1007900080919B058170880F822B833019F5C701EA
:1007A000B6010F94A29620E030E849E055E40F949A
:1007B0007D9887FF3EC02091E1123091E212409176
:1007C000E3125091E4126091DD127091DE1280917B
:1007D000DF129091E0120F94229520E030E048E47F
:1007E00053E423C0E0EDCE16E7E0DE06E104F104B9
:1007F00024F09F79906490939A05823000F52091BF
:10080000E1123091E2124091E3125091E4126091B2
:10081000DD127091DE128091DF129091E0120F9440
:10082000229520E030E041E654E40F947D981816BC
:1008300034F480919A058F79806480939A05BE0183
:10084000675E7F4F89E0FB0111928A95E9F783EAA1
:10085000898F85E98A8F8AE18B8FDD8ECC8E862DFC
:10086000972DA02FB12F8E8F9F8FA8A3B9A349E0FA
:1008700050E08DE89CE00F94BB7C4AC40E94C028E5
:1008800080919A05E090DD12F090DE120091DF1267
:100890001091E0122091E1123091E2124091E312A6
:1008A0005091E412982F991F9927991F83FD25C015
:1008B000A090B710B090B810C090B910D090BA10F6
:1008C00060919B056170660F692B9091C6109F9394
:1008D0009091C5109F939091C4109F939091C310D5
:1008E0009F939091C2109F939091C1109F9390916C
:1008F000C0109F939091BF1024C0A090BB10B090E7
:10090000BC10C090BD10D090BE1060919B0561706E
:10091000660F692B9091CE109F939091CD109F936D
:100920009091CC109F939091CB109F939091CA106F
:100930009F939091C9109F939091C8109F9390910D
:10094000C7109F9383FB882780F90E947C2E0FB6E7
:10095000F894DEBF0FBECDBF10919A05912F991F5D
:100960009927991F80919B058170880F892B09F029
:10097000BFC0C090DD12D090DE12E090DF12F09088
:10098000E01220E030EA4CE056E4C701B6010F94D3
:100990007D9818160CF4C2C020E030E041EE55E41A
:1009A000C701B6010F94009687FF32C013FD13C034
:1009B0008090B7109090B810A090B910B090BA1075
:1009C00020E030E040E85EE3C501B4010F940096FA
:1009D0001816A4F41DC08090BB109090BC10A0907D
:1009E000BD10B090BE1020E030E040E85EE3C501ED
:1009F000B4010F940096181634F40AC02AE037EDBB
:100A000043E25CE30FC12AE037ED43E25CE31BC144
:100A10002091E1123091E2124091E3125091E412E0
:100A2000C701B6010F94229520E030E041E654E47E
:100A30000F947D989091E51218160CF4A7C1191621
:100A40001CF491509093E51280919A052FE632E1C3
:100A500043E85AE383FD26C06091BF107091C01037
:100A60008091C1109091C2100F942395FB01462FE5
:100A70005F2F682F792F4093BF105093C010609361
:100A8000C1107093C2102FE832EC45E75CE38F0190
:100A9000BF010F947D9887FD85C28FE892ECA5E792
:100AA000BCE327C16091C7107091C8108091C91034
:100AB0009091CA100F942395FB01462F5F2F682F4A
:100AC000792F4093C7105093C8106093C91070934A
:100AD000CA102FE832EC45E75CE38F01BF010F94A9
:100AE0007D9887FD5FC28FE892ECA5E7BCE330C13B
:100AF000813009F036C1C090DD12D090DE12E09056
:100B0000DF12F090E01220E030EA4CE056E4C7013A
:100B1000B6010F947D9818160CF04EC02AE037ED00
:100B200043EA5BE313FD30C06091B7107091B810D9
:100B30008091B9109091BA100F942295FB01462F25
:100B40005F2F682F792F4093B7105093B8106093A0
:100B5000B9107093BA102AE037ED43E25CE38F01DD
:100B6000BF010F94009687FF1DC280919A05836094
:100B700080939A0582E20E94BD4280E00E945478F0
:100B800082E00E944278C4C26091BB107091BC1098
:100B90008091BD109091BE100F942295FB01462FBD
:100BA0005F2F682F792F4093BB105093BC10609338
:100BB000BD107093BE10CFCF20E030E041EE55E481
:100BC000C701B6010F94009687FF4AC013FD13C0FA
:100BD0008090B7109090B810A090B910B090BA1053
:100BE00020E030E040E85EE3C501B4010F940096D8
:100BF0001816A4F435C08090BB109090BC10A09043
:100C0000BD10B090BE1020E030E040E85EE3C501CA
:100C1000B4010F940096181694F422C02AE037ED20
:100C200043EA5BE3C501B4010F9423956093B710C9
:100C30007093B8108093B9109093BA10B3C12AE0A2
:100C400037ED43EA5BE3C501B4010F94239560934C
:100C5000BB107093BC108093BD109093BE10A2C1C6
:100C60002091E1123091E2124091E3125091E4128E
:100C7000C701B6010F94229520E030E041E654E42C
:100C80000F9400969091E51287FD80C019161CF410
:100C900091509093E51280919A052FE632E143E05E
:100CA0005AE383FD2FC06091BF107091C0108091F6
:100CB000C1109091C2100F942295FB01462F5F2F17
:100CC000682F792F4093BF105093C0106093C110CC
:100CD0007093C2102FE632E143E85BE38F01BF015E
:100CE0000F94009618160CF45DC18FE692E1A3E80C
:100CF000BBE38093BF109093C010A093C110B0933A
:100D0000C2104AC16091C7107091C8108091C9107B
:100D10009091CA100F942295FB01462F5F2F682FE8
:100D2000792F4093C7105093C8106093C9107093E7
:100D3000CA102FE632E143E85BE38F01BF010F9455
:100D4000009618160CF42EC18FE692E1A3E8BBE3DF
:100D50008093C7109093C810A093C910B093CA1085
:100D60001BC1823009F07FC020E030EA4CE056E43D
:100D70006091DD127091DE128091DF129091E0128D
:100D80000F947D989091E512181624F49F5F90932C
:100D9000E51208C119161CF491509093E512809148
:100DA0009A052AE037ED43EA5BE383FD2EC06091AC
:100DB000B7107091B8108091B9109091BA100F943B
:100DC0002395FB01462F5F2F682F792F4093B71093
:100DD0005093B8106093B9107093BA1020E030E0CF
:100DE00040E85EE38F01BF010F947D9887FDDAC074
:100DF00080E090E0A0E8BEE38093B7109093B81035
:100E0000A093B910B093BA10C7C06091BB10709195
:100E1000BC108091BD109091BE100F942395FB01E2
:100E2000462F5F2F682F792F4093BB105093BC1033
:100E30006093BD107093BE1020E030E040E85EE3A8
:100E40008F01BF010F947D9887FDACC080E090E0DA
:100E5000A0E8BEE38093BB109093BC10A093BD109C
:100E6000B093BE1099C0833009F09CC0C090DD12D1
:100E7000D090DE12E090DF12F090E01220E030E837
:100E800049E055E4C701B6010F947D981816A4F007
:100E90002091E1123091E2124091E3125091E4125C
:100EA000C701B6010F94229520E030E048E453E4F6
:100EB0000F947D98181634F48091E5128F5F80931B
:100EC000E51270C08091E51218161CF481508093D1
:100ED000E51280919A0520E030E040E05FE383FD79
:100EE0002EC06091C3107091C4108091C510909174
:100EF000C6100F942395FB01462F5F2F682F792F83
:100F00004093C3105093C4106093C5107093C610E3
:100F100020E030E040E751E48F01BF010F947D985D
:100F200087FD40C080E090E0A0E7B1E48093C3106B
:100F30009093C410A093C510B093C6102DC06091BB
:100F4000CB107091CC108091CD109091CE100F9459
:100F50002395FB01462F5F2F682F792F4093CB10ED
:100F60005093CC106093CD107093CE1020E030E001
:100F700040E751E48F01BF010F947D9887FD12C0B7
:100F800080E090E0A0E7B1E48093CB109093CC1088
:100F9000A093CD10B093CE1084E08093E51283E24D
:100FA0000E94BD4280919A0584FB992790F921E027
:100FB000922790FB84F980939A059091E5129430E2
:100FC0000CF497C01092E512382F331F3327331FCC
:100FD00020919B05922F9170990F932B933061F084
:100FE0009F5F90FB87F980939A05969591702E7F6D
:100FF000292B20939B057DC0182F1F7710939A05EE
:101000002E7F20939B0520E030E040E45FE383FDEA
:1010100016C06091C3107091C4108091C51090915A
:10102000C6100F94CD986093C3107093C410809332
:10103000C5109093C610186010939A055AC060911D
:10104000CB107091CC108091CD109091CE100F9458
:10105000CD983B014C015B016C01E090C310F09016
:10106000C4100091C5101091C610762F272F372D70
:10107000482D592D6E2D7F2D802F912F0F94009686
:1010800087FD02C0730184018E2D9F2DA02FB12FEB
:101090008093C3109093C410A093C510B093C61052
:1010A000262D372D482D592D6E2D7F2D802F912FD8
:1010B0000F94009687FF02C0570168018A2D9B2D6F
:1010C000AC2DBD2D8093CB109093CC10A093CD1060
:1010D000B093CE1080919A058C7F826080939A05A0
:1010E00081E00E94427881E20E94BD4280E00E943D
:1010F000547880919A058F7980939A050E94AA2A44
:101100006093CD127093CE128093CF129093D01231
:101110008091550790915607892B31F480916D107D
:10112000823014F40E94BC3E80911E0E82FF1EC0CD
:101130008B7F80931E0E1AC01092D1121092D21281
:101140001092D3121092D4120C94B47B1092D51238
:101150001092D6121092D7121092D8120C94AF7C23
:10116000452B11F00C949F800C949B80A196E0E19C
:101170000D94559BACE0B0E0E0ECF8E80D94459B95
:1011800080911511823009F483C030F4882369F00E
:10119000813009F0FFC043C0843009F4DDC008F499
:1011A00091C0853009F0F6C0F0C082E00E9454780A
:1011B00083E00E94856083E00E94163181E00E94F6
:1011C0008B5D0E94AE6D0E94712A19821A821B8269
:1011D0001C821D821E821F8218860F94A296698728
:1011E0007A878B879C87BE016F5F7F4F81E29EE08D
:1011F0000E94ACD781E29EE00E9411D260930D1153
:1012000070930E1180930F11909310116093111130
:1012100070931211809313119093141137C0809121
:10122000210E80FFDBC083E00E9416310E94712AEC
:1012300019821A821B821C821D821E821F821886BE
:101240000F94A29669877A878B879C87BE016F5F10
:101250007F4F81E29EE00E94ACD781E29EE00E9437
:1012600011D260930D1170930E1180930F11909312
:1012700010116093111170931211809313119093B8
:10128000141181E00E948B5D0E94AE6D82E0A4C0CB
:101290008091210E80FFA2C00E94AA2A609316119D
:1012A00070931711809318119093191181E00E9487
:1012B0008B5D882311F089E001C080E00E94AE6D53
:1012C00083E08AC00E94AA2A00911611109117117A
:1012D0002091181130911911601B710B820B930B27
:1012E0000091F3061091F4062091F5063091F60670
:1012F000061717072807390708F070C08091E00625
:101300009091E106009709F447C02091901021FDCB
:1013100043C066C083E00E9416316091E006709180
:10132000E106882777FD8095982F0F94A296198261
:101330001A821B821C821D821E821F821886698768
:101340007A878B879C87BE016F5F7F4F81E29EE02B
:101350000E94ACD784E040C08091E0069091E10605
:10136000AA2797FDA095BA2F409101115091021123
:10137000609103117091041184179507A607B707B0
:101380004CF48091210E81703EC080911E0E869596
:10139000817039C081E037C085E00E94547882E0D6
:1013A0000E94163119821A821B821C821D821E82A3
:1013B0001F82188619861A861B861C86BE016F5FDF
:1013C0007F4F81E29EE00E9470C480E00E94AE6D7B
:1013D00084E00E94856085E08093151180E013C051
:1013E000AA2797FDA095BA2F4091011150910211A3
:1013F000609103117091041184179507A607B70730
:101400000CF0A8CF87CF2C96E4E00D94619BA4E26A
:10141000B0E0EDE0FAE80D94399B8091DB10809309
:10142000EC0620910D0730910E0730FF04C06EEEE0
:1014300070E10E94002F0E94E52A8091EE10833116
:1014400009F4E2C148F4813109F4CFC008F05AC16F
:10145000803109F077C262C0853109F4C1C008F457
:101460006EC2863109F06EC282E00E94547880E03C
:101470000E94AE6D83E00E94856083E00E94163179
:101480008CE0EEE7FCE0DE01119601900D928A956A
:10149000E1F7E984FA844B845C846091F1107091E7
:1014A000F2108091F3109091F4100F94A2963B01EA
:1014B0008C01762F272F372D402F512F6E2D7F2D0A
:1014C000842D952D0F947D98181614F43701820100
:1014D00020E030E048EC52E4662D772D802F912FEC
:1014E0000F947D98181624F0612C712C08EC12E4EE
:1014F000862D972DA02FB12F89879A87AB87BC8720
:10150000BE016F5F7F4F81E29EE00E94ACD70E94D8
:10151000BC3E0E94E13E0E94C83E14C282E00E948E
:10152000547883E00E94856083E00E9416318090A9
:10153000EE109090EF10A090F010B090F110C090CD
:10154000F210D090F310E090F410F090F5100091AC
:10155000F6101091F7102091F8103091F910409189
:10156000FA105091FB106091FC10CE0101960E9480
:10157000EA6CBE016F5F7F4F81E29EE00E94ACD7B4
:1015800081E29EE00E9411D260930D1170930E11C2
:1015900080930F1190931011609311117093121199
:1015A000809313119093141110926511109266118B
:1015B00010926711109268118091F01090E0909352
:1015C0006A1180936911892B29F48091210E826020
:1015D0008093210E80E00E948B5D0E94AE6DB2C1AF
:1015E0008EEE90E10E94B079ADC11D8A1E8A1F8ADD
:1015F000188E198A1A8A1B8A1C8A1D861E861F86C7
:10160000188A82E00E94547883E00E94856080E01E
:101610000E94AE6D8CE0EEE7FCE0DE0111960190D9
:101620000D928A95E1F78091F5109091F610A091B6
:10163000F710B091F810892B8A2B8B2BC9F480916D
:10164000F9109091FA10A091FB10B091FC10892B29
:101650008A2B8B2B69F49E01235F3F4F46E65CE0AB
:10166000BE016F5F7F4F81E29EE00E9461C32BC08D
:101670008090EE109090EF10A090F010B090F110CC
:10168000C090F210D090F310E090F410F090F510AC
:101690000091F6101091F7102091F8103091F91088
:1016A0004091FA105091FB106091FC10CE014996C8
:1016B0000E94EA6C8CE0FE017996DE011D96019095
:1016C0000D928A95E1F78091F1109091F210A0911E
:1016D000F310B091F410892B8A2B8B2B41F4898560
:1016E0009A85AB85BC858D8B9E8BAF8BB88F83E045
:1016F0000E941631BE01635F7F4F81E29EE00E942F
:10170000ACD720C182E00E94547883E00E948560BB
:1017100081E00E9416316091F1107091F210809179
:10172000F3109091F410611571058105910551F048
:101730000F94A2966093780E7093790E80937A0E30
:1017400090937B0E8091F5109091F610A091F71078
:10175000B091F810892B8A2B8B2B61F48091F910B2
:101760009091FA10A091FB10B091FC10892B8A2B5C
:101770008B2BD1F14090B7095090B8096090B9090E
:101780007090BA098090EE109090EF10A090F01039
:10179000B090F110C090F210D090F310E090F410DF
:1017A000F090F5100091F6101091F7102091F810BC
:1017B0003091F9104091FA105091FB106091FC109B
:1017C000CE0101960E94EA6C63015201E980FA8021
:1017D0000B811C812D813E814F81588569857A85D9
:1017E0008B859C850E94672F84E00E94AE6D1092CD
:1017F0003F111092401110924111109242118091AC
:10180000F01080936B119EC01D8A1E8A1F8A188E4D
:10181000198A1A8A1B8A1C8A1D861E861F86188AA8
:1018200082E00E94547883E00E94856080E00E94FC
:10183000AE6D8CE0EEE7FCE0DE01119601900D92BA
:101840008A95E1F78091F5109091F610A091F7102C
:10185000B091F810892B8A2B8B2BC9F48091F91049
:101860009091FA10A091FB10B091FC10892B8A2B5B
:101870008B2B69F49E01235F3F4F46E65CE0BE017F
:101880006F5F7F4F81E29EE00E9461C32BC080901A
:10189000EE109090EF10A090F010B090F110C0906A
:1018A000F210D090F310E090F410F090F510009149
:1018B000F6101091F7102091F8103091F910409126
:1018C000FA105091FB106091FC10CE0149960E94D5
:1018D000EA6C8CE0FE017996DE011D9601900D9276
:1018E0008A95E1F78091F1109091F210A091F31098
:1018F000B091F410892B8A2B8B2B41F489859A8522
:10190000AB85BC858D8B9E8BAF8BB88F83E00E949F
:101910001631BE01635F7F4F81E29EE00E94ACD72B
:101920001092651110926611109267111092681151
:101930008091F0108093691110926A1103C0109287
:10194000151118DC1092DD10A496E0E10D94559B62
:10195000AFE0B0E0EEEAFCE80D94469B182F8091D2
:101960006D10833031F58091EB06482F552747FDE8
:101970005095212F30E02417350714F0182F1150FF
:10198000612F70E0CE0101960E941142898180365C
:1019900080F40E94622A8FE0FE013196AEEEB0E143
:1019A00001900D928A95E1F71093DB101092DC10F4
:1019B0002EDD2F96E3E00D94629BCF93DF93C82F2B
:1019C000D091C40CD095D17090E020916D10332748
:1019D00027FD30958217930709F400C1FC01EE3012
:1019E000F10508F0FDC0EC54FF4F0D946E9B81E0B3
:1019F0000E94AE6D81E00E94547880E0E5C080E0F6
:101A00000E94AE6D80E00E94547881E0DDC080E0ED
:101A10000E94AE6D80E0D5C08091C20581FDE0C01E
:101A20000E94342C882329F08091EB0682300CF040
:101A300090C0D1118EC0D4C08091C20581FDD0C0AC
:101A40000E94342C811188C0D11186C0C9C08091F8
:101A5000C20581FDC5C00E94342C81118AC0D111FC
:101A600088C0BEC08091C20581FDBAC00E94342CDE
:101A7000811187C0D11185C0B3C08091C20581FD9D
:101A8000AFC00E94342C811187C0D11185C0A8C07D
:101A900080E090E00E94B0799CC00E94342C8111BB
:101AA00088C0D11186C09CC08091C20581FD98C0BC
:101AB0008091DE06811181C0D1117FC091C088E084
:101AC0000E94AE6D84E00E94547880E00E9416313E
:101AD00081E00E9485607DC080E00E94AE6D86E05E
:101AE0000E94547882E00E94856080E00E94163156
:101AF0004091BB095091BC096091BD097091BE092C
:101B00004093D3105093D4106093D5107093D61097
:101B10004091BF095091C0096091C1097091C209FB
:101B20004093D7105093D8106093D9107093DA1067
:101B30004091C3095091C4096091C5097091C609CB
:101B40004093750D5093760D6093770D7093780DDB
:101B500040C00E94622A3DC082E00E94547882E028
:101B60000E94856081E00E94163184E00E94AE6D83
:101B700030C080E00E94AE6D85E00E94547882E023
:101B800007C080E00E94AE6D85E00E94547881E03D
:101B90000E94856082E01BC080E00E948B5D0E94F5
:101BA000AE6D82E00E94547883E00E94856083E0FD
:101BB0000EC010921511DEDA0CC080E00E94AE6DEE
:101BC00083E00E94547882E00E94856080E00E9459
:101BD0001631C0936D108C2F0E94422F81E005C0FA
:101BE0006C2F8AE00E941D2E80E0DF91CF91089536
:101BF000CF93C82F9091901091FB882780F98C1774
:101C000009F46BC0C0FB91F99093901091FD02C054
